:100000000C948C110C94BD110C94BD110C94BD1169
:100010000C94BD110C94BD110C94BD110C94BD1128
:100020000C94BD110C94BD110C94BD110C94BD1118
:100030000C94BD110C94BD110C94BD110C94BD1108
:100040000C94BD110C94BD110C94BD110C94BD11F8
:100050000C94BD110C94BD110C94BD110C948BC16A
:100060000C94BD110C94D59C0C94AB9C0C94BD11BC
:100070000C94BD110C94BD110C94BD110C94BD11C8
:100080000C94BD110C94BD110C94BD110C94BD11B8
:100090000C94819C0C94579C0C94BD110C940121E0
:1000A0000C94BD110C94BD110C94BD110C94BD1198
:1000B0000C94BD110C94BD110C94BD110C94BD1188
:1000C0000C94BD110C94BD110C94BD110C942D9C7D
:1000D0000C94039C0C94BD110C94D99B0C94AF9B75
:1000E0000C94BD1107634236B79BD8A71A396856DE
:1000F00018AEBAAB558C1D3CB7CC5763BD6DEDFD4A
:10010000753EF6177231BF000000803F0800000006
:10011000BE922449123EABAAAA2ABECDCCCC4C3EFC
:1001200000000080BEABAAAAAA3E00000000BF00EB
:100130000000803F0000000000084178D3BB4387E7
:10014000D1133D190E3CC3BD4282AD2B3E68EC82FB
:1001500076BED98FE1A93E4C80EFFFBE01C4FF7F80
:100160003F00000000000C94DE170C94B72A0C949A
:10017000983F0C94A5640C94D9110C94B22A0C9459
:10018000F25B0C94F25C0C94E72E0C94A1640C943A
:1001900029130C945A340C94C6650C9495890C94CC
:1001A000BF110C9408610C94B7BB0C9415310C94DE
:1001B000D9150C94825B0C9479790C9401910C9470
:1001C00062640C9424990C9420610C9453E30C9475
:1001D00078650C94C5770C94D4170C94A35F0C9499
:1001E00078130C943D130C9401650C9497130C94A4
:1001F00078BA0C9452150C94285F0C941DBB0C9487
:100200006A650C9479160C94025F0C94646F0C94DC
:1002100004920C94F52F0C94041E0C947F340C94CF
:100220006A910C9470BA0C94D6170C943B350C94CC
:10023000DB5E0C9407180C9434BB0C94D9240C94FA
:10024000D0620C9497240C94D65B0C9489650C9422
:100250005C650C94D25B0C94A48E0C94CE7E0C94B2
:1002600032BA0C94F3780C94EF110C9404340C947F
:100270001F910C9431300C943CBA0C94711A0C946C
:1002800005310C943A130C943C800C94CC620C9481
:100290009E190C94DC620C9492890C943D7E0C9413
:1002A000DA170C947C130C9400660C945B830C940A
:1002B00082240C94B62A0C94009F0C9457830C94BF
:1002C00059130C94EE790C9412190C9443300C943D
:1002D000DB5B0C9498300C94F6120C9419300C944F
:1002E000F4810C941B8F0C9454BA0C9485880C9454
:1002F0002C130C940E140C9474BA0C941B8E0C9446
:10030000D8170C942B1C0C9415D60C9473620C9477
:1003100026900C94FA110C9474610C948B150C9427
:1003200055830C94A9160C9414730C94F22B0C9412
:100330001E820C94B5450C94806D0C948FBB0C946C
:10034000BB790C940F370C947C340C94EF5E0C94B6
:10035000D8130C94D91C0C94E8120C942ABB0C945E
:1003600042650C94DE6E0C9450BA0C9461780C9437
:1003700076BB0C94D3630C942E910C94B59E0C9484
:1003800082160C94815E0C94F2870C94DC170C940A
:100390003EBB0C94D01F0C9450780C946C440C947D
:1003A000D2620C943F880C94B6770C94C6230C94BC
:1003B00083140C944B9F0C940B880C947ACD0C9462
:1003C000D66E0C94181F0C947A6D0C94CA620C941F
:1003D00047240C94BA5B0C941D900C9448BB0C946D
:1003E0001BD60C946C880C94EA6D0C94855B0C9471
:1003F000507F0C94F8330C94155C0C94335F0C9480
:10040000496C0C94776D0C9462BA0C94CD640C9486
:10041000959E0C9420900C9441980C9484650C94B7
:1004200080D00C9468920C94D7770C946D130C9434
:1004300044130C94CED60C9458BB0C94715F0C945E
:100440003F820C941C920C94EF230C9450BB0C94A0
:1004500086240C9470150C9403810C94C75F0C9443
:1004600090130C94EA8E0C9499BB0C946C240C940D
:100470001C130C94382D0C947F310C9471910C94B6
:1004800068200C947E240C9446BA0C949E9E0C9486
:100490006ED10C9495640C94DD640C949A800C9449
:1004A000C45B0C946F5B0C94BC1D0C94BC870C94C7
:1004B00064310C9424130C940C1A0C94D5700C9485
:1004C000D36E0C94A5D60C94ADBB0C947A140C94FA
:1004D000EC1C0C94255F0C94D85B0C9496810C94C6
:1004E00038BA0C9461130C94A1220C9416900C94BD
:1004F00082590C947F5B0C94A3BB0C94B21A0C949D
:1005000057640C94D4620C9462BB0C949D160C94AA
:10051000C0D60C94D5110C9428D60C9415D50C94F7
:10052000994A0C94E9880C9425BB0C94FB120C940A
:1005300064160C9437890C94129F0C9438650C94B3
:1005400078640C9480130C94B12A0C94231D0C94A1
:100550001A730C94EC180C9421130C94DA620C941A
:1005600056610C94F3920C94DF140C946B130C945E
:100570005EBA0C94B52A0C94A38E0C94B7150C9407
:100580004F610C94E0240C94A1A00C940D8F0C945A
:1005900001200C942F610C94E5130C9417650C94B6
:1005A0006CBB0C946CBA0C94708F0C94CE620C944F
:1005B00062600C94A8230C94BBCE0C9493200C94F2
:1005C000AF900C945C610C9463900C94365F0C9427
:1005D0002B470C9466BA0C9458910C944ABA0C941C
:1005E000C61C0C94B6630C946A680C94D3330C94B8
:1005F000D8620C949A5B0C9499650C9449D60C942F
:1006000026E30C948F890C94195F0C94445E0C942F
:10061000E4910C94FC8F0C9477BA0C94C5780C94EC
:10062000905F0C9470130C94C9650C949B310C94DE
:10063000E36D0C940B730C94849E0C9431250C94F4
:10064000C2CE0C9440BA0C94E9630C94F98E0C94CD
:1006500065610C9457140C9484240C9428610C94B8
:10066000D47F0C945D130C94C7880C9449810C942E
:1006700058BA0C9471140C9485BB0C9402890C9498
:1006800011610C94961F0C9423810C9480CD0C94D2
:1006900024250C9427240C949B630C94B6890C9409
:1006A000DB330C94981A0C94F4130C9438200C94AB
:1006B00096900C94D96E0C94425F0C94085C0C9448
:1006C00058230C94D0630C94EC240C94D2700C94AA
:1006D00086870C94D6620C94E34A0C94885B0C9445
:1006E00076240C942D140C94B72B0C94D06E0C948F
:1006F0003D360C949A650C94B78F0C9420660C943C
:10070000918E4E414E494E495459494E46CDCCCC1E
:100710003D0AD7233C17B7D13877CC2B329595E6D5
:10072000241FB14F0A000020410000C84200401CB5
:100730004620BCBE4CCA1B0E5AAEC59D746364698C
:100740006E6F70737578585B0053617665643A001C
:1007500020537566663A002041543A00436F6E6636
:100760006967206368616E676564206C6F63616CA4
:100770006C792C20706F7274616C20646973616293
:100780006C6564002F636F6E6669672E6A736F6EA7
:10079000007265626F6F742000436D643A20002F11
:1007A000636F6D6D616E642F002F72616D2F002F6E
:1007B0006974656D2F002F6974656D2F004C6F6330
:1007C0006174696F6E3A20687474703A2F2F6C618F
:1007D0007A79686F6D652E72752F707761003F6D45
:1007E00061633D002669703D0026706F72743D00A4
:1007F000266E616D653D002F002000436F6D706CAB
:100800006574652E2052656D6F766520746F706912
:1008100063200024636F6D6D616E6400536B6970BB
:1008200070696E672E2E00436C65616E5570207284
:10083000657461696E656420746F7069632000225D
:100840000022004F75744F664D656D6F72792100FF
:100850005D20003A5B000A005D00456D7074793AD6
:10086000205B000A003A004D41433A0055445020B5
:100870005379736C6F6720696E697469616C697A0A
:1008800065642E0A005379736C6F67207061726122
:100890006D733A002E6C6F63616C005365727669FC
:1008A0006365207265636F72643A20006D444E5335
:1008B00020726573706F6E646572207374617274F8
:1008C00065642E004572726F722073657474696E70
:1008D00067207570204D444E5320726573706F6EA3
:1008E0006465722100476F7420495020616464720E
:1008F0006573733A00276970205B69705B2C646EC6
:10090000735B2C67775B2C7375626E65745D5D5DE0
:100910005D27202D207365742073746174696320D2
:1009200049500A004661696C656420746F20636FEA
:100930006E6669677572652045746865726E657468
:10094000207573696E6720444843502E20596F7597
:100950002063616E20736574206970206D616E750F
:10096000616C6C792100204D41534B3A0020475770
:100970003A0020444E533A004C6F6164656420662F
:10098000726F6D20666C6173682049503A000A7579
:1009900073657320444843500A005374617274694C
:1009A0006E67206C616E0043757272656E74204CC8
:1009B000414E20636F6E6669672869702C646E73A0
:1009C0002C67772C7375626E6574293A000A55732B
:1009D0006520746865736520636F6D6D616E647307
:1009E0003A202768656C7027202D20746869732071
:1009F000746578740A276D61632064653A61643AAE
:100A000062653A65663A66653A30302720736574E8
:100A100020616E642073746F7265204D41432D61B7
:100A200064647265737320696E20454550524F4D62
:100A30000A276970205B69705B2C646E735B2C679E
:100A4000775B2C7375626E65745D5D5D5D27202D2F
:100A500020736574207374617469632049500A2798
:100A60007361766527202D2073617665206375722A
:100A700072656E7420636F6E66696720696E204EC2
:100A80005652414D3B204F4E7C4F4646202D20650F
:100A90006E61626C652F64697361626C652061755B
:100AA000746F736176650A2767657427205B636FCF
:100AB0006E66696720616464725D27202D2067651A
:100AC0007420636F6E6669672066726F6D20707246
:100AD000652D636F6E666967757265642055524C4B
:100AE00020616E642073746F726520616464722C7F
:100AF000204F4E7C4F4646202D20656E61626C650E
:100B00002F64697361626C6520646F776E6C6F61CE
:100B100064206F6E20737461727475700A276C6F35
:100B2000616427202D206C6F616420636F6E66699D
:100B3000672066726F6D204E5652414D0A277077BE
:100B40006427202D20646566696E6520616E6420CF
:100B500073746F7265204D515454207061737377B4
:100B60006F72640A276F746170776427202D206488
:100B70006566696E6520616E642073746F726520AE
:100B800048545450204150492070617373776F72FC
:100B9000640A276C6F67205B73657269616C5F6CB8
:100BA0006F676C6576656C5D205B7564705F6C6FFC
:100BB000676C6576656C5D27202D20646566696EBF
:100BC00065206C6F67206C6576656C2028302E2E52
:100BD00037290A276B696C6C27202D207465737484
:100BE000207761746368646F670A27636C6561725C
:100BF00027202D20636C65617220454550524F4D72
:100C00000A277265626F6F7427202D207265626FEC
:100C10006F7420636F6E74726F6C6C657200536FCB
:100C20006674207265626F6F74696E672E2E2E0077
:100C300052414D3D000A5379736C6F6720000A6D75
:100C400071747420000A696E7075747320000A69EB
:100C500074656D7320000A436F6E6669677572650F
:100C6000643A003B003D0050696E3A003B003D4C49
:100C70004F5700546865726D6F3A004170706C791F
:100C8000696E6720636F6E666967004C6F616465AB
:100C90006420455441473A004E6F2073746F72656B
:100CA0006420636F6E666967004C6F6164656420E1
:100CB00066726F6D20454550524F4D006C6F6164F8
:100CC000206661696C656400547279696E67204CB6
:100CD0006F61642066726F6D20454550524F4D0024
:100CE0004C6F6164696E6720436F6E66696720664A
:100CF000726F6D20454550524F4D00436F6E6669CF
:100D000067206175746F736176653A000A53797371
:100D10006C6F67206465627567206C6576656C3AF8
:100D20000053657269616C206465627567206C654B
:100D300076656C3A0053617665640A0053657420E9
:100D400064796E616D69632049500A0045455052CF
:100D50004F4D20636C65617265640A004D515454B7
:100D60002050617373776F7264207570646174656D
:100D7000640A004F54412050617373776F7264208E
:100D8000757064617465640A00636F756C64206ECD
:100D90006F742070617273653A20005570646174DD
:100DA00065640A004E6F2049502061647265737358
:100DB0000052656C656173696E6720736F636B6564
:100DC0007420616E642072657472790020536176BC
:100DD0006564004C6F6164696E672048545450200C
:100DE000636F6E666967206F6E20737461727475CD
:100DF000703A004F4646004F4E002B002D004554E0
:100E000061673A200047657420455441473A200005
:100E1000485454502F312E310025733A2025730D3C
:100E20000A0020485454502F312E310D0A486F7358
:100E3000743A2025730D0A4163636570743A202A61
:100E40002F2A0D0A436F6E6E656374696F6E3A20C8
:100E5000636C6F73650D0A0025730020000D0A0096
:100E6000474554006661696C656420746F20636F48
:100E70006E6E6563740A004552524F523A205365B4
:100E8000727665722072657475726E6564200043B7
:100E90006F6E666967206E6F74206368616E676548
:100EA000640A00446F6E652E0A00436F6E666967C0
:100EB0002070617273696E67206661696C65640A8F
:100EC00000676F7420436F6E6669670A0068747408
:100ED0007020726574636F646520006672656520BA
:100EE00000436F6E666967205552493A20687474F2
:100EF000703A2F2F002044656661756C7420636F13
:100F00006E666967207365727665722075736564B5
:100F10003A20006C617A79686F6D652E7275000AEF
:100F2000282B29454C455641544F52000A4E4F53E9
:100F3000455249414C000A282B294D554C544956DD
:100F4000454E54000A282B2950574D5F52454C41BD
:100F500059000A282B294D444E53000A282D2955A3
:100F6000415254425249444745000A282B295359BB
:100F7000534C4F47000A282D29504944000A282D78
:100F8000294D43503233303137000A282D29415240
:100F9000544E4554000A282B294F5441000A282D4D
:100FA00029535049204C4544000A282D294D4F54BF
:100FB0004F5220435452000A282B294143204841D4
:100FC000494552206F6E2053657269616C33000A87
:100FD000282D2943435338313120262048444331BA
:100FE000303830000A282B29524553544152545F5F
:100FF0004C414E5F4F4E5F4D5154545F4552524FDE
:101000005253000A282D2948415244524553455411
:101010002C207573696E6720736F6674000A282D23
:1010200029434F554E544552000A282D294448540F
:10103000000A282D294F57495245000A282D2949D1
:10104000504D4F44425553000A282D294D4F4442DC
:101050005553000A282D29444D58000A282B29579A
:10106000697A6E657435783030000A282B2946720B
:10107000656552616D207072696E74696E67000AF1
:10108000282B295741544348444F47006C617A79D3
:10109000686F6D652E7275000A436F6E6669672012
:1010A0007365727665723A003230313730334C00F6
:1010B00020432B2B2076657273696F6E3A0065634F
:1010C00033303663345F323032332D30342D3032AA
:1010D000000A4C617A79686F6D652E7275204C69D3
:1010E00067687448756220636F6E74726F6C6C65AC
:1010F000722000204F464600204F4E00204259509B
:1011000041535300757074696D650066726565685A
:10111000656170002054696D65723A00204C6F6300
:101120006B733A002000204C6F636B733A000A52D5
:10113000414D3D0020457870697265640A00202D9C
:10114000746172676574207A6F6E652D0020416C42
:1011500061726D20457870697265640A0020636D64
:10116000643A00204375723A00205365743A005384
:101170006176656420746F20454550524F4D005391
:101180006176696E6720636F6E66696720746F2091
:10119000454550524F4D2E2E002069732000446566
:1011A0006C6574696E6720636F6E662E2052414DC8
:1011B000207761733A0053746F70706564005374E4
:1011C0006F7070696E67206368616E6E656C732006
:1011D0002E2E2E004E6F7420756E6C6F636B6564DF
:1011E00020696E20313073202D20636F6E74696E1C
:1011F0007565202E2E2E00556E6C6F636B696E67C1
:1012000020636F6E666967202E2E2E00203C3C0006
:10121000416972436F6E200053657269616C20757D
:10122000736564206279204143202D2064697361D5
:10123000626C696E672073657269616C206C6F67A0
:1012400067696E6720616E6420636D6400414320AE
:10125000496E69743A200041432044652D496E6906
:10126000743A2000455252004452590046414E5FA4
:101270004F4E4C59004845415400434F4F4C0020BD
:101280004F4B00203E3E2000416972436F6E2000AC
:10129000506F6C6C696E67004C4F57004D45444968
:1012A000554D0048494748004155544F00726177F9
:1012B000007175656974007377696E67006C6F63A0
:1012C0006B0044656661756C742073657269616C4E
:1012D000206D6F6465204E38312075736564003869
:1012E0004531002600384E31000600384532002EC8
:1012F00000384E32000E00384F31003600384F3281
:10130000003E00374531002400374532002C0037BD
:101310004F31003400374F32003C00374E3100046B
:1013200000374E32000C002C002C002C002C004505
:101330006C657661746F723A20636F6E66696720C0
:101340006661696C65643A00456C657661746F72BC
:1013500020636F6E666967206572726F7200456CFC
:10136000657661746F7220636F6E666967206C6F5B
:10137000616465642000456C657661746F723A2023
:101380004F7574206F66206D656D6F727900456CC6
:10139000657661746F722044652D496E69740040F2
:1013A00030305252303030303031303033463030DF
:1013B00034313043303034322A00403030525230F1
:1013C00030303030323030374630303032313030FB
:1013D0003033302A004030305252303030303034E8
:1013E00030303346303038343134303033382A00FE
:1013F0003C003E00556E6B6E6F776E2073756666AF
:1014000069782000556E6B6E6F776E20636D642077
:1014100000536574206E6F7420696D706C656D6526
:101420006E74656400466F726365642065786563F9
:101430007574696F6E00556E6B6E6F776E20737585
:101440006666697800454C45563A20004D756C74C7
:101450006956656E7420636F6E66696720666169A0
:101460006C6564004D756C746956656E7420696EA8
:101470006974004D756C746976656E742044652DD1
:10148000496E697400204F75743A00206D33002056
:1014900066726F6D2000204D6178207265717565F0
:1014A00073743A002066616E253A002061637469A6
:1014B000766520563A00546F74616C20563A0020CD
:1014C000696E69740050574D2D4F757420230020AC
:1014D00073746F700050574D2D4F75742023003D6D
:1014E0000050696E3A0020696E69740052656C6143
:1014F000792D4F75742023002073746F700052652E
:101500006C61792D4F75742023003D3E003A0070C8
:10151000756220616374696F6E200069646C650098
:101520006F66660068656174696E670066616E006B
:10153000647279696E6700636F6F6C696E67002013
:10154000697320004F75742000556E6B6E6F776E57
:10155000207375666669782000556E6B6E6F776EC6
:1015600020636D642000616374696F6E0072656C46
:1015700061794374723A20005B305D3A2000202D7F
:10158000202D202D20EFBBBF003E003E31202D201E
:101590000020002E00696E00735F6F7574006D7916
:1015A000686F6D65004354524C2F657865633A202F
:1015B0004F75744F664D656D6F72793A2000202D1E
:1015C0003E2000456D69743A2000202D3E200049E0
:1015D00074656D436D643A2000202D3E20004974EF
:1015E000656D3A2000556E6B6E6F776E2073756671
:1015F0006669782000556E6B6E6F776E20636D6440
:101600002000636C724374723A2000454F46002FED
:1016100000496E3A20003D00494E3A003D004C45DD
:101620004741435920494E3A00000020002300263C
:101630000029002C002F00320000010000030106E9
:101640000109012D3E00200023002D3E0020005006
:10165000656E6465643A2023007261770076616C80
:101660000074656D70007361740068756500666173
:101670006E0052474200485356006D6F6465005338
:101680006574436D643A0053746F72656420455805
:10169000543A00737566666978436F64653A002052
:1016A000666F7220286D73293A004354524C3A20D9
:1016B0005363686564756C6520636D642000206DFC
:1016C00073203A0041726D656420666F72200020BD
:1016D00044697361726D656400584F4E0048414C17
:1016E00054002074696D653A004354524C3A2052BC
:1016F00065733A002054533A0020543A003D00509C
:10170000696E3A004354524C3A20436F6D6D616EDE
:101710006420626C6F636B65642062792064726917
:10172000766572206F72206368616E6E656C2066EC
:10173000726F7A656E004354524C3A204F4E3A41D4
:101740006C7265616479204163746976650A00434F
:1017500054524C3A2048414C543A416C7265616491
:101760007920496E6163746976650A004354524C6E
:101770003A20584F4E3A2044697361626C65640A9E
:10178000004354524C3A20584F4E3A416C726561B6
:101790006479204163746976650A004354524C3A77
:1017A00020584F464620736B69707065642E205038
:1017B00072657620636D643A004354524C3A20546B
:1017C00075726E6564206F66662066726F6D3A0092
:1017D0004354524C3A20526573746F7265642066AC
:1017E000726F6D3A004354524C3A2049676E6F72E3
:1017F00065642C206368616E6E656C20636D643D6A
:101800000020457865633A004354524C3A204163C6
:10181000746976653A004354524C3A2048414C541E
:101820003A416C726561647920496E6163746976CE
:10183000650A004354524C3A20584F4E3A204469AE
:101840007361626C65640A004354524C3A20584FED
:101850004E3A416C726561647920416374697665C2
:101860000A004354524C3A20584F464620736B6945
:10187000707065642E205072657620636D643A0046
:101880004354524C3A205475726E6564206F6666FC
:101890002066726F6D3A004354524C3A2052657381
:1018A000746F7265642066726F6D3A004354524CD7
:1018B0003A204E6F7420656E6F756768206D656D98
:1018C0006F727920666F722067726F7570206F700B
:1018D00065726174696F6E004354524C3A20556EC4
:1018E0006B6E6F776E2073756666697800536B69EF
:1018F0007070656420686F6D6965207374756666C5
:10190000002000205375623D00204974656D3D0044
:101910004354524C3A2052414D3D004354524C3AAC
:10192000204F75744F664D656D6F72793A200028AF
:101930002D292000282B2920002076616C75652038
:101940006973200020756E6B6E6F776E0A005D3DC7
:10195000005B0020696E76616C6964002000206F76
:101960006B003A00206661696C6564003A0052655C
:10197000747279696E67206D6F6462757320434D70
:10198000440A004354524C2F706F6C6C3A204F75D0
:10199000744F664D656D6F72793A200020736563F0
:1019A0002072656D61696E696E670053746174754C
:1019B000732064656666657265640A002D3E00509A
:1019C00075623A20006374726C00454E41424C458A
:1019D00000465245455A450044495341424C450052
:1019E0002D3E005075623A2000636D640046414E02
:1019F0005F4F4E4C590044525900434F4F4C0048E2
:101A0000454154004155544F002D3E005075623AF7
:101A100020007365740064656C002D3E0050756293
:101A20003A20002D3E005075623A2000556E6B6ED4
:101A30006F776E20636D64200A004F4646004F4E5C
:101A40000020002D3E00436F6E76657274696E67EC
:101A500020002D3E0057726F6E67204173736967D7
:101A60006E6D656E742000524742783A20002076F1
:101A70004C6576656C3A0020436F6E76563A0020CE
:101A8000436F6E76533A0020486F743A00436F6C90
:101A9000643A0020436F6E76657274656420563A2E
:101AA00000436F6E76657274656420533A002D3E74
:101AB0000057726F6E672041737369676E6D656E54
:101AC0007420002D3E0057726F6E6720417373695A
:101AD000676E6D656E7420003E3E3E004E6F204D79
:101AE000414320636F6E666967757265643A20735F
:101AF0006574206669726D776172652773204D4148
:101B0000430A004142434445464748494A4B4C4DED
:101B10004E4F505152535455565758595A6162635B
:101B20006465666768696A6B6C6D6E6F70717273FD
:101B30007475767778797A30313233343536373890
:101B4000392B2F3D00426173696320006172647517
:101B5000696E6F3A004F544120696E697469616C17
:101B6000697A65640A0044454641554C54207061C9
:101B70007373776F726420666F72204F54412041F7
:101B800050492E20557365206F746170776420630F
:101B90006F6D6D616E6420746F2073657400706189
:101BA0007373776F726400546F6F206D616E79206C
:101BB0004D51545420636F6E6E656374696F6E206F
:101BC0006572726F72732E20526573746172742025
:101BD0004C414E002074727920616761696E206902
:101BE0006E2035207365636F6E6473006661696C87
:101BF00065642C2072633D004177616974696E678A
:101C000020666F722072657461696E656420746FFE
:101C10007069637300636F6E6E65637465642061E1
:101C2000732000202E2E2E0020757365723A003A24
:101C3000000A417474656D7074696E67204D51546B
:101C40005420636F6E6E656374696F6E20746F20CD
:101C500000646973636F6E6E6563746564005573C9
:101C6000696E67204D5154542070617373776F72A1
:101C7000642066726F6D20636F6E666967002E6CFC
:101C80006F63616C006D444E53206E616D6520750D
:101C90007064617465643A20004465766963652008
:101CA0004E616D653A004174206C65617374206407
:101CB0006576696365206E616D6520616E64206282
:101CC000726F6B6572204950206D75737420626568
:101CD00020636F6E666967757265640075707469FC
:101CE0006D652C667265656865617000247374614A
:101CF000747300656333303663345F323032332DB2
:101D000030342D3032004C696768744875622000A9
:101D1000246E616D6500726561647900247374617D
:101D2000746500526562696E6420737563636573E0
:101D3000732E20495020616464726573733A0045C4
:101D400072726F723A20726562696E6420666169B0
:101D50006C0052656E6577656420737563636573A7
:101D6000732E20495020616464726573733A004594
:101D700072726F723A2072656E6577656420666173
:101D8000696C000A4E6F206C696E6B00526573744B
:101D90006F72696E6720636F6E6669672066726F27
:101DA0006D20454550524F4D004163636570746925
:101DB0006E6720636F6D6D616E64732E2E2E0A0048
:101DC0004E6F204D51545420636F6E666967757273
:101DD0006564004C6F6164696E6720636F6E66694D
:101DE000672066726F6D20706F7274616C20646919
:101DF0007361626C65642E2075736520676574205D
:101E00004F4E20746F20656E61626C6500436F6E8B
:101E10006669672069732076616C696400436F6E40
:101E200074696E756520776974682070726576696B
:101E30006F75736C79206C6F6164656420636F6E7D
:101E40006669670000002100240027002A002D0099
:101E50003000330001010000040107010A01000005
:101E60002200250028002B002E0031003400020142
:101E70000000050108010B01050505050705080817
:101E80000808020202020A0A080804040404010104
:101E90000101010101010303030303030303040719
:101EA00007070C0C0C0C0C0C0C0C020202020606B0
:101EB0000606060606060B0B0B0B0B0B0B0B05059C
:101EC00005080807070404040A0A0A0A0A0A0102A4
:101ED000102020080810204010204080020102013C
:101EE00008040201010204081020408080402010F4
:101EF000080402018004020180402010080402014D
:101F000008040201010204081020408001020408B4
:101F100010204080044080048008101020400408F5
:101F20001020408000000B0C030A0D0E0F0908045E
:101F3000050200000000000000000000000000009A
:101F40000000000000000000000000000000000091
:101F5000131211000000000000000000000000004B
:101F60000000000000000000000000000000000071
:101F7000000000000000000000002F646174610098
:101F80002F736B65746368004163636573732D43DE
:101F90006F6E74726F6C2D526571756573742D5010
:101FA0007269766174652D4E6574776F726B3A2035
:101FB00074727565004163636573732D436F6E744E
:101FC000726F6C2D416C6C6F772D48656164657222
:101FD000733A202A004163636573732D436F6E74F7
:101FE000726F6C2D416C6C6F772D4D6574686F64EA
:101FF000733A20504F53542C4745542C4F5054495A
:102000004F4E53004163636573732D436F6E74725B
:102010006F6C2D416C6C6F772D43726564656E74C7
:1020200069616C733A2074727565004F5054494F62
:102030004E530044454C45544500505554004745C7
:102040005400504F535400617574686F72697A611F
:1020500074696F6E3A2000417574686F72697A61B5
:1020600074696F6E3A2000436F6E74656E742D4C08
:10207000656E6774683A20006F637465742F7374BB
:102080007265616D00696D6167652F6A70656700D3
:10209000696D6167652F67696600746578742F687C
:1020A000746D6C006170706C69636174696F6E2F20
:1020B0006A736F6E00746578742F706C61696E005E
:1020C000436F6E74656E742D547970653A200043C9
:1020D0006F6E6E656374696F6E3A20636C6F7365C3
:1020E000004163636573732D436F6E74726F6C2D63
:1020F000416C6C6F772D4F726967696E3A202A00C8
:10210000556E6B6E6F776E004E6F74204D6F646905
:1021100066696564004F4B004D6F7665642070659D
:10212000726D616E656E746C7900496E7465726E65
:10213000616C20536572766572204572726F720011
:102140005061796C6F616420546F6F204C617267CD
:1021500065004E6F7420666F756E64005757572D7B
:1021600041757468656E7469636174653A20426193
:10217000736963207265616C6D3D224163636573B1
:102180007320726573747269637465642200556E9E
:10219000617574686F72697A6564005061796C6FFB
:1021A00061642073697A652077726F6E670042619F
:1021B00064207265717565737400485454502F31F2
:1021C0002E31200020000000000000000000004F21
:1021D0004E000000000000004F46460000000000D6
:1021E00000524553540000000000544F47474C45EF
:1021F00000000048414C540000000000584F4E00C1
:102200000000000000584F46460000000000494E04
:1022100043524541534500444543524541534500CF
:10222000454E41424C4500000044495341424C4513
:102230000000554E465245455A4500465245455ABE
:10224000450000004155544F000000000046414E3B
:102250005F4F4E4C59004849474800000000004D70
:10226000454449554D0000004C4F57000000000008
:1022700000484541540000000000434F4F4C00000F
:1022800000000044525900000000000053544F5019
:1022900000000000005247420000000000004853C8
:1022A0005600000000000057726F6E672070617961
:1022B0006C6164004354524C2F7478743A204F750B
:1022C000744F664D656D6F72793A2000202D3E2067
:1022D00041543A004368616E20747970653A004E4B
:1022E0006F2073746F7265642076616C75657320FE
:1022F0002D2064656661756C743A200053617665C3
:102300006420455441473A00536574204554414781
:102310003A20000053E326E311241FBECFEFD1E2A1
:10232000DEBFCDBF00E00CBF17E0A0E0B2E0E4E903
:10233000F2EF01E00BBF02C007900D92A63AB10781
:10234000D9F72FE0A6EAB7E001C01D92AB35B2077E
:10235000E1F711E1CBE8D1E100E006C021970109E6
:10236000802FFE010E941AF1CA38D10780E00807C9
:10237000A9F70E9407CC0C9438F90C940000CF9375
:10238000DF931F92CDB7DEB76983DC01ED91FC913D
:102390000280F381E02D41E050E0BE016F5F7F4F8E
:1023A00019950F90DF91CF910895FC01818D928D49
:1023B0000895CF93DF931F92CDB7DEB76983DC0119
:1023C000ED91FC910280F381E02D41E050E0BE01EF
:1023D0006F5F7F4F19950F90DF91CF910895FC01AA
:1023E0009485FB018485981303C081E0983008F040
:1023F00080E00895CF93DF931F92CDB7DEB7698356
:10240000DC01ED91FC910280F381E02D41E050E090
:10241000BE016F5F7F4F19950F90DF91CF910895A7
:1024200085ED8093BC008091BC0084FDFCCF1092B0
:102430008F09089520916B09260F3327331F21320E
:102440003105ECF420918F09FC0190E080E024300C
:1024500069F082E00895A0916B092191AC01455B80
:10246000564FA40FB52FB11D2C930196861798F3E4
:1024700080916B09680F60936B0980E0089581E09B
:1024800008958FEF9FEF08958FEF9FEF089580914C
:102490004A0990E09195819591090895CF93DF9332
:1024A000CB01EA01642F0E941A12CE01DF91CF9175
:1024B0000895CF93DF931F92CDB7DEB7698361E0B4
:1024C000CE0101960E941A1281E090E00F90DF91F8
:1024D000CF91089590E0FC01E858F14EE491F0E0CE
:1024E000EE0FFF1FE25AF14EA591B4912C91825349
:1024F000914EFC018491822391E009F490E0892FB0
:102500000895FC01DC018D918111FDCF30E020E0C8
:1025100050E040E08AE09191992301F14430510567
:102520005CF59E3271F42F3F310509F02CF5DB018B
:10253000A40FB51F12962C934F5F5F4F30E020E041
:10254000EACF829FD001839FB00D1124292F990FCC
:10255000330B205331092A0F3B1FDDCF2F3F3105AD
:1025600009F054F4443051053CF4640F751FFB012D
:10257000228381E090E0089590E080E00895CF9379
:10258000DF93EA01282FDC01ED91F0E094E0F5956E
:10259000E7959A95E1F7EA55FD4F80818883FD0123
:1025A0003197E081EF70F0E0EA55FD4F808189833B
:1025B00022968A2F821B861738F3615070E0660FCF
:1025C000771F460F571FFA011282DF91CF910895AE
:1025D000DC0115968D919C91009739F0DC01ED910D
:1025E000FC910680F781E02D199408958091F308FD
:1025F0009091F4080895DC011296ED91FC911397E7
:102600003097B9F016968D919C918430910541F0E8
:102610008530910541F0039749F482E090E00895F8
:1026200081E090E0089581E190E00895808590E058
:10263000089590E080E008958091F1089091F2086B
:10264000089590E080E008958091EF089091F0085F
:10265000089584E090E00895DC011496ED91FC91DA
:10266000309729F08081082E000C990B089590E096
:1026700080E0089585E090E0089580913808909179
:102680003908817099270895DC011296ED91FC912B
:10269000309761F00190F081E02D808585958595DA
:1026A00085958595082E000C990B089590E080E0A3
:1026B0000895FC01848195810895FC0176876587E2
:1026C0000895DC01ED91FC91068CF78DE02D1995B4
:1026D00091E089270895862F089581E0862708953F
:1026E00021E0FC018485883008F020E0822F0895E5
:1026F000FC01848595850895FC0184899589089558
:1027000027E934E0FC0131832083FB0140895189B2
:1027100062897389FC0142835383648375830895BE
:10272000DC01ED91FC91048CF58DE02D1994CF9294
:10273000DF92EF92FF920F931F93CF93DF9300D01E
:1027400000D0CDB7DEB78C016B017A01FC01808D22
:10275000883010F40E94B1A787E994E09A838983B6
:10276000F60182819381A481B5818B839C83AD83A3
:10277000BE83B701CE0101960E9430B9F801808F67
:102780008830A0F4F586E486128E118E81E02696BC
:102790000FB6F894DEBF0FBECDBFDF91CF911F9172
:1027A0000F91FF90EF90DF90CF90089580E0EFCFF2
:1027B000CF93DF93EC01888D883020F40E94B1A77D
:1027C00088E0888FDF91CF910895FC01808D88305B
:1027D00040F4218D328D232B21F00E9483A690E0BE
:1027E00008958FEF9FEF0895CF93DF93FC01248529
:1027F000283028F08FEF9FEFDF91CF910895EC0103
:102800000190F081E02D0084F185E02D1995892B50
:1028100089F38C850E9483A690E0EECFCF93DF935F
:10282000FC01218D328D2115310529F48FEF9FEFA9
:10283000DF91CF910895EC01808D4217530708F086
:10284000A9010E94D2A61816190684F7298D3A8D7F
:10285000281B390B3A8F298FEBCF0F931F93CF9300
:10286000DF931F92CDB7DEB7FC01218D328D232B74
:1028700041F48FEF9FEF0F90DF91CF911F910F9158
:1028800008958C0141E050E0BE016F5F7F4FFC0175
:10289000808D0E94D2A6181619065CF7F801818D6A
:1028A000928D0197928F818F898190E0E4CFCF93B1
:1028B000DF931F92CDB7DEB741E050E0BE016F5FFE
:1028C0007F4FFC0184850E94D2A61816190634F4A5
:1028D000898190E00F90DF91CF9108958FEF9FEF66
:1028E000F9CFFC018485883010F40C94D2A690E0D6
:1028F00080E00895FC018485883010F40C94ABA628
:1029000090E080E008950F931F93CF93DF9300D062
:1029100000D01F921F92CDB7DEB78C01D801599617
:102920004D915C915A974115510551F0ED91FC91F3
:10293000048CF58DE02D70E060E0C8011995EECFB4
:10294000F801808D0E94ABA6892BB1F148E050E0E0
:10295000BE016F5F7F4FD80158968C910E94D2A61E
:1029600018161906F4F4D801509684E0FE01319649
:1029700001900D928A95E1F78D8190E0982F88273C
:102980002E81820F911DF801958B848B8F81282FCA
:1029900030E0322F22278885820F932F911D928F4E
:1029A000818F28960FB6F894DEBF0FBECDBFDF91A2
:1029B000CF911F910F91089590E080E0F2CFCF92D8
:1029C000DF92EF92FF920F931F93CF93DF93CDB7D8
:1029D000DEB7AF970FB6F894DEBF0FBECDBF7C0158
:1029E0006A0107E914E01A8309831C861B8688EEB6
:1029F00093E0A0E0B0E08D879E87AF87B88B8DE62F
:102A000094E09A878987188F0F8B198E1A8E1B8EE8
:102A10001C8E88E089A31BA70AA71CA61DA61EA6BC
:102A20001FA68091120D9091130DA091140DB091DD
:102A3000150D8EA39FA3A8A7B9A78B839C83AD83F5
:102A4000BE8318861F82AE01465D5F4FCE010196A0
:102A50000E9426BF81309105B1F4D701ED91FC9120
:102A60000488F589E02D1DA30CA38CA59DA5AEA51A
:102A7000BFA58EA39FA3A8A7B9A7A601BE016C5DA1
:102A80007F4FC7011995AF960FB6F894DEBF0FBE02
:102A9000CDBFDF91CF911F910F91FF90EF90DF900D
:102AA000CF9008950F931F93CF93DF93EC018B0189
:102AB000888D883010F40E94B1A7B80182E00E948E
:102AC000FAA7888F883050F41D870C871A8E198ECC
:102AD00081E0DF91CF911F910F91089580E0F9CFB0
:102AE0000F931F93CF93DF938C01EA01FC01848540
:102AF000883048F40E9421A6892B39F481E090E0C7
:102B0000F80193838283D0E0C0E0CE01DF91CF91C2
:102B10001F910F910895EF92FF920F931F93CF9300
:102B2000DF937C018091640AD4E0833309F0D8E01C
:102B300004E51AE0C0E0F801219131918F01F7011D
:102B4000848195812817390729F0CF5FDC13F3CFF3
:102B500080E006C08C2F0E94BFA78431B1F781E0CE
:102B6000DF91CF911F910F91FF90EF900895CF9338
:102B7000DF93EC018C858830D0F40E94BFA78431AC
:102B800089F0882379F0883169F021E08C3159F49B
:102B9000E881F9810084F185E02DCE01199521E0CD
:102BA000892B09F420E0822FDF91CF91089580E0F6
:102BB000FBCFCF92DF92EF92FF920F931F93CF93B1
:102BC000DF93CDB7DEB7AF970FB6F894DEBF0FBE79
:102BD000CDBF8C016B017A0187E994E09A838983E8
:102BE0001B821C821D821E821C861B8648EE53E0BF
:102BF00060E070E04D875E876F87788B2DE634E06C
:102C00003A872987988F8F8B198E1A8E1B8E1C8E70
:102C100028E029A39BA78AA71CA61DA61EA61FA65F
:102C2000D8011C968C91883060F40E94BFA788233D
:102C300021F0F80184850E94A3A788E0D8011C96A2
:102C40008C938091120D9091130DA091140DB09161
:102C5000150D8EA39FA3A8A7B9A78B839C83AD83D3
:102C6000BE8318861F82AE01465D5F4FB601CE015E
:102C700001960E9426BF0097C1F0D801ED91FC910A
:102C80000684F785E02D87E994E09DA38CA38CA5AD
:102C90009DA5AEA5BFA58EA39FA3A8A7B9A7A70171
:102CA000BE016C5D7F4FC8011995AF960FB6F894C1
:102CB000DEBF0FBECDBFDF91CF911F910F91FF906F
:102CC000EF90DF90CF900895CF93DF93EC018C8548
:102CD000883060F40E94BFA7873111F08C3131F445
:102CE0008C850E9404A68115984088F3DF91CF91CE
:102CF0000895FC018485883010F40C9404A690E0BB
:102D000080E0089563E774E183EF9DE00E94CC9931
:102D100083EF9DE00E9436981092F0081092EF0821
:102D200081E090E008956AEF7DE0811102C06CEFD0
:102D30007DE08FED9DE00C94CC996EE17CE08FED11
:102D40009DE00E94CC99F0E0E0E0199584EF91E0DD
:102D500008954F925F926F927F92AF92BF92DF92EF
:102D6000EF92FF920F931F93CF93DF9300D000D089
:102D7000CDB7DEB77C01D62E80914709882309F4B0
:102D8000BEC0D70114969C9180912802891708F43F
:102D9000B6C08091450990914609BAE06B13F0C026
:102DA0008B50974FFC011082D70118960D911C9102
:102DB0000115110509F49FC0F8016185728561153F
:102DC000710591F4458056806780708480910C0D68
:102DD00090910D0DA0910E0DB0910F0D4816590652
:102DE0006A067B0609F487C0D8011B964D915C9159
:102DF0001C974115510509F47EC0F70124815396B3
:102E00008C91539790E0322F377002C0959587953B
:102E10003A95E2F780FF6FC0A22EB12CC501887FE2
:102E20009370892B39F451968D919C91887F937082
:102E3000A82AB92AD8018D919C91DC01ED91FC91D1
:102E40006115710509F486C00688F789E02D19958A
:102E5000019709F050C06CE3F801808191810E94D4
:102E6000D598A50170E060E02AE0D8018D919C9191
:102E70000E94EA97F8012281808191816BE875E1D7
:102E8000222311F069E875E10E94CC99D8011D96C2
:102E90006D917C911E978D919C910E94669960E244
:102EA000F801808191810E94D598D8011F966D917B
:102EB0007C9150978D919C910E946699F801228196
:102EC000808191816EE775E1222311F068E775E159
:102ED0000E94CC9965EF78E0D8018D919C910E9479
:102EE0006699F80180819181DC01ED91FC91008C63
:102EF000F18DE02D19951092460910924509D701E0
:102F000015968D919C911697009771F014963C91AF
:102F100020912902231740F0DC01ED91FC910190F2
:102F2000F081E02D6D2D199581E090E026960FB689
:102F3000F894DEBF0FBECDBFDF91CF911F910F91EF
:102F4000FF90EF90DF90BF90AF907F906F905F9079
:102F50004F9008950488F589E02D27E934E03A83FD
:102F60002983D80115964D905D906D907C901897AF
:102F70004B825C826D827E82BE016F5F7F4F67CF26
:102F80008F3491050CF0BBCFBDE06B1709F4B7CFC0
:102F90009C012F5F3F4F30934609209345098B508A
:102FA000974FFC016083ABCF0C94B3E70C94B3E76D
:102FB0000C94B3E70C94B3E70C94B3E7CF93DF938F
:102FC000FC0122813381232BF9F0EC0167E572E1EA
:102FD00083EF9DE00E94CC994AE050E06C8183EF42
:102FE0009DE00E943A9883EF9DE00E943698EA8126
:102FF000FB810190F081E02D80858F70808781E0DA
:1030000090E0DF91CF91089590E080E0FACFCF93E8
:10301000C1E068EE73E080E090E00E9401BC4AE00D
:1030200050E06C2F8FED9DE00E943A98CF5FC43145
:1030300081F784EF91E0CF910895FF920F931F9352
:10304000CF93DF93CDB7DEB764970FB6F894DEBFAA
:103050000FBECDBF8C01F62E8FE290E09A8389835C
:10306000FE01339688E0DF011D928A95E9F7F801A9
:103070006681FF2011F081E06827D80114968C91B9
:103080000E947BBAF80187819085A185B285883E30
:103090009340A105B10508F48BC064E475E183EFAA
:1030A0009DE00E94CC99D80114966D917C9183EF9C
:1030B0009DE00E94AAAE6FE375E183EF9DE00E9460
:1030C000CC996F2D70E083EF9DE00E94AAAE83EF54
:1030D0009DE00E94369866E675E1CE0101960E9459
:1030E00045E9F801828193810E94C570FF2009F4AF
:1030F0006BC067E375E1843151F060E375E18531C0
:1031000031F064E275E18F3011F46CE275E1CE01CB
:103110000B960E9459E96FE075E183EF9DE00E94F4
:10312000CC99D8011296ED91FC9113970190F08102
:10313000E02D60817181ED91FC910288F389E02D91
:103140009E012F5F3F4FAE01455F5F4FC80119954C
:10315000BC0183EF9DE00E94AAAE6DE075E183EFB4
:103160009DE00E94CC99D8011296ED91FC910190BE
:10317000F081E02D6081718183EF9DE00E9466996E
:10318000BE016F5F7F4F83EF9DE00E9466996AE00A
:1031900075E183EF9DE00E94CC99BE01655F7F4F92
:1031A00083EF9DE00E94669983EF9DE00E94369830
:1031B00064960FB6F894DEBF0FBECDBFDF91CF91FE
:1031C0001F910F91FF90089560E275E1823009F43C
:1031D0009ECF6BE175E19BCFCF93DF93EC016EEF58
:1031E00074E183EF9DE00E94CC996C817D8183EF37
:1031F0009DE00E94AAAE68EF74E183EF9DE00E941B
:10320000CC9983EF9DE00E94369860E08C810E940B
:10321000A9BA1092F4081092F30881E090E0DF91CF
:10322000CF910895CF93DF93EC0165ED74E183EFC7
:103230009DE00E94CC996C817D8183EF9DE00E948E
:10324000AAAE6FEC74E183EF9DE00E94CC9983EF0E
:103250009DE00E943698E881F981048CF58DE02D7F
:10326000CE0119958130910529F0029759F060E05F
:103270008C811AC063E070E0CE010E94068E60E08F
:103280000E94A9BA60E08C810E94A9BA61E070E056
:10329000CE010E94068E60E00E94A9BA62E070E052
:1032A000CE010E94068E60E00E94A9BA1092F20838
:1032B0001092F10881E090E0DF91CF910895EF92B4
:1032C000FF921F93CF93DF93192F7B01C82FD92F24
:1032D000D7FF03C0D195C195D10961E08C2F0E9421
:1032E000A9BA82E0E816F10499F460E08C2F0E94FC
:1032F0007BBA6CEF70E183EF9DE00E94CC9983EF85
:103300009DE0DF91CF911F91FF90EF900C94369844
:10331000612FEF2851F46095661F6627661F8C2F7A
:103320000E947BBA68EF70E1E6CF661F6627661FD2
:103330008C2F0E947BBA63EF70E1DDCFCF93DF93D8
:10334000EC0165EC74E183EF9DE00E94CC996C8107
:103350007D8183EF9DE00E94AAAE6FEB74E183EF65
:103360009DE00E94CC9983EF9DE00E9436988A816F
:103370009B81892B09F44DC08C819D81892B09F09B
:1033800048C0E881F981048CF58DE02DCE011995B6
:103390008130910529F0029759F061E08C811AC0C3
:1033A00063E070E0CE010E94068E61E00E94A9BA3F
:1033B00061E08C810E94A9BA61E070E0CE010E94B8
:1033C000068E61E00E94A9BA62E070E0CE010E9420
:1033D000068E61E00E94A9BA8091A100887F809347
:1033E000A10080919100887F809391008091A1003D
:1033F00082608093A100809191008260809391000F
:1034000081E090E09093F2088093F108DF91CF91F2
:10341000089590E080E0FACFCF93DF93DC0114961B
:10342000ED91FC91309709F44FC0C681D781209768
:10343000C1F1E881F981309781F18081882369F1B8
:1034400068EB74E0CE010E9423AE892B41F42FEF8C
:103450003FEFA90168EB74E0CE010E9440B261E148
:1034600075E0CE010E9423AE892B41F42FEF3FEF90
:10347000A90161E175E0CE010E9440B265EA74E005
:10348000CE010E9423AE892B41F42FEF3FEFA9011B
:1034900065EA74E0CE010E9440B20A80DB81C02D53
:1034A000C6CF64E674E183EF9DE00E94CC9983EF80
:1034B0009DE00E94369881E090E09093F008809320
:1034C000EF08DF91CF9108956CE474E183EF9DE004
:1034D0000E94CC9983EF9DE00E94369890E080E0B6
:1034E000F0CF0F931F93CF93DF9300D000D01F92A4
:1034F0001F92CDB7DEB7FC0182819381009759F00E
:1035000040E050E061E070E00E94B96B21E0672B81
:10351000682B692B09F020E0822F28960FB6F894CB
:10352000DEBF0FBECDBFDF91CF911F910F910895E8
:10353000CF93DF93EC016EE873E183EF9DE00E948F
:10354000F0998C819D810E94B3E770E060E08A81F0
:103550009B810E94DB681D821C8281E090E0DF91EC
:10356000CF910895CF92DF92EF92FF920F931F9326
:10357000CF93DF93EC018C819D81892B61F40A81CB
:103580001B8185E090E00E9417E7BC01C8010E9402
:10359000DB689D838C83EC80FD80E114F104A9F449
:1035A00066E773E189EE9DE00E94CC9989EE9DE08B
:1035B0000E94369890E080E0DF91CF911F910F91AB
:1035C000FF90EF90DF90CF9008951092EA0810924C
:1035D000E9081092E4081092E3081092EB081092A8
:1035E000EC081092ED081092EE081092E508109287
:1035F000E6081092E7081092E8081092610810920D
:10360000A308EA81FB81309759F08281938100976A
:1036100039F0DC0118962C912F70263009F468C01F
:103620006FE273E189EE9DE00E94CC9961E070E069
:103630008C819D81892B11F470E060E089EE9DE022
:103640000E94AAAE6DE273E189EE9DE00E94CC99E2
:1036500061E070E08A819B81892B11F470E060E069
:1036600089EE9DE00E94AAAE6BE273E189EE9DE0D7
:103670000E94CC99EA81FB8161E070E082819381B4
:10368000892B11F470E060E089EE9DE00E94AAAE03
:1036900069E273E189EE9DE00E94CC99EA81FB81A9
:1036A0000280F381E02D80858F7061E070E08630CC
:1036B00011F470E060E089EE9DE00E94AAAE67E23E
:1036C00073E189EE9DE00E94CC9989EE9DE00E9415
:1036D000369868E473E189EE9DE00E94CC9989EE0A
:1036E0009DE00E943698EC81FD818FEF808362CF50
:1036F00069EA74E00E9423AE009709F4A1C0FC01BE
:1037000020852F70243009F09BC0C184D28410E042
:1037100000E0C114D10409F486C0B80161527D4EA5
:10372000C6010E9450E9892B09F077C0F801ED51DC
:10373000FD4E25913491922F832FD70113969C93A0
:10374000139714968C93EA81FB8160EB74E082817D
:1037500093810E9423AEEC81FD81009709F476C02D
:10376000DC0118962C9118972F70223009F06EC04A
:1037700019964D915D916D917C911C974115510564
:103780006105710509F462C0528341834181528110
:10379000052E000C660B770B238181EB9BE00E94CA
:1037A000FF9CEC81FD8141815281052E000C660B4E
:1037B000770B238184E19BE00E94FF9CEA81FB81DF
:1037C0006AE275E0828193810E9423AE009739F00E
:1037D000FC01818592859093A2088093A1086EE5F3
:1037E00073E18FED9DE00E94CC99EA81FB8101900D
:1037F000F081E02D608171818FED9DE00E946699DE
:103800008FED9DE00E943698EC81FD8181E0808300
:103810008093270281E090E0CFCE0A5F1F4F0834EB
:10382000110509F076CF62EC72E183EF9DE00E9412
:10383000CC9983EF9DE00E94369896E080E07DCFA2
:1038400086E090E0F701948383837DCF80E09BE462
:10385000928381839BCFCF93DF93FC0122813381BD
:10386000232B09F441C0EC016DE472E183EF9DE08C
:103870000E94CC994AE050E06C8183EF9DE00E9469
:103880003A9883EF9DE00E9436988C81811115C093
:1038900062E00E94A9BA68E172E18FED9DE00E94AA
:1038A000CC9990E080E00E940CB2682F70E08FED20
:1038B0009DE00E94AAAE1092290226E040E855E25F
:1038C00060E070E08D819E810E94FF9CEA81FB8117
:1038D0000190F081E02D80858F708061808781E08C
:1038E00090E0DF91CF91089590E080E0FACFCF9300
:1038F000DF9300D000D01F921F92CDB7DEB7E9EC66
:10390000FDE0128A118A80E090E19587848784E83F
:1039100090E0948B838B81E0868780E090E2908BAF
:10392000878787E7858B1C821B8284E992E09A83D4
:103930008983FE83ED838FEF9FEF98878F836FE7F7
:1039400071E18FED9DE00E94CC996091A607709186
:10395000A707CE0101960E94569E89EC9DE00E9429
:10396000155C6FE671E18FED9DE00E94CC998FEDC3
:103970009DE00E9436980E9444C228960FB6F894A3
:10398000DEBF0FBECDBFDF91CF910895892B71F0BF
:10399000FB01828193810E94C0AF63E77DE08FEDE0
:1039A0009DE00E94CC9988EC90E0089590E080E042
:1039B000F2CF892B71F0FB01828193810E9472AF5B
:1039C0006CE57DE08FED9DE00E94CC9988EC90E065
:1039D000089590E080E0F2CF8091BB0D9091BC0DF6
:1039E000892B51F00E94BBC2882331F06CE47DE04A
:1039F0008FED9DE00E94CC991092DB0D1092DA0DB4
:103A000080E090E19093D60D8093D50D84E890E00E
:103A10009093DD0D8093DC0D81E08093D70D80E0E5
:103A200090E29093D90D8093D80D82E78093DE0DBC
:103A300089EC9DE00E94C45B89EC9DE00E94155CCE
:103A400088EC90E00895EF92FF920F931F93CF932D
:103A5000DF93CDB7DEB72C970FB6F894DEBF0FBE5D
:103A6000CDBF8C017B0187E994E09A8389831B8217
:103A70001C821D821E8298878F8319861A861B8658
:103A80001C8605301105ECF0BE01695F7F4FF70120
:103A9000808591850E948112892B99F0CE0107962D
:103AA0000E9463B0BE01695F7F4FF70186819781F5
:103AB0000E948112892B61F0CE0107960E940DB100
:103AC0000EC0CE0101960E9463B00430110554F778
:103AD000CE0101960E940DB103301105A4F1BE0183
:103AE000695F7F4FF701848195810E948112892B44
:103AF00051F1CE0107960E94B8B0BE01695F7F4FB9
:103B0000F701828193810E948112892B19F1CE01E4
:103B100007960E940EB065E37DE08FED9DE00E9468
:103B2000CC9980E00E94F9B188EC90E02C960FB619
:103B3000F894DEBF0FBECDBFDF91CF911F910F91E3
:103B4000FF90EF900895CE0101960E94B8B0023028
:103B500011059CF6CE0101960E940EB001301105B0
:103B6000D1F6CE0101960E940EB06CE37DE08FEDA0
:103B70009DE00E94CC99CFCF0F931F93CF93DF93FB
:103B80008C01EB010297C4F08A819B810E94E4E8DA
:103B90008093290299270E940CB20230110549F046
:103BA0008C819D810E94E4E88093280299270E94DD
:103BB00016B2C8ECD0E002C0C0E9D1E061E27DE01D
:103BC0008FED9DE00E94CC994AE050E0609129027F
:103BD0008FED9DE00E943A986CE07DE08FED9DE0D6
:103BE0000E94CC994AE050E0609128028FED9DE060
:103BF0000E943A988FED9DE00E943698CE01DF91A9
:103C0000CF911F910F910895CF93DF93EB0102970E
:103C1000A4F167EF7DE08A819B810E9432E9892BC4
:103C200029F40E9462B16F770E94A9B163EF7DE031
:103C30008A819B810E9432E9892B29F40E9462B11A
:103C400060680E94A9B16BEF7CE08FED9DE00E945F
:103C5000CC990E9462B16095661F6627661F70E06E
:103C60008FED9DE00E94AAAE8FED9DE00E943698F8
:103C700088EC90E0DF91CF9108950E94771CF8CFF7
:103C8000DA01E091B809F0E0FE2FEE27E60FF71F0A
:103C900090E0982F8827A901BD018E0F9F1F0C94DB
:103CA00076A3CF93DF931F92CDB7DEB72091B809EB
:103CB00030E0322F2227260F371F90E0982F8827D9
:103CC000498341E050E0BE016F5F7F4F820F931F39
:103CD0000E9476A30F90DF91CF910895CF93DF9349
:103CE0001F92CDB7DEB741E050E0BE016F5F7F4F5E
:103CF0000E94EBA289810F90DF91CF9108952091CE
:103D0000B80930E0322F2227620F731F90E0982FFE
:103D10008827860F971F0C946E1E63E070E00C944A
:103D20007F1E9F92AF92BF92CF92DF92EF92FF924F
:103D30000F931F93CF93DF93EC017B018091640A73
:103D4000811121C01B821A8288EE93E0A0E0B0E0CE
:103D50008C839D83AE83BF8381E294E099838883C3
:103D600088E08C8788EE93E09E878D87CE01DF9177
:103D7000CF911F910F91FF90EF90DF90CF90BF9068
:103D8000AF909F90089534E0932E833311F028E094
:103D9000922E84E5C82E8AE0D82E10E098E0B92E45
:103DA000A12CD6012D913D916D01F7018481958162
:103DB0002817390791F4812F0E94BFA7082F873158
:103DC00011F08C3139F5812F0E94ABA6892B59F562
:103DD0000C3119F4812F0E94A3A71F5F9112E1CF2C
:103DE000A11008C0D701ED91FC910084F185E02D70
:103DF000C70119951B821A8288EE93E0A0E0B0E01B
:103E00008C839D83AE83BF8381E294E09983888312
:103E1000BC86A8CF843149F08111DFCFF6013297FB
:103E200011821082DACFB12ED8CFAA24A394D5CF95
:103E30008F929F92AF92BF92CF92DF92EF92FF92BA
:103E40000F931F93CF93DF93CDB7DEB72F970FB6A6
:103E5000F894DEBF0FBECDBF5C014B017A018091AB
:103E6000640A8823C9F104E0833309F008E0B5014E
:103E7000CE0101960E94911E84E5C82E8AE0D82EBC
:103E800010E0F601219131916F01F5018481958156
:103E90002817390751F4812F0E94BFA7873129F4D1
:103EA000A701B401812F0E9421A61F5F0113E9CF52
:103EB000C7012F960FB6F894DEBF0FBECDBFDF91BE
:103EC000CF911F910F91FF90EF90DF90CF90BF9017
:103ED000AF909F908F900895F12CE12CE9CFDA01FB
:103EE000E091B809F0E0FE2FEE27E60FF71F90E013
:103EF000982F8827A901BD018E0F9F1F0C94EBA25C
:103F000044E050E0BC018FE090E00C9476A344E0E4
:103F100050E0BC0185E090E00C9476A344E050E0D2
:103F2000BC0181E090E00C9476A308959F92AF923B
:103F3000BF92CF92DF92EF92FF920F931F93CF9396
:103F4000DF938C015B01942EE52EFC01C688D78897
:103F5000F08C80E591E00E94ECB68F2D0E94C7A501
:103F6000C92DDE2D8C179D0708F4EC019E01A501DB
:103F7000B6018F2D0E9444A5F801868997898C0F80
:103F80009D1F978B868BCE01DF91CF911F910F9153
:103F9000FF90EF90DF90CF90BF90AF909F900895EB
:103FA000CF93FC01C08D80E591E00E94ECB660E209
:103FB00070E08C2F0E94DBA262E070E08C2F0E94E8
:103FC0007F1E84FD16C062E070E08C2F0E947F1E71
:103FD00083FF0AC048E162E070E08C2F0E94511E0E
:103FE00080E090E0CF91089580E591E00E94ECB6EA
:103FF000E3CF40E162E070E08C2F0E94511E81E02F
:10400000F0CFFF920F931F93CF93DF93EB01FC014F
:10401000178A168A2A81211109C02B81211106C015
:104020002C81211103C02D81222301F1411551055D
:10403000E9F08A01FC01F08C80E591E00E94ECB689
:10404000AE014E5F5F4F24E030E06CE070E08F2DFA
:104050000E94401EB8018F2D0E94CEA781E090E003
:10406000DF91CF911F910F91FF90089580E0F7CFDE
:104070000F931F93CF938C01FC016481758181E2C2
:104080000E94FAA7C82F8830F8F480E591E00E94DA
:10409000ECB68C2F0E948D1E833131F08C2FCF9186
:1040A0001F910F910C94A3A762E070E08C2F0E94E7
:1040B000DBA2F80184819581EC2FF0E0EE0FFF1F69
:1040C000EC5AF54F91838083CF911F910F91089502
:1040D0000F931F93CF93DF931F921F92CDB7DEB73D
:1040E000FC0124852830E0F48C0180E591E00E94F9
:1040F000ECB622E030E0AE014F5F5F4F60E170E070
:10410000F80184850E946F1F89819A8198278927E9
:1041100098270F900F90DF91CF911F910F910895E5
:1041200090E080E0F6CF0F931F93CF93DF931F9221
:104130001F92CDB7DEB7FC0124852830E0F48C0156
:1041400080E591E00E94ECB622E030E0AE014F5FE6
:104150005F4F64E070E0F80184850E946F1F8981E1
:104160009A819827892798270F900F90DF91CF91F8
:104170001F910F91089590E080E0F6CFCF93DF93E9
:10418000EC0187E994E0998388831A821B821C8260
:104190001D8280E591E00E94ECB6BE016E5F7F4F0C
:1041A00044E050E08FE090E00E94EBA2CE01DF916E
:1041B000CF9108950E9437A4882331F08091640A3A
:1041C000843329F0873381F090E080E0089580E522
:1041D00091E00E94ECB685E390E00E946E1E85FDA2
:1041E0000DC082E090E0089580E591E00E94ECB679
:1041F0008EE290E00E946E1E80FFF3CF81E090E09F
:1042000008951F920F920FB60F9211240BB60F92C2
:104210002F933F934F935F936F937F938F939F93CE
:10422000AF93BF93EF93FF938091B900887F80365F
:1042300009F44DC008F040C0883209F4A7C028F541
:10424000803109F49BC0C8F4882309F4F7C0883092
:1042500009F494C0FF91EF91BF91AF919F918F911D
:104260007F916F915F914F913F912F910F900BBE76
:104270000F900FBE0F901F901895883109F486C0DB
:10428000803241F780938E0914C0803409F49BC0BA
:1042900040F48033B9F38833E9F680938E0985ECD6
:1042A000AEC0803509F483C0883509F494C08834E1
:1042B00089F60E941012CECF883909F48AC038F5E9
:1042C000883729F050F4883611F0803719F683E0EA
:1042D00080938F0910928D0955C0883809F479C0F0
:1042E000803919F0803809F0B5CF80918D0980327E
:1042F00008F06FC0E0918D0981E08E0F80938D09E9
:104300008091BB00F0E0E359F64F80833BC0803BD7
:1043100039F0D0F4803A09F477C0883A09F09ACF9E
:1043200084E080938F0910926C0910926B09F0E081
:10433000E0E0199580916B0981110FC081E08093B5
:104340006B0910924B0909C0803C09F4A8CF883C46
:1043500009F4A5CF883B09F07DCFE0916C0981E09D
:104360008E0F80936C09F0E0E55BF64F80818093BF
:10437000BB0090916C0980916B0929C08091B409B0
:104380008093BB0085EC8093BC0064CF9091B3090F
:104390008091B209981758F5E091B30981E08E0F2A
:1043A0008093B309F0E0EE56F64F8081E9CFE091BB
:1043B000B30981E08E0F8093B3098091BB00F0E0D8
:1043C000EE56F64F80839091B3098091B209981709
:1043D000C8F285E8D8CFE091B30981E08E0F8093D1
:1043E000B3098091BB00F0E0EE56F64F80838091D8
:1043F000910981115ECF81E08093900984EA8093D6
:10440000BC0010928F0926CF85EC8093BC001092DF
:104410008F0980918D09803230F4E0918D09F0E0B0
:10442000E359F64F108260918D0970E08DE699E0B6
:10443000F0E0E0E0199510928D090CCF10928E09F2
:1044400038CF4F925F926F927F92AF92BF92CF928E
:10445000DF92EF92FF920F931F93CF93DF9300D0E1
:104460001F92CDB7DEB72B013C0129833A834B83E2
:104470005C83A6019501C801B701640D751D861DF9
:10448000971D211531054105510511F00E948FF04E
:1044900029813A814B815C816217730784079507F4
:1044A000D0F4241535054605570530F521E0822F57
:1044B0000F900F900F900F90DF91CF911F910F9160
:1044C000FF90EF90DF90CF90BF90AF907F906F9074
:1044D0005F904F900895461657066806790650F487
:1044E00021E089819A81AB81BC8184159505A6055F
:1044F000B705E8F220E0DBCF21E046165706680654
:104500007906A8F2F7CF0F931F93182F0E9433BCA0
:1045100004C096958795779567951A95D2F78B0184
:104520009C0101501109210931090E3F1F4F2F4FE6
:104530003F4F20F061E070E080E090E01F910F912C
:104540000895CF93DF93EC016CEE74E183EF9DE06F
:104550000E94CC996C817D8183EF9DE00E94AAAE80
:1045600066EE74E183EF9DE00E94CC9983EF9DE0BD
:104570000E94369861E08C810E94A9BA6E818C817C
:104580000E947BBA8A819B81009729F040E050E02D
:10459000BA010E94246981E090E09093F40880932E
:1045A000F3088A819B810E948472181619065CF4B4
:1045B0000A80DB81C02D80E00E948322AB01BC0118
:1045C000CE010E94246981E090E0DF91CF910895AF
:1045D000CF92DF92EF92FF920F931F93CF93DF93CF
:1045E000EC017B018D819E818A0101501109DC0162
:1045F000ED91FC910280F381E02DA80119958D8148
:104600009E81DC01ED91FC910190F081E02DD701BC
:10461000129660E09D012E193F092017310718F40A
:104620002D91620FF7CF1995CA80DB8080E00E9440
:104630008322AB01BC01C6010E94246960E172E1E2
:1046400083EF9DE00E94CC994AE050E06C8183EFBB
:104650009DE00E943A986CE072E183EF9DE00E9439
:10466000CC99E701CE018E199F0980179107A0F41C
:10467000688140E150E06A3048F465EB74E083EF14
:104680009DE00E94669940E150E0688183EF9DE0E3
:104690000E943A982196E6CF83EF9DE0DF91CF917B
:1046A0001F910F91FF90EF90DF90CF900C94369870
:1046B0004F925F926F927F928F929F92AF92BF9232
:1046C000CF92DF92EF92FF920F931F93CF93DF93DE
:1046D000CDB7DEB762970FB6F894DEBF0FBECDBF81
:1046E0004C010B871C872D873E874F87588B698B22
:1046F0007A8B6DEB72E1C7010E9450E9EEE0F0E0C9
:10470000892BF1F067EB72E1C7010E9450E9E0E10B
:10471000F0E0892BA9F061EB72E1C7010E9450E93A
:10472000EFE0F0E0892B61F01F706DEA72E1C701E4
:104730000E9450E9E12FF0E0892B11F4EDE0F0E068
:104740009B85992341F0309731F4EF2809F47FC01D
:104750008FEF9FEFAAC0E131F10508F040C0882734
:10476000EB54FC4D8F4F0C941AF1A8232724C62339
:10477000EF23EF23EF23EF239724D924EF23EF2315
:10478000EF23EF23EF23E0242425EC24CE010B9626
:104790000E9433617093600860935F089B01205111
:1047A000310929313105A0F620EF260F20935D084D
:1047B0009B01770F440B550BD4011296ED91FC91A0
:1047C00013970190F081E02D60817181ED91FC9152
:1047D0000684F785E02D07EB14E0C40119951092CB
:1047E0004B0881E0809343088DE4809344088FE573
:1047F00080934508F40185819681DC01ED91FC915F
:104800000680F781E02D1995F401828193810E9441
:1048100084692B013C01411451046104710491F03D
:104820000E9433BC9B01AC01A12CB12C650114E6A4
:10483000E12EF12C00E010E0C301B2010E94212220
:10484000882349F345E250E06AE378E029C09150BB
:10485000953128F6E92FF0E08827EE5CFB4D8F4F6D
:104860000C941AF147246C24EF23EF236C24472483
:10487000EF23EF23EF23EF23EF23EF23EF23762420
:104880008624EF23EF23EF2382247E248424809147
:1048900038088160809357084DE050E06AE172E08B
:1048A000C4010E94E82281E090E062960FB6F8947D
:1048B000DEBF0FBECDBFDF91CF911F910F91FF9053
:1048C000EF90DF90CF90BF90AF909F908F907F90B0
:1048D0006F905F904F900895809138088E7F8093FD
:1048E00057084DE050E06DE072E0DACF10925108C9
:1048F0008091380881608093570871CF81E0809360
:104900005108F6CF82E0FBCF84E0F9CF83E08093BB
:10491000510880913808816080935708809153082E
:10492000833009F05CCF82E08093530858CF19821E
:104930009031A1F148F49E3089F0CE010B960E948F
:1049400033616093530813C0913169F19231A9F733
:1049500082E08093530868E972E105C083E08093A8
:10496000530868EA72E1CE0101960E9459E9D40128
:104970001296ED91FC9113970190F081E02D6081EA
:104980007181ED91FC910288F389E02D2CEB34E0EC
:10499000AE014F5F5F4FC401199521CF10925308AC
:1049A00063EA72E1E0CF81E0809353086CE972E141
:1049B000DACFCE010B960E943361609351080FCF7E
:1049C000913031F0923009F00ACF1092560807CF9B
:1049D00080E58093560803CF913049F09230F1F092
:1049E000CE010B960E94336160935508F8CE83E0A8
:1049F00080935508D4011296ED91FC911397019084
:104A0000F081E02D60817181ED91FC910288F38944
:104A1000E02D21EC34E04EEC55E0BDCF109255086E
:104A2000D4011296ED91FC9113970190F081E02D45
:104A300060817181ED91FC910288F389E02D21EC78
:104A400034E049ED55E0A7CF913039F0923009F0CC
:104A5000C6CE80915708877F4ECF809157088860D7
:104A60004ACF8F929F92AF92BF92CF92DF92EF92F6
:104A7000FF920F931F93CF93DF9300D000D000D00D
:104A80001F92CDB7DEB76130710509F0BCC24C0191
:104A90000E9433BC9B01AC016091340870913508D1
:104AA0008091360890913708A12CB12C650118E847
:104AB000E12E13E1F12E00E010E00E942122882374
:104AC000C1F080E00E94832260933408709335081F
:104AD000809336089093370860E972E183EF9DE098
:104AE0000E94F0994DE050E060E072E0C4010E9445
:104AF000E822D40115968D919C91DC01ED91FC91F9
:104B00000084F185E02D199585970CF479C245E272
:104B100050E06AE378E0F401858196810E94B897BD
:104B2000D40115968D919C91DC01ED91FC9100844E
:104B3000F185E02D1995892B89F062E070E080E025
:104B400090E00E9401BCF40185819681DC01ED9129
:104B5000FC910284F385E02D1995E2CF68E872E1BB
:104B600083EF9DE00E94CC994AE050E0F40164811B
:104B700083EF9DE00E943A9863E872E183EF9DE045
:104B80000E94CC990AE318E08EE5E82E88E0F82E22
:104B9000D8016D918D0140E150E06A3058F465EB29
:104BA00074E083EF9DE00E94669940E150E0F801D7
:104BB0003197608183EF9DE00E943A98E016F106FC
:104BC00039F780915E0890913308891709F414C26F
:104BD0008093330880915D0890E09C01205F3F4FF7
:104BE0003093600820935F08499708F0FFC18091D7
:104BF000470890E0909332088093310880915108E3
:104C000090E09093300880932F088091530890E0B3
:104C100090932E0880932D088091550890E09093F2
:104C20002C0880932B088091570890E090933908C6
:104C3000809338088091560890E090932A088093DA
:104C40002908D401ED91FC9111970288F389E02D98
:104C500012968D919C91DC018D919C91DC016D915E
:104C60007C918091590828EC34E04EEC55E080FDB1
:104C700002C049ED55E0C401199580912908909131
:104C80002A0880389105A9F4D4011296ED91FC917F
:104C900013970190F081E02D60817181ED91FC917D
:104CA0000288F389E02D2FEC34E04EEC55E0C4018E
:104CB00019958091290890912A08892BA9F4D4018B
:104CC0001296ED91FC9113970190F081E02D608197
:104CD0007181ED91FC910288F389E02D2FEC34E095
:104CE00049ED55E0C401199565ED74E083EF9DE051
:104CF0000E946699609138087091390883EF9DE0B1
:104D00000E94AAAE83EF9DE00E94369880913808F9
:104D1000F40120813181A281B3810D90BC91A02D3D
:104D20006D917C91D9015296ED91FC912CED34E07E
:104D30004EEC55E083FD02C049ED55E0C4011995E4
:104D4000D401ED91FC9111970288F389E02D129620
:104D50008D919C91DC018D919C91DC016D917C91F8
:104D60008091380823EE34E04EEC55E081FD02C01E
:104D700049ED55E0C401199520912B0830912C087C
:104D8000032E000C440B550BD4011296ED91FC91AF
:104D900013970190F081E02D60817181ED91FC917C
:104DA0000684F785E02D01EC14E0C401199580918B
:104DB0002D0890912E08892BA9F4D4011296ED911B
:104DC000FC9113970190F081E02D60817181ED914C
:104DD000FC910288F389E02D2CEB34E04FEE54E097
:104DE000C401199580912D0890912E080197A9F47E
:104DF000D4011296ED91FC9113970190F081E02D72
:104E000060817181ED91FC910288F389E02D2CEB9A
:104E100034E044EF54E0C401199580912D0890913D
:104E20002E080297A9F4D4011296ED91FC911397E4
:104E30000190F081E02D60817181ED91FC910288FB
:104E4000F389E02D2CEB34E04BEF54E0C4011995CD
:104E500080912D0890912E080397A9F4D401129601
:104E6000ED91FC9113970190F081E02D60817181AB
:104E7000ED91FC910288F389E02D2CEB34E04FEFAB
:104E800054E0C4011995D401ED91FC911197028869
:104E9000F389E02D12968D919C91DC018D919C916E
:104EA000DC016D917C9180912B0890912C0821EC74
:104EB00034E049ED55E0892B11F04EEC55E0C4018A
:104EC000199520915F0830916008032E000C440B67
:104ED000550BD4011296ED91FC9113970190F0813E
:104EE000E02D60817181ED91FC910684F785E02DC4
:104EF00007EB14E0C4011995209131083091320874
:104F00002F3F3105B9F0032E000C440B550BD40193
:104F10001296ED91FC9113970190F081E02D608144
:104F20007181ED91FC910684F785E02D04E015E098
:104F3000C4011995198280912F089091300868EA70
:104F400072E10097C9F06AE772E181309105A1F042
:104F500065E772E18230910579F06CE672E18330A9
:104F6000910551F068E672E18430910529F08D36A3
:104F7000910531F464E672E1CE0101960E9459E98F
:104F800020912F0830913008032E000C440B550B54
:104F9000D4011296ED91FC9113970190F081E02DD0
:104FA00060817181ED91FC910684F785E02D0AE026
:104FB00015E0C401199580913808F40120813181F0
:104FC000A281B3810D90BC91A02D6D917C91D901EE
:104FD0005296ED91FC9120E135E0AE014F5F5F4FBD
:104FE00080FD02C049ED55E0C40119956FE772E1FB
:104FF00083EF9DE00E94CC9983EF9DE00E9436985C
:1050000081E090E002C090E080E02A960FB6F8942C
:10501000DEBF0FBECDBFDF91CF911F910F91FF90EB
:10502000EF90DF90CF90BF90AF909F908F900895BA
:105030008F929F92AF92BF92CF92DF92EF92FF92A8
:105040000F931F93CF93DF937C014A015901C091C5
:105050004809D0914909062F660F110B209709F4D2
:105060005CC088858F70863009F055C065E175E0B9
:10507000CE010E9423AE6C0182E08816910449F0B3
:1050800065EA74E0E3E08E16910429F0D0E0C0E018
:1050900006C06AE175E0CE010E9423AEEC01C114A6
:1050A000D104D9F1F60180858F708430B1F5618526
:1050B0007285A801C7010E94A9F5A8016FE175E0FA
:1050C000C7010E948BF5209779F188858F70843015
:1050D00059F569857A85A801C7010E948BF5A80159
:1050E0006FE175E0C7010E948BF5A114B10429F0AE
:1050F000A801B501C7010E948BF5C701DF91CF91CF
:105100001F910F91FF90EF90DF90CF90BF90AF90E5
:105110009F908F900895D0E0C0E0A8016EE975E1FE
:10512000C7010E9487E9C9CFF2E08F16910481F090
:1051300083E08816910429F06091B9097091BA0949
:10514000CACFA80168E975E1C7010E9469E9C7CF24
:10515000A80165E975E1F8CFCF92DF92EF92FF9257
:105160000F931F93CF93DF93CDB7DEB7C154D1090F
:105170000FB6F894DEBF0FBECDBF6C01AB0130E0BF
:1051800020E060E4CE0101967C010E941828F7011E
:1051900001900020E9F731978F010E191F09A8012E
:1051A000B701C6010E949BF5892B11F010E000E0C9
:1051B000C801CF5BDF4F0FB6F894DEBF0FBECDBF87
:1051C000DF91CF911F910F91FF90EF90DF90CF90E3
:1051D0000895AF92BF92CF92DF92EF92FF921F930A
:1051E000CF93DF9300D000D0CDB7DEB76C017C0148
:1051F00010E08AE0A82EB12C133061F1F701828112
:1052000090E0B0E0A0E089839A83AB83BC83BE8248
:10521000AD82BE016F5F7F4F8FED9DE00E9486865D
:1052200063E975E10E94CC991F5FFFEFEF1AFF0A57
:10523000143011F726960FB6F894DEBF0FBECDBF1F
:10524000DF91CF911F91FF90EF90DF90CF90BF90B3
:10525000AF900895F601858190E0B0E0A0E08983E9
:105260009A83AB83BC83BE82AD82BE016F5F7F4FEA
:105270008FED9DE00E94868661E975E1D3CFCF93E3
:10528000DF931F921F92CDB7DEB780914F0F9091A1
:10529000500F009711F48BE59FE0BE016F5F7F4FC9
:1052A000681B790B072E000C880B990B0F900F9041
:1052B000DF91CF9108954F925F926F927F929F926C
:1052C000AF92BF92CF92DF92EF92FF920F931F9314
:1052D000CF93DF93CDB7DEB760970FB6F894DEBFFC
:1052E0000FBECDBFFC0119861A861B861C869A85C7
:1052F0009F7090669A87A081B181109709F4EEC0E3
:105300008C91882309F4EAC000811181D8019C9115
:10531000992309F4ADC09D3209F4E4C090539A304A
:1053200028F00F5F1F4F11830083EECFC801912C2F
:10533000DC016D01C81AD90A2D91022E000C330B25
:10534000205331092A303105A0F37F016EE270E06D
:10535000C8010E9470F5FC01009709F448C0DC0107
:105360005D01AE1ABF0A11968C911197082E000CA0
:10537000990BC09711960A9798F32181022E000C81
:10538000330B205331092A30310508F075C02A301B
:10539000310514F029E030E037FF02C030E020E0B2
:1053A000032E000C440B550BAAE0B0E00E94D0F095
:1053B0002B013C018281082E000C990BC0978A308A
:1053C000910588F48A30910514F089E090E097FF08
:1053D00002C090E080E0092E000CAA0BBB0B480E27
:1053E000591E6A1E7B1EA114B10409F049C0C801F0
:1053F0000E9402E92B013C018A858F70806A8A87AE
:105400006CE270E0D7018D919C910E9470F500973D
:1054100009F05FC0F701118210824D865E866F86AB
:10542000788A88E0FE013996DE01119601900D928E
:105430008A95E1F729813A814B815C816D817E817A
:105440008F81988560960FB6F894DEBF0FBECDBFF2
:10545000DF91CF911F910F91FF90EF90DF90CF9050
:10546000BF90AF909F907F906F905F904F90089506
:10547000912CD12CC12C69CF20E030E0A90194CF30
:10548000C801B3E0AB16B104DCF4E8E0CE16D104F9
:10549000BCF40E9402E99B01AC01A4E6B0E00E94CA
:1054A000D0F0992041F07094609450944094411C45
:1054B000511C611C711C460E571E681E791EA0CF20
:1054C0000E94E0E82A852F7020672A872B013C0183
:1054D00097CF0196D7018D939C939FCF412C512C50
:1054E00032019BCFC80101969924939421CFEF926A
:1054F000FF920F931F93CF93DF93EC01A881B981A3
:10550000109761F18C91882349F108811981F80184
:105510008081882351F08D3241F080538A3028F009
:105520000F5F1F4F19830883F0CFC8010E94E4E882
:105530007C016CE270E0C8010E9470F5009751F4A4
:1055400019821882C701DF91CF911F910F91FF90AF
:10555000EF900895019699838883F4CFF12CE12C84
:10556000F1CF089583E090E0089508950895089597
:105570008F929F92AF92BF92CF92DF92EF92FF9263
:105580000F931F93CF93DF9300D000D0CDB7DEB73A
:105590002091240830912508232B09F4C5C02091BF
:1055A00017082111C1C04C01809117088F5F8093AB
:1055B00017088091C1098F5F8093C1090E9433BC95
:1055C0009B01AC016091130870911408809115083B
:1055D00090911608A12CB12C65011BE0E12EF12C55
:1055E00000E010E00E942122882309F452C0E091DB
:1055F0002408F09125080681178101151105B9F1DC
:10560000F80180858F70863071F561E275E0C80120
:105610000E9423AE0097D1F0FC0120852F70253029
:10562000A9F4E680F780E114F104E9F0FA82E98256
:10563000B801CE0101960E948A8DB401CE01019677
:105640000E949686F701E280F380EDCF1A830983EA
:1056500070E060E0CE0101960E948A8DB401CE0117
:1056600001960E949686F80102811381C6CFF3E06D
:105670008F16910451F00E9433BC6093130870930D
:10568000140880931508909316081092160D109226
:10569000170D83E088169104E9F10E9433BC9B0149
:1056A000AC0160910F0870911008809111089091E1
:1056B0001208A12CB12C650118E8E12E13E1F12E9E
:1056C00000E010E00E942122882321F1E0912408CB
:1056D000F0912508068117810115110589F0F8015F
:1056E00080858F70863041F41A83098370E060E012
:1056F000CE0101960E948A8DF80102811381ECCFC0
:105700000E9433BC60930F087093100880931108B7
:10571000909312088091C10981508093C1098091B2
:10572000170881508093170826960FB6F894DEBFAD
:105730000FBECDBFDF91CF911F910F91FF90EF90E2
:10574000DF90CF90BF90AF909F908F900895809101
:10575000A8078F5F8093A807A89583E090E00E9438
:10576000B82A8091A80781508093A8070895CF9206
:10577000DF92EF92FF92CF93DF93EC018C8588301C
:1057800068F40E94A3A70E9433BC6B017C018C8546
:105790000E94BFA7811109C088E08C87DF91CF915B
:1057A000FF90EF90DF90CF9008950E94A72B61E0CB
:1057B00070E080E090E00E9401BC0E9433BCAB012D
:1057C000BC014C195D096E097F098D859E85B0E08D
:1057D000A0E0481759076A077B07C8F28C850E942A
:1057E000B1A7DACFCF92DF92EF92FF921F93CF93C0
:1057F000DF93EC017B016A018C85883048F40E94BC
:10580000BFA7882319F08C850E94A3A788E08C8706
:10581000F70182819381A481B5810097A105B1052B
:1058200051F490E080E0DF91CF911F91FF90EF90D5
:10583000DF90CF9008958F3F9F4FAF4FBF4F89F3B9
:1058400070E060E081E20E94FAA7182F8C87883010
:1058500040F780E591E00E94ECB6A7014E5F5F4FF4
:1058600024E030E06CE070E0812F0E94401EB60121
:10587000812F0E94CEA764E070E0812F0E94DBA2FE
:105880000E9433BC6B017C018C850E94BFA78731CD
:1058900021F18C3111F1882321F20E9433BCAB013C
:1058A000BC014C195D096E097F098D859E85B0E0AC
:1058B000A0E084179507A607B70748F00E94A72B1A
:1058C00061E070E080E090E00E9401BCDDCF8C855B
:1058D0000E94B1A788E08C87A4CF81E090E0A3CF9D
:1058E00061ED70E18FED9DE00E94CC996EEB70E16F
:1058F0008FED9DE00E94CC9960EB70E18FED9DE013
:105900000E94CC9968EA70E18FED9DE00E94CC99ED
:105910008FED9DE00E94369868E970E18FED9DE083
:105920000E94CC996CE870E18FED9DE00E94CC99CB
:105930006FE770E18FED9DE00E94CC996AE670E11F
:105940008FED9DE00E94CC996BE570E18FED9DE0BD
:105950000E94CC9963E570E18FED9DE00E94CC99A7
:1059600068E470E18FED9DE00E94CC996BE370E1FB
:105970008FED9DE00E94CC9961E370E18FED9DE099
:105980000E94CC9969E270E18FED9DE00E94CC9974
:105990006DE170E18FED9DE00E94CC9963E070E1D4
:1059A0008FED9DE00E94CC9964EE7FE08FED9DE04D
:1059B0000E94CC996FEC7FE08FED9DE00E94CC9926
:1059C00067EB7FE08FED9DE00E94CC9969EA7FE074
:1059D0008FED9DE00E94CC996DE97FE08FED9DE019
:1059E0000E94CC9965E97FE08FED9DE00E94CC9903
:1059F0006AE87FE08FED9DE00E94CC996DE77FE043
:105A00008FED9DE00E94CC9965E77FE08FED9DE0F2
:105A10000E94CC996AE67FE08FED9DE00E94CC99D0
:105A20006BE57FE08FED9DE00E94CC9962E57FE021
:105A30008FED9DE00E94CC9964E47FE08FED9DE0C6
:105A40000E94CC9966E37FE08FED9DE00E94CC99A7
:105A50006CE27FE08FED9DE00E94CC996FE17FE0EA
:105A60008FED9DE00E94CC998FED9DE00C943698CF
:105A70000F931F93CF93DF9300D000D0CDB7DEB745
:105A80000E94702C67EA79E08FED9DE00E94CC992E
:105A9000CE0101960E94BE20CE0101960E94E92807
:105AA00007E914E01A8309838091120D9091130D78
:105AB000A091140DB091150D8B839C83AD83BE8393
:105AC000CE0101960E94E9281A8309831B821C8259
:105AD0001D821E8280E591E00E94ECB644E050E019
:105AE000BE016D5F7F4F81E090E00E94EBA2CE018E
:105AF00001960E94E9281A8309831B821C821D8259
:105B00001E8280E591E00E94ECB644E050E0BE01C8
:105B10006D5F7F4F85E090E00E94EBA2CE01019681
:105B20000E94E9286DEC79E08FED9DE00E94CC9910
:105B300088EC90E026960FB6F894DEBF0FBECDBF7E
:105B4000DF91CF911F910F910895009789F0FC018B
:105B500020852F70253061F40E949BAE009741F0A4
:105B6000FC0120852F70243019F4818592850895D9
:105B700090E080E00895CF92DF92EF92FF920F9332
:105B80001F93CF93DF9300D000D0CDB7DEB78091C5
:105B9000470981119AC08091C3099091C409029765
:105BA0000CF493C08091A6079091A707009709F481
:105BB0008CC067E275E00E9423AE8C01009709F467
:105BC00084C00E94B2AEE82EF12CE114F10409F475
:105BD0007CC070E060E0C8010E94A52D6C01EA94D1
:105BE000EF2809F481C061E0C8010E949BAEFC016E
:105BF00001851285CE0101960E94BE20CE0101963C
:105C00000E94EFB665E878E08FED9DE00E94CC99A8
:105C1000B6018FED9DE00E94669961EE75E08FED13
:105C20009DE00E946699B8018FED9DE00E94AAAEAA
:105C300061EE75E08FED9DE00E94669965E67AE081
:105C40008FED9DE00E9466998FED9DE00E94369851
:105C500062E072E081E19EE00E945215D092070E50
:105C6000C092060E1093090E0093080E85E69AE086
:105C7000892BE9F585E295E090930B0E80930A0E4F
:105C80008091BE099091BF09009741F070E060E0FB
:105C90000E94A52D9093BA098093B9098091B90902
:105CA0009091BA09009731F190930D0E80930C0EEC
:105CB00010920F0E10920E0E81E0809347096CE651
:105CC00078E08FED9DE00E94CC9926960FB6F8946F
:105CD000DEBF0FBECDBFDF91CF911F910F91FF901F
:105CE000EF90DF90CF90089502E012E083CF85E639
:105CF0009AE0C2CF80EA93E0892B19F485E295E01F
:105D0000D3CF80EA93E0D0CFCF92DF92EF92FF9291
:105D10001F93CF93DF9300D000D0CDB7DEB767E6F7
:105D200078E08FED9DE00E94CC9983ECE82E8DE029
:105D3000F82E10E090E1C92ED12CF70181917F015E
:105D4000803130F465EB74E08FED9DE00E94669940
:105D5000153041F1F7013197808190E0B0E0A0E08B
:105D600089839A83AB83BC83DE82CD82BE016F5F61
:105D70007F4F8FED9DE00E94868665E678E00E9469
:105D8000CC991F5F1630C9F626960FB6F894DEBF81
:105D90000FBECDBFDF91CF911F91FF90EF90DF90AD
:105DA000CF9008958091C80D90E0B0E0A0E0898385
:105DB0009A83AB83BC83DE82CD82BE016F5F7F4F4F
:105DC0008FED9DE00E9486860E943698DACFEF9292
:105DD000FF920F931F93CF93DF9300D000D01F92B9
:105DE000CDB7DEB77B01CE0107969F938F930197C6
:105DF0009F938F9301979F938F9301979F938F9377
:105E000001979F938F9301979F938F938E010F5FBD
:105E10001F4F1F930F938EE295E09F938F93DB01AB
:105E200013968C9113978F9312968C918F930E9457
:105E300030F60FB6F894DEBF0FBECDBF0697ECF478
:105E400069E87DE089EE9DE00E94CC99D701129629
:105E50006D917C9189EE9DE00E94669980E991E0C8
:105E600027960FB6F894DEBF0FBECDBFDF91CF915E
:105E70001F910F91FF90EF9008958091BB0D90912D
:105E8000BC0D892BA9F10E9403AF882389F181E61B
:105E90000E94EEAE8091BB0D9091BC0DDC01ED91A6
:105EA000FC910088F189E02D64E070E01995809103
:105EB000BB0D9091BC0DDC01ED91FC910280F38152
:105EC000E02D46E050E0B801199586E0F801A3EC1A
:105ED000BDE001900D928A95E1F78091BB0D909104
:105EE000BC0DDC01ED91FC910488F589E02D19953C
:105EF0000E94842E6BE97DE08FED9DE00E94CC999D
:105F000088EC90E0ADCF2F923F924F925F926F92CC
:105F10007F928F929F92AF92BF92CF92DF92EF9239
:105F2000FF920F93CF93DF9300D01F92CDB7DEB7D0
:105F30007C017A8369835C834B83DB011C92FC01C7
:105F40006081662309F44EC030FF4CC0F9E06F9FBA
:105F5000B00111246A537E4DCD010E9487E9D7011B
:105F600011968C91807F41F04B815C8162E475E0F9
:105F700089819A810E948BF5E981FA810190002044
:105F8000E9F7319729813A81E21BF30B19012E0EB3
:105F90003F1E4B815C814E1B5F0B415051095C835E
:105FA0004B83D7011196EC9111978E2F807F09F4C6
:105FB000F7C0E295EF70E150EC3008F0F1C0F0E08E
:105FC0008827EA51F04D8F4F0C941AF1F52F983035
:105FD000053164317F3143301531153115313130A0
:105FE00019309B3129803A80DCCFF7018481282F3A
:105FF00030E050E040E0002359F030E0A4E6B0E0AB
:106000000E94E3F02FEF30E040E050E00E94B1F05A
:106010005F934F933F932F9384E495E09F938F93E7
:10602000FC81FF932B812F933F922F920E94C3F507
:10603000B2C017968C9117978F9316968C911697DE
:106040008F9315968C9115978F9314968C918F93AF
:1060500087E495E09F938F93BC81BF93EB81EF938F
:10606000E3CF17968C9117978F9316968C9116976E
:106070008F9315968C9115978F9314968C918F937F
:106080008BE495E0E7CF1496CD90DD90ED90FC90F9
:106090001797F7FE34C084E6882E912CA12CB12CE2
:1060A000C701B601A50194010E94B1F09B01AC01AA
:1060B00088279927DC01821B930BA40BB50BBF9398
:1060C000AF939F938F9366277727CB016C197D0938
:1060D0008E099F09A50194010E94B1F05F934F932F
:1060E0003F932F938FE495E09F938F933C813F9351
:1060F0004B814F933F922F920E94C3F54CC0C70132
:10610000B60124E630E040E050E00E94B1F09F93F9
:106110008F937F936F935F934F933F932F9380E57C
:1061200095E09F938F939C819F93AB81AF93E2CF38
:10613000C7010E94DF62BC01D7011696CC9016976A
:106140001796DC901797D0FADD24D0F814969C911E
:1061500014971596FC90EB80BC80292F30E050E01E
:1061600040E077FD35C0011135C07F936F931F92DA
:106170001F921F929F931F92FF92DF92CF9289E509
:1061800095E09F938F93FC81FF932B812F933F92F8
:106190002F920E94C3F50FB6F894DEBF0FBECDBF9D
:1061A00089819A810F900F900F900F90DF91CF917E
:1061B0000F91FF90EF90DF90CF90BF90AF909F90A6
:1061C0008F907F906F905F904F903F902F900895A9
:1061D000002361F0292F30E0A4E6B0E00E94E3F054
:1061E0002FEF30E040E050E00E94B1F05F934F931A
:1061F0003F932F931F92FF92DF92CF928CE595E011
:106200009F938F93BF92EF9275CF15968C911597B0
:106210001F928F9316969C91169717968C9181706A
:106220008F939F938FE595E015CF14968D909D9059
:10623000AD90BC90179720E030E0A901C501B401F2
:106240000E9445EF2401350187FF04C077FA70945E
:1062500077F87094C301B2010E9417F26B01072E08
:10626000000C880B990B0E944CEF9B01AC01C30101
:10627000B2010E9438F120E030E04AE754E40E9485
:10628000ABEF0E94A2F20E9417F2062F772E20E0B9
:1062900030E0A901C501B4010E9445EF87FF07C0A6
:1062A0007F920F93DF92CF9285E695E0D3CE7F92D7
:1062B0000F93DF92CF9286E695E09F938F933C8178
:1062C0003F934B814F93B0CE14968C9114971F92AD
:1062D0008F9315968C9115971F928F9316968C918C
:1062E0001F928F938CE595E09F938F93BC81BF9312
:1062F000EB81EF933F922F920E94C3F54CCF1796FC
:106300008C9117971F928F9314968C9114971F92CC
:106310008F9315968C9115971F928F9316968C914B
:106320001F928F9389E595E09F938F93BC81BF93D4
:10633000EB81EF93DFCE14966D917C914B815C8164
:10634000C1010E94A9F52CCFEF92FF920F93CF933A
:10635000DF93CDB7DEB7A0970FB6F894DEBF0FBEC0
:10636000CDBF7C0100E020E033E040E250E0BE0120
:106370006F5F7F4F0E94832FBE016F5F7F4F83EF60
:106380009DE00E94669967E577E083EF9DE00E94BB
:10639000CC99F701618162956F704AE050E083EF1C
:1063A0009DE00E943A9860E577E083EF9DE00E94CF
:1063B000CC99F70161816F704AE050E083EF9DE076
:1063C0000E943A9883EF9DE00E943698A0960FB6FF
:1063D000F894DEBF0FBECDBFDF91CF910F91FF903C
:1063E000EF900895CF92DF92FF920F931F93CF9378
:1063F000DF93F12C6115710509F499C06A01EB0175
:106400008C01CB010E94CF68F82E882309F48FC03D
:10641000D2FE09C0D8018C918B3009F44BC0E8F54D
:106420008A3009F44CC0D0FE09C0F801608186EFC3
:10643000860F843018F0CE010E949470D1FE6EC099
:10644000D80114964D915D916D917C91179711969D
:106450008C9182958F70873038F0893008F43EC077
:106460008A50823008F46CC0CE010E94A069EC8191
:10647000FD81309709F452C080858F709EEF980F90
:10648000923010F081114AC0D80111969C91907FF2
:1064900080858F70892B808741C08C30B9F040E0B7
:1064A00050E062E070E08D3009F0BDCFCE010E9477
:1064B000906BB9CF40E050E061E070E0F7CF40E092
:1064C00050E061E070E0CE010E94676B40E050E078
:1064D00062E070E0CE010E94676BA5CFEC81FD8188
:1064E0003097E1F080858F709EEF980F923010F01A
:1064F000811114C04187528763877487EC81FD81C5
:106500008085807F83608087EC81FD818085982FE6
:10651000907F8F708067903609F4BDCF69E477E093
:1065200083EF9DE00E94CC99C8010E94A4318F2D79
:10653000DF91CF911F910F91FF90DF90CF90089541
:10654000CE010E94A069EACFCF92DF92EF92FF9234
:106550000F931F93CF93DF936115710509F460C00A
:106560006A017B018C01CB010E94CF68D82F882360
:1065700089F1D70114968D919C91009709F43FC041
:10658000FC01C0852C2F2F703EEF320F323010F0FF
:1065900021112AC0C595C595C595C595D0FE5EC08B
:1065A000C7010E94C570F8018083CC2351F1C295C8
:1065B000C07F81818F70C82BC183D7011496ED9164
:1065C000FC9181859285A385B485F80184839583A8
:1065D000A683B7838D2FDF91CF911F910F91FF90ED
:1065E000EF90DF90CF900895253049F460E00E944D
:1065F0009BAE009721F0DC011896CC91CBCFC0E088
:10660000CDCFD7011496ED91FC9180858295807F46
:106610008595859585958595823021F0833081F02B
:10662000D0E0D8CF4185528563857485F80181819A
:106630008F70806A81834483558366837783CACF52
:106640004185528563857485F80181818F708067EB
:1066500081834483558366837783BCCFCC2389F2BF
:10666000C295C07FF801A5CFCF93DF9300D000D0B3
:106670001F921F92CDB7DEB7FC01862F8F7061810C
:10668000607F682B618388E0DE01119601900D9296
:106690008A95E1F729813A814B815C816D817E8108
:1066A0008F81988528960FB6F894DEBF0FBECDBFB8
:1066B000DF91CF910895CF93DF9300D000D01F9248
:1066C0001F92CDB7DEB7FC01608398E0DE01119622
:1066D00001900D929A95E1F729813A814B815C8175
:1066E0006D817E818F81988528960FB6F894DEBFE4
:1066F0000FBECDBFDF91CF910895CF93DF9300D030
:1067000000D01F921F92CDB7DEB7FC016F3F71051D
:1067100019F014F06FEF70E077FD60E09181892F40
:1067200082958F7081508230C8F4648388E0DE01E6
:10673000119601900D928A95E1F729813A814B815A
:106740005C816D817E818F81988528960FB6F89443
:10675000DEBF0FBECDBFDF91CF9108959F709061D6
:106760009183E3CF0F931F93CF93DF93DC01C62F69
:106770001196EC911197E295EF70EC3008F0BCC0E7
:10678000F0E08827E953FC4C8F4F0C941AF1D33377
:10679000F833F8337C347C347C345A3404347C341D
:1067A0007C34DB33DB3370E060E0CB01DF91CF91F1
:1067B0001F910F91089514968D919D910D90BC910C
:1067C000A02D8F3F9105A105B10529F024F08FEF91
:1067D00090E0A0E0B0E0B7FF03C080E090E0DC0113
:1067E0006FEF70E0681B790BC111DFCFBC01DDCF0B
:1067F00014966C9170E0CC23C1F28FEF90E09C0175
:10680000261B370BB901D1CF862F14960C91149704
:1068100015961C9115971696DC9116971796CC91A4
:1068200020E030E0A901B801882331F18D2F9C2FA1
:106830000E9445EF87FD1BC020E030E04FE753E4A6
:10684000B8018D2F9C2F0E944DF2181624F400E001
:1068500010E0DFE7C3E498014D2F5C2F60E070E0AB
:106860008FE793E40E9438F10E9417F29ECF00E078
:1068700010E0D0E0C0E0EFCF8D2F9C2F0E9445EFBD
:1068800087FD13C020E030E04FE753E4B8018D2FBF
:106890009C2F0E944DF2181624F400E010E0DFE770
:1068A000C3E4B8018D2F9C2FDFCF00E010E0D0E0D3
:1068B000C0E0F7CF14966D917D918D919C911797C3
:1068C00024E630E040E050E00E94B1F02F3F310577
:1068D0004105510529F024F02FEF30E040E050E071
:1068E00057FF03C020E030E0A9016FEF70E0621BAA
:1068F000730BC1115ACF86CF6FEF7FEF56CFAF9298
:10690000BF92CF92EF92FF920F931F93CF93DF939B
:1069100000D000D01F921F92CDB7DEB75C01098373
:106920001A832B833C834D835E836F8378876DE668
:1069300075E183EF9DE00E94CC99CE0101960E9403
:10694000A431E114F10439F066E675E1C7010E9453
:1069500050E9009721F1F50102811381011511051C
:10696000E1F0898181115BC08A818F70813009F4E7
:106970005EC038F1823019F1082F10E069E475E14A
:1069800083EF9DE00E94CC99B80183EF9DE00E94C7
:10699000AAAE83EF9DE00E94369890E080E02896B2
:1069A0000FB6F894DEBF0FBECDBFDF91CF911F9120
:1069B0000F91FF90EF90CF90BF90AF900895CC20B3
:1069C000C1F060E0CE0101960E94B233892B09F438
:1069D00047C0C8010E948469672B682B692BE1F4CA
:1069E00080E00E948322AB01BC01C8010E9424699F
:1069F00013C0C8010E94C5708E3019F050F4813068
:106A000059F460E0CE0101960E94B233892B21F047
:106A1000E0CF83518330A8F381E090E0C0CF803194
:106A2000D0F48E30B0F68130A1F28230C9F069E541
:106A300075E183EF9DE00E94CC994AE050E06981C6
:106A400083EF9DE00E943A9883EF9DE00E94369884
:106A500001E010E093CF8351833008F4BACFE7CF41
:106A600040E050E0BA01C8010E94246960E0C5011D
:106A70000E941D18D1CF2F923F924F925F926F923A
:106A80007F928F929F92AF92BF92CF92DF92EF92BE
:106A9000FF920F931F93CF93DF93CDB7DEB760972D
:106AA0000FB6F894DEBF0FBECDBF6130710509F49B
:106AB00095C0DC0112966D917C916115710509F408
:106AC0008DC04C0119821A821B821C821D821E827B
:106AD0001F8218868A818F708A8340E052E0CE013F
:106AE00001960E94A43260E0CE0101960E94B2336A
:106AF0001C01F401828193810E9484692B013C0175
:106B0000D40117962D913D914D915C911A97D10129
:106B10000E94DBF02FEF30E040E050E00E948FF069
:106B200029873A874B875C870E9433BC9B01AC0165
:106B300089859A85AB85BC850097A105B10509F4C7
:106B400068C0A12CB12C65017C018D01C301B2018B
:106B50000E94212289874114510461047104F1F1DA
:106B6000D40117968D919D910D90BC91A02D8D878C
:106B70009E87AF87B88B0E9433BC9B01AC018D858B
:106B80009E85AF85B8890097A105B10561F0A12C5C
:106B9000B12C65017C018D01C301B2010E9421224B
:106BA000882309F451C0D40112966D907C9080E046
:106BB0000E948322AB01BC01C3010E9424692328E7
:106BC00069F0F40184810E946A12D40116969C91A6
:106BD000891304C061E0C4010E941D1890E080E0A8
:106BE00060960FB6F894DEBF0FBECDBFDF91CF9198
:106BF0001F910F91FF90EF90DF90CF90BF90AF90DB
:106C00009F908F907F906F905F904F903F902F90CC
:106C1000089591E099879FCFB985BB23F1F060E09B
:106C2000C4010E941D18F401828193810E94847224
:106C3000892BA1F640E050E0BA01D40112968D9163
:106C40009C910E942469CACFF40184810E946A1237
:106C5000D40116969C918913DFCF232809F4BECF67
:106C6000F40184810E946A12D40116969C918913C2
:106C7000B5CFB985B111B2CFADCFAF92BF92CF92A0
:106C8000DF92EF92FF920F931F93CF93DF93CDB7D5
:106C9000DEB768970FB6F894DEBF0FBECDBFFC011C
:106CA000098B1A8B2B8B3C8B4D8B5E8B6F8B788F6C
:106CB00082819381009709F49FC024813581232B21
:106CC00009F49AC0CC2009F497C06F0170E060E02D
:106CD0000E94CA69192FD601ED91FC91048CF58DA3
:106CE000E02DC60119955C018230910509F478C048
:106CF000039709F447C095E0F1E0AF16B10409F03D
:106D000091E019861A861B861C861D861E861F86A4
:106D1000188A9295907F8A858F70892B8A87EE24B6
:106D2000EA94FE2C09891A892B893C894D895E8950
:106D30006F89788DCE0109960E943C63F1E0AF1611
:106D4000B10409F44FC082E0A816B10409F045C0AF
:106D50006F8570E0D60114968C910E94E5BA61E0CF
:106D600070E0C6010E94068E6E8570E00E94E5BA52
:106D700062E070E0C6010E94068E6D8570E00E94A0
:106D8000E5BA2BC0612F661F6627661FCE014196AC
:106D90000E94B2335C01BC01D60114968C910E9412
:106DA000E5BA61EE74E183EF9DE00E94CC99F601B3
:106DB0006481758183EF9DE00E94AAAE6FED74E15E
:106DC00083EF9DE00E94CC99B50183EF9DE00E9486
:106DD000AAAE83EF9DE00E94369881E090E00EC05D
:106DE00094E08FCF63E070E0C6010E94068E688950
:106DF00070E00E94E5BAACCF90E080E068960FB6F4
:106E0000F894DEBF0FBECDBFDF91CF911F910F91E0
:106E1000FF90EF90DF90CF90BF90AF900895EF92EA
:106E2000FF920F931F93CF93DF9300D01F92CDB7A4
:106E3000DEB78C017B01FB0184858830A8F087E9EF
:106E400094E0F80191838083128213821482158268
:106E5000C8010F900F900F900F90DF91CF911F916D
:106E60000F91FF90EF90089580E591E00E94ECB6BD
:106E700024E030E0AE014F5F5F4F6CE070E0F7015F
:106E800084850E946F1FBE016F5F7F4FC8010E9403
:106E9000029ADECF8F929F92AF92BF92CF92DF92F3
:106EA000EF92FF920F931F93CF93DF93CDB7DEB78F
:106EB000C456D1090FB6F894DEBF0FBECDBF87E927
:106EC00094E02F969FAF8EAF2F9763961CAE1DAEAA
:106ED0001EAE1FAE639765969FAF8EAF659769969E
:106EE0001CAE1DAE1EAE1FAE69976B969FAF8EAFE8
:106EF0006B976F961CAE1DAE1EAE1FAE6F97A19620
:106F00009FAF8EAFA197A5961CAE1DAE1EAE1FAE55
:106F1000A5976AE979E08FED9DE00E94CC998FED0D
:106F20009DE00E9436988091BB0D9091BC0D8E0122
:106F30000F5F1F4F892B09F452C00E9403AF8823B3
:106F400009F44DC082E70E94EEAE8091BB0D909196
:106F5000BC0DDC01ED91FC910088F189E02D60E130
:106F600070E0199544E050E0B8018091BB0D90911C
:106F7000BC0D0E94B89789819A81AB81BC816396D0
:106F80008CAF9DAFAEAFBFAF63978091BB0D9091BB
:106F9000BC0DDC01ED91FC910488F589E02D19957B
:106FA00060968FAD60978823D1F08F3F79F461961A
:106FB0008FAD61978F3F51F462968FAD62978F3F8F
:106FC00029F463968FAD63978F3F49F00E9462B1B9
:106FD00070FF8BC18091BD09833008F086C16EE8D7
:106FE00079E08FED9DE00E94CC990FB6F894A895BA
:106FF00080916000886180936000109260000FBEF5
:107000008091070881112AC01092EF071092EE07B5
:1070100088EE93E0A0E0B0E08093F0079093F10752
:10702000A093F207B093F3078DE694E09093ED07F9
:107030008093EC0787E994E09093FB078093FA072D
:107040001092FC071092FD071092FE071092FF07A6
:1070500088E08093040881E08093070889EA97E03C
:107060009093BC098093BB090E9437A4F12CE12CBA
:10707000882309F4A6C080E591E00E94ECB646E0C2
:1070800050E063EC7DE089E090E00E9476A387E920
:1070900094E09A8389831B821C821D821E82CE010A
:1070A00003960E94801F8091BB099091BC09FC014E
:1070B00012A213A214A215A2DC0116A217A210A6F6
:1070C00011A612A613A614A615A640EE5EE260E075
:1070D00070E046AB57AB60AF71AF40EA5FE060E095
:1070E00070E042AF53AF64AF75AF189626E0FD0174
:1070F000322F11923A95E9F7AC01425F5F4F34E1CC
:10710000FA0111923A95E9F7E3ECFDE001900D9256
:107110002A95E1F7FC01EE5BFF4F10820E9457A118
:107120007C01019709F04DC080E591E00E94ECB62A
:107130006091BB097091BC09625F7F4FC8010E94DA
:10714000029ACE0103960E94801F6091BB09709144
:10715000BC096A5E7F4FC8010E94029ACE01039665
:107160000E948E1F6091BB097091BC096E5E7F4FBB
:10717000C8010E94029ACE0103960E94871F609167
:10718000BB097091BC09625E7F4FC8010E94029AE0
:107190008B819C81AD81BE818093120D9093130DE4
:1071A000A093140DB093150D0E94DCBB7F738091EA
:1071B0002A0290912B026827792770932B02609303
:1071C0002A0288E199E20FB6F894A89580936000AE
:1071D0000FBE90936000A895EF2809F48CC265EE6D
:1071E00078E08FED9DE00E94CC99C8010E94BE20FE
:1071F0008B819C81AD81BE8163968CAF9DAFAEAF1C
:10720000BFAF639737E9E32E34E0F32EFA82E982C9
:10721000C8010E94E9288FED9DE00E943698CE01BA
:10722000835B9F4F0E940EB08091120D9091130DC1
:10723000A091140DB091150D8B839C83AD83BE83FB
:1072400069968CAF9DAFAEAFBFAF6997CE018D5A37
:107250009F4F0E94B8B0FA82E9821B821C821D8275
:107260001E8280E591E00E94ECB644E050E0BE0151
:107270006D5F7F4F81E090E00E94EBA28B819C814B
:10728000AD81BE816F968CAF9DAFAEAFBFAF6F9734
:10729000CE01875A9F4F0E940DB1FA82E9821B826C
:1072A0001C821D821E8280E591E00E94ECB644E0C3
:1072B00050E0BE016D5F7F4F85E090E00E94EBA241
:1072C0008B819C81AD81BE81A5968CAF9DAFAEAF09
:1072D000BFAFA597CE01815A9F4F0E9463B081E056
:1072E0000E94F9B11092BD099CC168E779E08FED69
:1072F0009DE00E94CC9987E994E09A838983639604
:107300008CAD9DADAEADBFAD63978B839C83AD83DC
:10731000BE83C8010E94E9288091BB0D9091BC0DED
:10732000892B09F4D6C10E9403AF882309F4D1C187
:1073300082E70E94EEAE8091BB0D9091BC0DDC0106
:10734000ED91FC910088F189E02D64E170E01995E0
:1073500044E050E0B8018091BB0D9091BC0D0E94BB
:10736000B89789819A81AB81BC8169968CAF9DAFBA
:10737000AEAFBFAF69978091BB0D9091BC0DDC01A2
:10738000ED91FC910488F589E02D199566968FADF5
:107390006697882309F49DC18F3F81F467968FAD6E
:1073A00067978F3F59F468968FAD68978F3F31F498
:1073B00069968FAD69978F3F09F48BC162E779E0D9
:1073C0008FED9DE00E94CC9987E994E09A838983B0
:1073D00069968CAD9DADAEADBFAD69978B839C8337
:1073E000AD83BE83C8010E94E9288091BB0D9091B6
:1073F000BC0D892B09F44CC10E9403AF882309F40A
:1074000047C182E70E94EEAE8091BB0D9091BC0D0A
:10741000DC01ED91FC910088F189E02D68E170E0DC
:10742000199544E050E0B8018091BB0D9091BC0DDE
:107430000E94B89789819A81AB81BC816F968CAF8D
:107440009DAFAEAFBFAF6F978091BB0D9091BC0D5C
:10745000DC01ED91FC910488F589E02D19956C967D
:107460008FAD6C97882309F413C18F3F81F46D961B
:107470008FAD6D978F3F59F46E968FAD6E978F3F9E
:1074800031F46F968FAD6F978F3F09F401C16DE6B0
:1074900079E08FED9DE00E94CC9987E994E09A8392
:1074A00089836F968CAD9DADAEADBFAD6F978B836D
:1074B0009C83AD83BE83C8010E94E9288091BB0DE7
:1074C0009091BC0D892B09F4AFC00E9403AF8823B3
:1074D00009F4AAC082E70E94EEAE8091BB0D9091A4
:1074E000BC0DDC01ED91FC910088F189E02D6CE18F
:1074F00070E0199544E050E0B8018091BB0D909187
:10750000BC0D0E94B89789819A81AB81BC81A596F8
:107510008CAF9DAFAEAFBFAFA5978091BB0D9091E3
:10752000BC0DDC01ED91FC910488F589E02D1995E5
:10753000A2968FADA297882309F476C08F3F81F47D
:10754000A3968FADA3978F3F59F4A4968FADA497C0
:107550008F3F31F4A5968FADA5978F3F09F464C096
:1075600066E679E08FED9DE00E94CC9947E9E42E34
:1075700044E0F42EFA82E982A5968CAD9DADAEADC5
:10758000BFADA5978B839C83AD83BE83C8010E944A
:10759000E9282996FFAEEEAE2997A5968CAD9DAD54
:1075A000AEADBFADA5972D968CAF9DAFAEAFBFAFC3
:1075B0002D972396FFAEEEAE23976F968CAD9DADC3
:1075C000AEADBFAD6F9727968CAF9DAFAEAFBFAFDF
:1075D0002797FAA2E9A269968CAD9DADAEADBFAD7D
:1075E00069978BA39CA3ADA3BEA3FA82E98263969D
:1075F0008CAD9DADAEADBFAD63978B839C83AD83EA
:10760000BE839E01295B3F4FAE014F5B5F4FBE01C2
:107610006F5D7F4FC8010E94C5B78FED9DE00E944E
:10762000369882E090E07AC087E994E023969FAF95
:107630008EAF23976F964CAD5DAD6EAD7FAD6F97FE
:1076400027964CAF5DAF6EAF7FAF27979AA389A304
:1076500069964CAD5DAD6EAD7FAD69974BA35CA3F4
:107660006DA37EA39A83898363968CAD9DADAEADE9
:10767000BFAD63978B839C83AD83BE83AE014F5BAD
:107680005F4FBE016F5D7F4FC8010E9404B8C5CF38
:1076900087E994E09AA389A369964CAD5DAD6EAD80
:1076A0007FAD69974BA35CA36DA37EA39A83898367
:1076B00063968CAD9DADAEADBFAD63978B839C8360
:1076C000AD83BE83BE016F5D7F4FC8010E9456B877
:1076D000A4CF87E994E09A83898363968CAD9DADAE
:1076E000AEADBFAD63978B839C83AD83BE83C80172
:1076F0000E94A1B892CF64E279E089EE9DE00E94F9
:10770000CC9965EF78E089EE9DE00E94CC9980915C
:10771000BD098F5F8093BD0986EF9FEF9093C409E9
:107720008093C30989E0EAE3F2E0D80101900D9269
:107730008A95E1F7FE013A9687E1DF011D928A956D
:10774000E9F7AE01475F5F4F62E087EC9DE00E9482
:10775000BF12CE018F5B9F4F0E94BE200E9433BCA0
:10776000683B7B408105910538F464E670E080E079
:1077700090E00E9401BCF2CF27968CAD9DADAEADDE
:10778000BFAD279780934C0D90934D0DA0934E0D58
:10779000B0934F0DC8010E948AB7892BC9F0E090C1
:1077A000480DF090490DD701ED91FC91C088D1882A
:1077B0006CE272E0CE0181960E94029A49EE54E199
:1077C000BE016F5D7F4FC701F6011995811117C189
:1077D00064EC78E089EE9DE00E94CC9989EE9DE012
:1077E0000E94369828E4E22E2DE0F22ED12CC12CF6
:1077F000D70154968D919C91892B71F1960143E0AC
:1078000050E060E070E0CB010E9432C3D701549693
:10781000ED91FC9180859185009711F00E94B3E76E
:10782000D7015496ED91FC9186819781009711F0D4
:107830000E94B3E7D7015496ED91FC918481958124
:107840000E94B3E7F701848995890E94B3E7D701C5
:1078500055961C921E925497BFEFCB1ADB0AE2E0BA
:10786000EE0EF11CF8E0CF16D10411F686E0EAE541
:10787000F2E0DE01919601900D928A95E1F7FE010A
:10788000B7968AE1DF011D928A95E9F7AE014A5D5C
:107890005F4F66E083EC9DE00E94BF126EE675E0EC
:1078A000C8010E9465F59CE5C92E9DE0D92EB12C3A
:1078B000A12CF601819191916F01892B09F0A8C04B
:1078C0008AE090E00E9417E77C01009709F4A0C0CD
:1078D000DC0119961C921E92189715961C921E9206
:1078E0001497F80101900020E9F7CF010197801B60
:1078F000910B0E9417E76C01D70115969C938E930C
:107900001497892B09F4A4C04E01B1E28B0E911C8F
:10791000F40101900020E9F7CF0101978819990936
:107920000E9417E7D70119969C938E93189700979A
:1079300009F48BC0B4010E9484F580E590E0F70162
:107940009183808313821282B801C6010E9484F55C
:10795000F60101900020E9F73197CE16DF0620F4FA
:10796000319781818E32C9F76F0122E0C20ED11C9E
:10797000D6010D900020E9F7CD018C199D090B96D9
:107980000E9417E74C01F70197838683009741F027
:10799000B6010E9484F565E775E0C4010E9465F5B3
:1079A000F501EE0FFF1FE45AF24FF182E0829501DC
:1079B00042E050E060E070E0CB010E9432C30197EA
:1079C00081F161E875E089EE9DE00E94669989EE9B
:1079D0009DE00E943698CC59DF4F0FB6F894DEBF79
:1079E0000FBECDBFDF91CF911F910F91FF90EF9010
:1079F000DF90CF90BF90AF909F908F9008956CEAEA
:107A000078E08FED9DE00E94CC998FED9DE0E8CE6F
:107A1000FFEFAF1ABF0A28E0A216B10409F049CF60
:107A2000D0CF6BE978E08FED9DE00E94CC99B80152
:107A30008FED9DE00E94669964E978E08FED9DE00E
:107A40000E94CC998FED9DE0C4CFC6010E94B3E7A0
:107A5000D70116968D919C91009711F00E94B3E783
:107A6000F70180859185009711F00E94B3E7C70167
:107A70000E94B3E7A6CF2F923F924F925F926F92F0
:107A80007F928F929F92AF92BF92CF92DF92EF92AE
:107A9000FF920F931F93CF93DF93CDB7DEB7C955F6
:107AA000D1090FB6F894DEBF0FBECDBF3C01562EF4
:107AB0006296EFAE62976396FFAE639764960FAFE0
:107AC000649765961FAF659766962FAF6697679622
:107AD0003FAF679768964FAF689769965FAF6997B2
:107AE0006A96CFAE6A972D2C4A2C3B2C009709F44E
:107AF00069C1FC0180858295807F859585958595F6
:107B00008595843009F449C12CF4882309F44EC1C9
:107B100080E02DC0853009F444C08630C9F761E2A9
:107B200075E0C3010E9423AE4C01009709F46FC0B9
:107B3000B12CA12CD12CC12C6296EFAC629763962C
:107B4000FFAC639764960FAD649765961FAD65971C
:107B500066962FAD669767963FAD679768964FAD6F
:107B6000689769965FAD6997652D0E943B3DC75A3E
:107B7000DF4F0FB6F894DEBF0FBECDBFDF91CF91C0
:107B80001F910F91FF90EF90DF90CF90BF90AF903B
:107B90009F908F907F906F905F904F903F902F902D
:107BA00008958091C1098F5F8093C1098680978075
:107BB0008114910431F1A42CB32C6A96CFAC6A974E
:107BC000D22C6296EFAC62976396FFAC6397649693
:107BD0000FAD649765961FAD659766962FAD669756
:107BE00067963FAD679768964FAD689769965FADAA
:107BF0006997652DC4010E943B3DF401828093800A
:107C0000D7CF8091C10981508093C10981CF62EAA9
:107C100075E0C3010E9423AE7C0167EA75E0C301F1
:107C20000E9423AE6C01552039F0F1E05F1609F493
:107C300095C010E000E00CC06CEA75E0C3010E9442
:107C400023AE4C0161EB75E0C3010E9423AE8C01B1
:107C50008114910409F443010115110509F483010C
:107C6000E114F10421F46A96EFAC6A97F22CC11486
:107C7000D10411F4C42CD32C8114910409F49FC0B5
:107C8000F40180858F70843009F099C081849284DA
:107C90000115110509F49EC0F80180858F708430AC
:107CA00009F098C001851285E114F10409F4DFC0E0
:107CB0008114910409F49DC06EED75E183EF9DE0A0
:107CC0000E94CC99F7016185728583EF9DE00E9447
:107CD000669969ED75E183EF9DE00E94CC99B4014E
:107CE00083EF9DE00E94669983EF9DE00E943698A5
:107CF000CE018F5A9F4F0E94A431C114D10409F0C4
:107D0000BFC0F70180858F70843009F00BC1618599
:107D10007285CE0101960E941471CE0101960E94D7
:107D2000CF688823B1F00E943F296B01683C710540
:107D30000CF073C065EA75E189EE9DE00E94CC9974
:107D4000B60189EE9DE00E94AAAE89EE9DE00E94F8
:107D50003698CE0101960E94A071E4C066EB75E0F2
:107D6000C3010E9423AE4C016BEB75E0C3010E947E
:107D700023AE8C018114910409F0D6C06CEA75E041
:107D8000C3010E9423AE4C010115110509F45ACF1D
:107D9000892B09F065CF430163CF10E000E0912CFF
:107DA000812CD12CC12CF12CE12C52CF10E000E021
:107DB000912C812CD12CC12CF12CE12C51CF912C68
:107DC000812C66CFCA2CDB2C6A96EFAC6A97F22C1A
:107DD000912C812C00E020E033E040E150E0BE0136
:107DE0006F5B7F4FCE018F5A9F4F0E94832F8C0174
:107DF0005BCF6FEC75E183EF9DE00E94CC99F701BA
:107E00006185728583EF9DE00E9466996AEC75E159
:107E100083EF9DE00E94CC996BCF8114910431F0E7
:107E2000B401CE0101960E9414B393CFCC24C39425
:107E3000F12CE12C62960FAD629763961FAD6397AC
:107E400064962FAD649765963FAD659766964FAD86
:107E5000669767965FAD679768966FAD6897699606
:107E60007FAD6997CE0101960E94857372CFC114D0
:107E7000D10409F457C00115110509F453C004C019
:107E80000115110509F43DCFF60180858F7084300E
:107E900009F044C063EC75E183EF9DE00E94CC994A
:107EA000F6016185728583EF9DE00E9466996EEB15
:107EB00075E183EF9DE00E94CC99B80183EF9DE0CE
:107EC0000E94669983EF9DE00E943698F6016185D5
:107ED000728540E450E0CE0101960E94A9F50E940F
:107EE00041AE8823D9F08091A807811117C06FE2B5
:107EF00070E0CE0101960E9470F5892B51F4F601D5
:107F00002185328543E050E060E4CE0101960E9475
:107F10001828B801CE0101960E9401BDE114F104B8
:107F200009F0EFCE81E023CE892B09F099CE8ACEDD
:107F30002F923F924F925F926F927F928F929F9279
:107F4000AF92BF92CF92DF92EF92FF920F931F9367
:107F5000CF93DF93CDB7DEB7C057D1090FB6F894F2
:107F6000DEBF0FBECDBFFC0162960FAF6297639676
:107F70001FAF639764962FAF649765963FAF659781
:107F800066964FAF669767965FAF679768966FAFD5
:107F9000689769967FAF699786EF800F823008F403
:107FA00098C4E196FFAEEEAEE197A396FFAFEEAFB9
:107FB000A397812F8F70282F30E0AB963FAF2EAF65
:107FC000AB97002361F1232B09F4C0C1873039F549
:107FD000013109F493C1023109F4B0C10031F9F45F
:107FE0006FEF70E0CE018F5A9F4F0E947D332A962B
:107FF0002FAF2A972B963FAF2B972C964FAF2C97EE
:108000002D965FAF2D972E966FAF2E972F967FAF41
:108010002F9760968FAF609761969FAF6197A396F9
:10802000AEADBFADA3971496ED91FC91309709F4D6
:108030007DC286809780AD961FAE1EAEAD97A59689
:108040001FAE1EAEA5976F961FAE1EAE6F97712C1A
:10805000612C512C412C8114910409F473C268EBFA
:1080600074E0C4010E9423AE1C0161E175E0C4010B
:108070000E9423AE6B969FAF8EAF6B9760EC75E05E
:10808000C4010E9423AEAF969FAF8EAFAF9721146D
:10809000310409F42EC16B96EEADFFAD6B973097AE
:1080A00009F427C1D10118968C918F70823009F0A4
:1080B00020C180858F70823009F01BC164EC75E0AF
:1080C000C4010E9423AEDC0119962D913D914D9182
:1080D0005C911C97A9962CAF3DAF4EAF5FAFA997AF
:1080E000E196EEADFFADE197309709F4BBC0D40146
:1080F000CD90DC90BF01C6010E947BF5892B09F071
:10810000B1C062968FAD6297811127C163968FAD22
:108110006397807FAB96EEADFFADAB97379709F0D5
:10812000B2C1882309F478C0CE018F5A9F4F0E94B4
:1081300033616B96EEADFFAD6B970185128523859C
:108140003485672B682B692B09F4BAC102301105FD
:108150002105310529F00F3F1F4F2F4F3F4F31F5BC
:1081600066EC75E083EF9DE00E94669983EF9DE0E9
:108170000E94369821E030E040E050E06B96AEADD2
:10818000BFAD6B9719962D933D934D935C931C97C0
:1081900061E0CE018F5A9F4F0E945B3329A33AA31F
:1081A0004BA35CA36DA37EA38FA398A7CE018F5A88
:1081B0009F4F0E943361F1016187728783879487A3
:1081C0008091C3099091C409059731F1D401CD90F4
:1081D000DC90E12C93E0F92E62960FAD62976396E6
:1081E0001FAD639764962FAD649765963FAD659715
:1081F00066964FAD669767965FAD679768966FAD69
:10820000689769967FAD6997A396EEADFFADA3978A
:10821000828193810E94DD6BAF96EEADFFADAF978B
:10822000309701F1B12CA12CD12CC12C6296EFAC6E
:1082300062976396FFAC639764960FAD64976596FB
:108240001FAD659766962FAD669767963FAD6797AA
:1082500068964FAD689769965FAD69976FEFCF01EC
:108260000E943B3D6B96EEADFFAD6B97818592858D
:10827000A385B48582309105A105B105A1F18F3F99
:108280009F4FAF4FBF4F79F1F10181859285A38553
:10829000B485A7964EAD5FADA797849F9001859F4B
:1082A000300D949F300D1124420E531EAD96EEAD4D
:1082B000FFADAD97AF01FF0F660B770B481759075E
:1082C0006A077B0784F4AD969FAF8EAFAD97A596F6
:1082D0003FAF2EAFA597A7962EAD3FADA7976F9650
:1082E0003FAF2EAF6F97A7964EAD5FADA797640EC9
:1082F000751ED40112968D909C90ADCE60E870E012
:10830000CE018F5A9F4F0E947D3322962FAF229726
:1083100023963FAF239724964FAF249725965FAFC0
:10832000259726966FAF269727967FAF2797289693
:108330008FAF289729969FAF299771CE6AE070E09A
:10834000CE018F5A9F4F0E94986069CE41E050E065
:10835000AB965FAF4EAFAB9762CE482F50E070E068
:1083600060E06B96AEADBFAD6B9719964D935D9384
:108370006D937C931C97813009F462C0823009F4BC
:1083800072C08091C3099091C409059761F16B9601
:10839000EEADFFAD6B9781859285A385B48501977E
:1083A000A105B10501F5F10181859285A385B4850B
:1083B0004497A105B105BCF42EE130E040E050E067
:1083C00021873287438754876EE170E0CE018F5A50
:1083D0009F4F0E947D3329A73AA74BA75CA76DA7A3
:1083E0007EA78FA798AB8091C3099091C409059788
:1083F00009F412CFF401C080D180E12C23E0F22EE9
:1084000062960FAD629763961FAD639764962FAD2A
:10841000649765963FAD659766964FAD669767968C
:108420005FAD679768966FAD689769967FAD6997FE
:10843000A396AEADBFADA39712968D919C91EACE57
:10844000F10161857285CE018F5A9F4F0E947D3365
:1084500029AF3AAF4BAF5CAF6DAF7EAF8FAF219618
:108460009FAF21978ECF70E060E0CE018F5A9F4F73
:108470000E947D3329AB3AAB4BAB5CAB6DAB7EABB3
:108480008FAB98AF7ECF882309F4C6CE60E0CE01D3
:108490008F5A9F4F0E94B233092E000CAA0BBB0BC0
:1084A000F10181879287A387B4878091C309909156
:1084B000C409059709F4B0CEE12C82E0F82EA0CFD4
:1084C000023011052105310559F10F3F1F4F2F4F84
:1084D0003F4F31F161ED75E083EF9DE00E946699B9
:1084E00083EF9DE00E94369822E030E040E050E0CB
:1084F0006B96AEADBFAD6B9719962D933D934D9393
:108500005C931C9762E0CE018F5A9F4F0E945B33B1
:10851000298F3A8F4B8F5C8F6D8F7E8F8F8F98A3B3
:10852000F10111861286138614864ACEA5961FAED7
:108530001EAEA5976F961FAE1EAE6F97712C612C65
:10854000512C412C6114710409F4C3C1C201B3015F
:108550000E9406F14B0166EB74E183EF9DE00E94FF
:10856000CC99B30183EF9DE00E94AAAE6BEA74E15F
:1085700083EF9DE00E94CC990FEF10E0C201B8019B
:108580000E9406F183EF9DE00E94AAAE64EA74E1C6
:1085900083EF9DE00E94CC99B40183EF9DE00E949F
:1085A000AAAE66E974E183EF9DE00E94CC99A5969E
:1085B0008EAD9FADA597B8010E9406F183EF9DE0B7
:1085C0000E94AAAE6FE874E183EF9DE00E94CC990F
:1085D0006F966EAD7FAD6F9783EF9DE00E94AAAE60
:1085E0006BE874E183EF9DE00E94CC9983EF9DE0FE
:1085F0000E94369819821A821B821C821D821E825A
:108600001F8218868A818F708A83B401CE010196F9
:108610000E947D3329873A874B875C876D877E87E9
:108620008F87988B61E08114910409F462E0CE0198
:1086300009960E945B3379018A012B013C01298B49
:10864000FA8A4B8B1C8B6D8B5E8A8F8B788E67E0E2
:1086500077E0A396EEADFFADA397848195810E944C
:1086600023AEB12CA12CD12CC12C9201A3016FEF10
:108670000E943B3D8928E1F481E090E0C059DF4F42
:108680000FB6F894DEBF0FBECDBFDF91CF911F9123
:108690000F91FF90EF90DF90CF90BF90AF909F90A1
:1086A0008F907F906F905F904F903F902F900895A4
:1086B000A396AEADBFADA3971496ED91FC91309704
:1086C000D9F2868097806F962EAD3FAD6F97032EBF
:1086D000000C440B550BA1962CAF3DAF4EAF5FAFD6
:1086E000A197A5968EAD9FADA597092E000CAA0B5C
:1086F000BB0B6D968CAF9DAFAEAFBFAF6D978114C6
:10870000910409F4B9CF64EC75E0C4010E9423AE72
:108710008C0165EA74E0C4010E9423AE3C0168EB61
:1087200074E0C4010E9423AE2C0161E175E0C40134
:108730000E9423AE6114710409F4C3C041145104B2
:1087400009F4BFC0009709F4BCC0D30118962C915E
:108750002F70223009F0B5C0F20120852F70223031
:1087600009F0AFC0DC0118962C9118972F702230B9
:1087700009F0A7C0F801C184D284E384F484C11451
:10878000D10409F49EC019968D919D910D90BC91D4
:10879000A02D82309105A105B10509F496C08F3F47
:1087A0009F4FAF4FBF4F09F490C0A5962EAD3FAD80
:1087B000A597232B09F489C0D20119968D919C911C
:1087C0008C9D80018D9D100D9C9D100D11242FEF0F
:1087D00030E0D8010E9431F19601DD0C440B550BBD
:1087E0000E94B1F0A1966CAD7DAD8EAD9FADA1970D
:1087F0000E947FF06D962CAD3DAD4EAD5FAD6D9797
:108800000E94B1F019012A01F4016081718183EFA6
:108810009DE00E9466996DED75E083EF9DE00E94FA
:108820006699C8016FEF70E00E9406F183EF9DE04A
:108830000E94AAAE65E874E183EF9DE00E94CC99A6
:108840002AE030E0B201A10183EF9DE00E94DC98B4
:1088500083EF9DE00E943698F30181859285A38580
:10886000B48582159305A405B50559F119861A86B4
:108870001B861C861D861E861F86188A8A858F7019
:108880008A87B101CE0109960E947D3329833A83FC
:108890004B835C836D837E838F839887B12CA12C5F
:1088A000D12CC12C79018A019B01AC016FEFC4016D
:1088B0000E943B3DD30119962D923D924D925C92C0
:1088C0001C97F401828093801ACF212C312C210136
:1088D000C3CF90E080E0D2CE8F929F92AF92BF92B2
:1088E000CF92DF92EF92FF920F931F93CF93DF937C
:1088F000CDB7DEB7CD55D1090FB6F894DEBF0FBEA8
:10890000CDBF8C016B016115710519F04115510541
:10891000D1F463E678E083EF9DE00E94CC996AE5AC
:1089200078E083EF9DE00E94CC99B80183EF9DE051
:108930000E94669968E578E083EF9DE00E94CC99FB
:1089400083EF9DE030C0460F571FDA011C920E9452
:108950003F294B0166E578E083EF9DE00E94CC99CA
:10896000B40183EF9DE00E94AAAE63E578E083EF57
:108970009DE00E94CC99B80183EF9DE00E9466992A
:1089800060E578E083EF9DE00E94CC99BAE38B1616
:10899000B1E09B06F4F463E478E089EE9DE00E9488
:1089A000CC9989EE9DE00E943698C35ADF4F0FB6EE
:1089B000F894DEBF0FBECDBFDF91CF911F910F9115
:1089C000FF90EF90DF90CF90BF90AF909F908F90EF
:1089D000089561E478E083EF9DE00E94CC99B601B0
:1089E00083EF9DE00E9466996FE378E083EF9DE05E
:1089F0000E94CC9983EF9DE00E9436981A821982DA
:108A0000FE0133968EE3DF011D928A95E9F780918E
:108A1000C3099091C409059791F563E070E0C8011E
:108A20000E94AC287C01892BE9F5E091200DF091A2
:108A3000210D808180FFB9CF61E070E0C8010E9404
:108A4000AC28892B09F4B1CF64E270E0C8010E9420
:108A5000B8F5892B09F0A9CF67E278E083EF9DE0B4
:108A60000E94CC99B80183EF9DE00E94669983EF44
:108A70009DE00E943698C8010E94D8B896CF61E068
:108A800070E0C8010E94AC287C01892B21F562E0CE
:108A900070E0C8010E94AC287C016CE178E0892B71
:108AA00009F44ACFE00EF11E63E178E0C7010E94AD
:108AB00050E9892BC1F4F60101900020E9F73197C4
:108AC000EC19FD09329778F0C8010E94D8B8C601A8
:108AD0000E947F9D6ACF4FE350E0B801CE0101961E
:108AE0000E94A9F5DFCF64E270E0C8010E94B8F5EA
:108AF000892B09F05ACFB701CE018F5B9F4F0E949F
:108B00001471CE018F5B9F4F0E94CF68882339F18B
:108B1000B601CE018F5B9F4F0E9414B31816190641
:108B2000F4F489818823D9F08091C3099091C40914
:108B30000597A9F06BEF77E083EF9DE00E94CC9959
:108B4000BE016F5F7F4F83EF9DE00E94669983EFC8
:108B50009DE00E943698CE0101960E94D8B8CE01C1
:108B60008F5B9F4F0E94A07120CFEF92FF920F93D7
:108B70001F93CF93DF93CDB7DEB764970FB6F8940A
:108B8000DEBF0FBECDBF0D871E872F87388B498B69
:108B90005A8B6B8B7C8B65E474E183EF9DE00E94C4
:108BA000CC99CE010D960E94A4319E85892F8F709D
:108BB000082F10E02D85222309F4B7C001151105F7
:108BC00009F488C0813009F485C08130A8F1823071
:108BD00009F44AC08D3009F094C092959F7069895C
:108BE0007A899C3011F070E060E0CE0101960E941D
:108BF00007976EEF75E0C7010E947BF5892B09F09E
:108C000051C0BE016F5F7F4FCE0107960E94FE9656
:108C1000CE0107960E9421B9BC0181EB9BE00E9426
:108C2000BE99CE0107960E94CB9601E010E0CE01DE
:108C300001960E94CB9628C0EF2861F066E374E1AC
:108C400083EF9DE00E94CC9983EF9DE00E943698CF
:108C500000E066C065E274E183EF9DE00E94CC997C
:108C600083EF9DE00E94369861E174E183EF9DE01F
:108C70000E94CC9983EF9DE00E9436988E85807F7C
:108C800001E010E009F400E0C80164960FB6F89422
:108C9000DEBF0FBECDBFDF91CF911F910F91FF902F
:108CA000EF9008956EE076E0C7010E947BF500E04A
:108CB000892B09F0BBCFBE016F5F7F4FCE010796B6
:108CC0000E94FE96CE0107960E9421B9BC0184E164
:108CD0009BE0A5CF213009F1223021F164E074E15D
:108CE00083EF9DE00E94CC994AE050E06D8583EFD0
:108CF0009DE00E943A9883EF9DE00E94369801E043
:108D000010E064EF73E183EF9DE00E94CC99B8011D
:108D100083EF9DE00E94AAAE97CF2093270201E047
:108D200010E0B2CF10922702FACF813009F04DCF78
:108D3000D5CFDF92EF92FF920F931F93CF93DF93E4
:108D400000D000D0CDB7DEB78C017B0165ED73E1BB
:108D5000CE0101960E94D096BE016F5F7F4FC70182
:108D60000E946195D82ECE0101960E94CB96DD20FF
:108D700019F1D8011296ED91FC9113970190F081B1
:108D8000E02D60817181ED91FC910288F389E02DE5
:108D900023EE35E044EC56E0C801199526960FB64F
:108DA000F894DEBF0FBECDBFDF91CF911F910F9121
:108DB000FF90EF90DF9008956AEB73E1CE0101968A
:108DC0000E94D096BE016F5F7F4FC7010E946195E0
:108DD000D82ECE0101960E94CB96DD20A1F0D801BD
:108DE0001296ED91FC9113970190F081E02D608136
:108DF0007181ED91FC910288F389E02D23EE35E03D
:108E000047EB56E0C9CF6FE973E1CE0101960E94AE
:108E1000D096BE016F5F7F4FC7010E946195F82E0B
:108E2000CE0101960E94CB96FF2009F4B7CFD8015E
:108E30001296ED91FC9113970190F081E02D6081E5
:108E40007181ED91FC910288F389E02D23EE35E0EC
:108E50004AEE55E0A1CF6F927F928F929F92AF9290
:108E6000BF92CF92DF92EF92FF920F931F93CF9317
:108E7000DF93CDB7DEB72C970FB6F894DEBF0FBEE9
:108E8000CDBF4C0181EB9BE00E941B8F892B39F1F8
:108E900080E00E9483226093EB087093EC0880933B
:108EA000ED089093EE0881EB9BE00E94F98E682E0E
:108EB0008DE290E09A83898369824FE350E0BE019E
:108EC0006F5F7F4F81E698E00E948BF58091E90803
:108ED0009091EA0801969093EA088093E90884E16A
:108EE0009BE00E941B8F892B39F180E00E94832236
:108EF0006093E5087093E6088093E7089093E8088C
:108F000084E19BE00E94F98E782E8DE290E09A83B6
:108F1000898379824FE350E0BE016F5F7F4F83EA20
:108F200098E00E948BF58091E3089091E408019607
:108F30009093E4088093E3088091EB089091EC080B
:108F4000A091ED08B091EE08892B8A2B8B2B09F0AC
:108F5000C7C08AE26812DEC01092EB081092EC08DB
:108F60001092ED081092EE081092EA081092E908AB
:108F700061E678E0CE0107960E940797109261089B
:108F8000CE0107960E945F948B859C85892B09F4FE
:108F9000DEC16CEE75E0CE0101960E940797BE011E
:108FA0006F5F7F4FCE0107960E943195182FCE013B
:108FB00001960E94CB96112321F0809127028823ED
:108FC000A1F0BE01695F7F4FCE0101960E94FE961F
:108FD000CE0101960E9421B9BC0184E19BE00E9470
:108FE000BE99CE0101960E94CB96BE01695F7F4F6C
:108FF000CE0101960E94FE96BE016F5F7F4FC401B5
:109000000E949946CE0101960E94CB9665EF75E0CD
:10901000CE0101960E940797BE016F5F7F4FCE0180
:1090200007960E943195182FCE0101960E94CB968B
:10903000112309F44FC1BE01695F7F4F8CE29EE0AE
:109040000E946195811183C1BE01695F7F4F8CE2EF
:109050009EE00E94B4964F815885D4011296ED91FE
:10906000FC9113970190F081E02D60817181ED9169
:10907000FC910288F389E02D2BEF35E0C4011995AE
:109080008091A1089091A208892B09F460C160EF3A
:1090900073E183EF9DE00E94CC9910E000E0F0E1E5
:1090A000EF2EF12CB801CE0107960E941F95FC010E
:1090B0008081882309F447C18B859C85081719078F
:1090C00008F041C18091A1089091A20881309105DA
:1090D00009F442C1029709F46AC10F5F1F4FE2CF42
:1090E0000E9433BC9B01AC016091EB087091EC08CD
:1090F0008091ED089091EE08A12CB12C65011AE049
:10910000E12EF12C00E010E00E942122882309F4D6
:1091100020CF22CFADE06A1609F41ECF8091E90876
:109120009091EA088034910508F016CF8091E50807
:109130009091E608A091E708B091E808892B8A2B66
:109140008B2B09F040C1BAE27B1257C11092E5089F
:109150001092E6081092E7081092E8081092E408CE
:109160001092E30863EA78E0CE0107960E94079721
:109170001092A308CE0107960E945F948B859C8570
:10918000892B09F49AC16CEE75E0CE0101960E941C
:109190000797BE016F5F7F4FCE0107960E94319502
:1091A000182FCE0101960E94CB96112321F08091B9
:1091B00027028823A1F0BE01695F7F4FCE0101968F
:1091C0000E94FE96CE0101960E9421B9BC0181EB5E
:1091D0009BE00E94BE99CE0101960E94CB96BE01F3
:1091E000695F7F4FCE0101960E94FE96BE016F5FC0
:1091F0007F4FC4010E949946CE0101960E94CB96F2
:1092000065EF75E0CE0101960E940797BE016F5F82
:109210007F4FCE0107960E943195182FCE010196FF
:109220000E94CB96112309F40BC1BE01695F7F4FE9
:1092300088E39EE00E94619581113FC1BE01695F94
:109240007F4F88E39EE00E94B4964F815885D401F9
:109250001296ED91FC9113970190F081E02D6081C1
:109260007181ED91FC910288F389E02D2BE036E0CD
:10927000C40119958091A1089091A208892B09F445
:109280001CC162EF73E183EF9DE00E94CC99912CA9
:10929000812C00E110E0B401CE0107960E941F95D9
:1092A000FC018081882309F404C18B859C85881684
:1092B000990608F0FEC08091A1089091A208813023
:1092C000910509F4FFC0029709F427C1BFEF8B1A7B
:1092D0009B0AE1CF60E076E0CE0101960E940797FD
:1092E000BE016F5F7F4FCE0107960E943195182F08
:1092F000CE0101960E94CB96112309F4C1CEBE0186
:10930000695F7F4F82E39EE00E94619581111FC0DB
:10931000BE01695F7F4F82E39EE00E94B4964F8159
:109320005885D4011296ED91FC9113970190F0812C
:10933000E02D60817181ED91FC910288F389E02D2F
:1093400026E036E09BCE83EF9DE00E943698CE016A
:1093500007960E94CB96EACEB801CE0107960E94EE
:109360001F95DC018C9167E077E0803114F465EBA8
:1093700074E083EF9DE00E946699B801CE010796E4
:109380000E941F95FC018081082E000C990BAA0BEE
:10939000BB0B89839A83AB83BC83FE82ED82BE01C3
:1093A0006F5F7F4F83EF9DE00E94868696CEB80167
:1093B000CE0107960E941F95DC016C9183EF9DE022
:1093C0000E94D5988ACE0E9433BC9B01AC0160916B
:1093D000E5087091E6088091E7089091E808A12CD3
:1093E000B12C65011AE0E12EF12C00E010E00E94A2
:1093F0002122882309F4A7CEA9CEEDE07E1609F438
:10940000A5CE8091E3089091E4088034910508F09E
:109410009DCE81E090E02C960FB6F894DEBF0FBE93
:10942000CDBFDF91CF911F910F91FF90EF90DF9013
:10943000CF90BF90AF909F908F907F906F90089546
:1094400060E076E0CE0101960E940797BE016F5F53
:109450007F4FCE0107960E943195182FCE010196BD
:109460000E94CB96112309F405CFBE01695F7F4F9F
:109470008EE39EE00E94619581111FC0BE01695F6D
:109480007F4F8EE39EE00E94B4964F815885D401B1
:109490001296ED91FC9113970190F081E02D60817F
:1094A0007181ED91FC910288F389E02D20E136E095
:1094B000DFCE83EF9DE00E943698CE0107960E9492
:1094C000CB96A7CFB401CE0107960E941F95DC0171
:1094D0008C9167E077E0803114F465EB74E083EF02
:1094E0009DE00E946699B401CE0107960E941F95E7
:1094F000FC018081082E000C990BAA0BBB0B898301
:109500009A83AB83BC831E830D83BE016F5F7F4F45
:1095100083EF9DE00E948686D9CEB401CE010796E6
:109520000E941F95DC016C9183EF9DE00E94D5980D
:10953000CDCEFF920F931F93CF93DF9300D000D037
:10954000CDB7DEB78C01BC01CE0101960E94FE961C
:10955000BE016F5F7F4F83EF9DE00E94BE9983EF56
:109560009DE00E943698CE0101960E94CB966EEF48
:109570007DE0CE0101960E94D096BE016F5F7F4FC5
:10958000C8010E943195F82ECE0101960E94CB961B
:10959000FF2069F0B801CE0101960E94FE96CE012F
:1095A00001960E94D5C1CE0101960E94CB962696C7
:1095B0000FB6F894DEBF0FBECDBFDF91CF911F91E4
:1095C0000F91FF9008955F926F927F928F929F927A
:1095D000AF92BF92CF92DF92EF92FF920F931F93C1
:1095E000CF93DF93CDB7DEB7CF56D1090FB6F8943E
:1095F000DEBF0FBECDBF4C018B01F42E4AE050E020
:109600006F2D83EF9DE00E943A9869EF77E083EF3A
:109610009DE00E94CC99B801CE0101965C010E94A8
:10962000FE96B50183EF9DE00E94BE9983EF9DE019
:109630000E943698C5010E94CB9692E0F9126BC247
:1096400067EF77E0C5010E94D096B501C8010E947E
:109650006195F82EC5010E94CB96FF2009F4D0C277
:1096600020E04DE251E0B4018AE89DE00E94519D66
:10967000E090B909F090BA0960EF77E0CE01865921
:109680009F4F0E94D09669EE77E0CE018C599F4F94
:109690000E94D096CE01885A9F4F0E94BE206E969F
:1096A0001FAD6E976D960FAD6D976C96DFAC6C9796
:1096B0006B96CFAC6B9767E077E0CE0181960E9406
:1096C0000797BE016F5D7F4FC5010E94FE966C2D0E
:1096D000C5010E941C9665E176E00E944D966D2DB5
:1096E0000E941C9665E176E00E944D96602F0E94D4
:1096F0001C9665E176E00E944D96612F0E941C96B3
:10970000BC01CE01825A9F4F0E94FE96C5010E9465
:10971000CB96CE0181960E94CB9664EE77E0CE0187
:109720008E5A9F4F0E94D09667E077E0CE01845B0F
:109730009F4F0E9407970BEB1DE0D80118966C9184
:1097400070E084E0759567958A95E1F7C5010E9400
:10975000C2AE4D815E8169817A81CE01845B9F4F6B
:109760000E949195C5010E94CB96F80160856F70AB
:1097700070E0C5010E94C2AE4D815E8169817A812F
:10978000CE01845B9F4F0E949195C5010E94CB96AC
:109790000F5F1F4FFDE0013C1F0779F66EED77E08C
:1097A000CE018A5B9F4F0E94D0966DEB77E0CE0191
:1097B00081960E94D096BE016F5D7F4FCE01CE96FE
:1097C0000E94FE96BE016A5B7F4FCE01CE960E943C
:1097D0006796BE01645B7F4F0E946796BE016E5A1A
:1097E0007F4F0E946796BE01625A7F4F0E94679624
:1097F000BE016C597F4F0E9467968C014AE0B5010B
:1098000080E590E00E94CCE9F50101900020E9F7A5
:109810003197AF014A195B09B501C8010E949195C2
:10982000811103C0C8010E940A96BE0166597F4F8C
:10983000C8010E946796B7010E944D96BC01C40101
:109840000E94BE99C4010E943698CE01CE960E9415
:10985000CB96CE0181960E94CB96CE018A5B9F4F1C
:109860000E94CB96CE01845B9F4F0E94CB96CE0187
:109870008E5A9F4F0E94CB96CE01825A9F4F0E94D4
:10988000CB96CE018C599F4F0E94CB96CE01865924
:109890009F4F0E94CB96C4010E94369864E670E008
:1098A00080E090E00E9401BCD401ED91FC9104881D
:1098B000F589E02DC401199501E010E088C02896D3
:1098C0006EAD7FAD2897CE0181960E9414B3892B8F
:1098D00009F450C122961CAE1DAE1EAE1FAE2297DB
:1098E00026961CAE1DAE1EAE1FAE26978FAD8F7096
:1098F0008FAF40E053E0BE016F5D7F4FCE01CE964B
:109900000E94A43200E020E033E040E250E0B501E4
:10991000CE01CE960E94832FBC01C6010E94A5965F
:1099200008EC10E129C1EE2009F4F3C046E050E054
:1099300070E060E0C8010E94BC94D8016D917C91F8
:10994000CE0181960E941471CE0181960E94CF684B
:1099500000E911E08823B9F189A5873061F4CE01CF
:1099600081960E94847261E0892B09F462E0CE0145
:1099700081960E94947022961CAE1DAE1EAE1FAE44
:10998000229726961CAE1DAE1EAE1FAE26978FAD3B
:109990008F708FAF40E053E0BE016F5D7F4FCE010F
:1099A000CE960E94A43200E020E033E040E250E096
:1099B000B501CE01CE960E94832FBC01C6010E9444
:1099C000A59608EC10E1CE0181960E94A071C80115
:1099D000C159DF4F0FB6F894DEBF0FBECDBFDF9188
:1099E000CF911F910F91FF90EF90DF90CF90BF909C
:1099F000AF909F908F907F906F905F900895F80147
:109A0000608171810E9423AE7C01892B09F040C1E5
:109A100004E911E0DCCFEE2009F47BC049E050E01E
:109A200070E060E0C8010E94BC944AE0B401C50146
:109A30000E94909741E050E062E475E0C8010E9406
:109A400091954D815E8169817A81C8010E949195CD
:109A500069E977E083EF9DE00E94CC99B801CE01DF
:109A600081960E94FE96BE016F5D7F4F83EF9DE061
:109A70000E94BE9983EF9DE00E943698CE018196A8
:109A80000E94CB9661E977E0CE0181960E94D09644
:109A9000F801848195812DA13EA182179307E1F4FD
:109AA000892BA1F1E080F18069A07AA0D7018D9186
:109AB0007D01882359F1082E000C990B0E9400F5B6
:109AC0006C01F30181913F01082E000C990B0E945B
:109AD00000F5C816D90651F3CE0181960E94CB96A7
:109AE000552041F021E048EC50E0B4018AE89DE0C7
:109AF0000E94519DD8018D919C910E947F9D00975D
:109B000011F484E991E08C01C5013DC055245394C2
:109B1000E3CF01E97ECFB1E0FB1270C066EB77E0E6
:109B2000C5010E94D096B501C8010E943195582EFA
:109B3000C5010E94CB96552049F1EE2051F346E035
:109B400050E070E060E0C8010E94BC944AE0B401BB
:109B5000CE018A5B9F4F0E949097F80160817181CE
:109B6000CE0181960E941471CE0181960E94CF6829
:109B70008111A5CE00E911E0CE0181960E94A0716D
:109B8000CE018A5B9F4F0E94CB9621CF6FE977E091
:109B9000C5010E94D096B501C8010E943195F82EEA
:109BA000C5010E94CB96F11036CF64E877E0C5017D
:109BB0000E94D096B501C8010E943195182FC501A9
:109BC0000E94CB9600E0112309F401CF80E00E94AF
:109BD00002B26CE577E08FED9DE00E94CC998FEDAD
:109BE0009DE00E94369867E077E0C5010E940797E4
:109BF000C5010E94D5C1C5010E94CB9600E05DCE93
:109C00006FEA77E0C5010E94D096B501C8010E94B5
:109C10003195F82EC5010E94CB96F11084CE69EAE9
:109C200077E0C5010E94D096B501C8010E94319528
:109C3000F82EC5010E94CB96FF2001F3EE2009F417
:109C400068CF45E050E070E060E0C8010E94BC943D
:109C500065E176E0C8010E944C95882339F0E090D8
:109C6000C509F090C609E114F10491F467E077E0CA
:109C7000C8010E944C95811107C08091C50990913F
:109C8000C609009709F0BBCEE090A607F090A707A1
:109C900020E048EC50E2B4018AE89DE00E94519D2A
:109CA000C4010E9436981C821B8284E992E09A8348
:109CB00089839E828D828FEF9FEF98878F83B70174
:109CC000C5010E94569EEACDAF92BF92CF92DF921D
:109CD000EF92FF920F931F93CF93DF93CDB7DEB731
:109CE0006D970FB6F894DEBF0FBECDBF0E9433BC98
:109CF0009B01AC016091200870912108809122089D
:109D000090912308A12CB12C650118EEE12E13E0EF
:109D1000F12E00E010E00E942122F82E882351F05D
:109D20000E9433BC6093200870932108809322081E
:109D3000909323088091C1098F5F8093C109E091BE
:109D4000C509F091C6090681178194E0C92ED12C6E
:109D5000F11003C082E0C82ED12CA090C509B090AC
:109D6000C609A114B10429F10115110511F1F80179
:109D700080858F708530A9F7C8010E94B2AE82300D
:109D800080F3B801CE0101960E94AE71CE0101961A
:109D90000E94CF68882329F0B601CE0101960E9467
:109DA000A284F80102811381CE0101960E94A07164
:109DB000D4CF8091C10981508093C1098091C3099A
:109DC0009091C4090597D9F1FF20C9F110E0609185
:109DD0002608709127086115710589F111112FC0AE
:109DE000FB0180858F70853091F4CE0101960E9431
:109DF000AE7161E070E0CE0101960E94A28411E094
:109E0000892B09F410E0CE0101960E94A071E09127
:109E10002608F0912708309791F0828193819093E2
:109E2000270880932608892B91F6E091C509F091C7
:109E3000C6098681978190932708809326086D969E
:109E40000FB6F894DEBF0FBECDBFDF91CF911F914B
:109E50000F91FF90EF90DF90CF90BF90AF9008955B
:109E60002F923F924F925F926F927F928F929F922A
:109E7000AF92BF92CF92DF92EF92FF920F931F9318
:109E8000CF93DF93CDB7DEB7C955D1090FB6F8949C
:109E9000DEBF0FBECDBF0E9433BC9B01AC01609101
:109EA0001C0870911D0880911E0890911F08A12C1C
:109EB000B12C650110E3E12E15E7F12E00E010E072
:109EC0000E942122882309F424C2E091C509F0915F
:109ED000C609309709F41DC28091C1098F5F809334
:109EE000C1092680378010E02114310409F434C1FF
:109EF000F10180858F708530F9F460E0C1010E9426
:109F00009BAEFC0181859285A385B4850597A1054B
:109F1000B10591F4B101CE0101960E94AE71CE015E
:109F200001960E94CF6866968FAF6697811108C030
:109F3000CE0101960E94A071F10122803380D4CF1E
:109F400025961CAE1DAE1EAE1FAE259729961CAEE3
:109F50001DAE1EAE1FAE299740E052E0BE016F5FFE
:109F60007F4FCE018F5B9F4F0E94A432CE0101969E
:109F70000E9484696B017C0169966FAF69976A964C
:109F8000DFAE6A9770E060E0CE0101960E94CA6978
:109F90004C01CE018F5B9F4F0E94EC6065966CAFC9
:109FA0007DAF8EAF9FAF6597CE0101960E94C570C1
:109FB000182FB601DD0C880B990B0E944CEF20E0A6
:109FC00030E048EC52E40E94A5F12B013C01CE01A7
:109FD00001960E94847268969FAF8EAF689769E67B
:109FE00071E183EF9DE00E94CC9965966CAD7DADEB
:109FF0008EAD9FAD65970E94C7B563E671E183EFB3
:10A000009DE00E94CC99C301B2010E94C7B56DE5E5
:10A0100071E183EF9DE00E94CC99612F70E083EFA6
:10A020009DE00E94AAAEE114F10409F48EC088E01C
:10A030000E9483229B01AC0144275527B70190E081
:10A0400080E0AA24AA94BA2CC12CD12C17E2E12ECC
:10A0500019E0F12E00E010E00E942122882371F126
:10A06000F1016081718189EE9DE00E9466996DE445
:10A0700071E189EE9DE00E94CC99F10160817181CE
:10A0800087E196E00E941CBD90E080E0BC016996EB
:10A090004FAD69976A965FAD6A97CE0101960E94AF
:10A0A000246962E070E0C4010E945F19CE0101964C
:10A0B0000E94A07166961FAD66973ECF20E030E00B
:10A0C00048E152E4C301B2010E944DF218163CF47B
:10A0D000F1016081718183E296E00E941CBD689667
:10A0E0008EAD9FAD6897892B19F461E070E0DBCFEE
:10A0F00020E030E040E85FE365966CAD7DAD8EAD6D
:10A100009FAD65970E9438F19B01AC01C301B2017C
:10A110000E9445EF70E060E087FDC5CFA30192018A
:10A1200065966CAD7DAD8EAD9FAD65970E9445EF98
:10A130001816DCF66EE371E183EF9DE00E94CC9986
:10A1400083EF9DE00E943698B1CF64E371E183EF25
:10A150009DE00E94CC99AACF8091C1098150809343
:10A16000C1090E9433BC60931C0870931D08809342
:10A170001E0890931F080E943F292B013C010E945A
:10A1800033BC6B017C010E9441AE882309F489C075
:10A190008091A807811185C030E020E041E050E0C7
:10A1A00060E4CE0101960E9418284FE350E06CEE67
:10A1B0007CE1CE0101960E9469E96FE175E0CE0174
:10A1C00001960E9465F54FE350E06BE071E1CE012E
:10A1D00001960E9469E92AE0AE014F5B5F4FC3011F
:10A1E000B2010E94F4E9BE016F5B7F4FCE01019680
:10A1F0000E9401BD30E020E041E050E060E4CE018B
:10A2000001960E9418284FE350E06CEE7CE1CE01ED
:10A2100001960E9469E96FE175E0CE0101960E9406
:10A2200065F54FE350E064E071E1CE0101960E94D4
:10A2300069E9C701B60128EE33E040E050E00E9432
:10A240008FF0CA01B9012AE0AE014F5B5F4F0E9457
:10A25000F4E9BE016F5B7F4FCE0101960E9401BD04
:10A2600030E020E041E050E060E4CE0101960E9441
:10A2700018284FE350E06CE17DE1CE0101960E9489
:10A2800069E94FE050E066E17DE1CE018F5B9F4FD1
:10A290000E9487E9BE016F5B7F4FCE0101960E944D
:10A2A00001BD112309F44FC06EE271E183EF9DE01F
:10A2B0000E94CC990E943F29AB01BC012AE083EFA8
:10A2C0009DE00E94EA9766E271E183EF9DE00E94C3
:10A2D000CC996091C109062E000C770B83EF9DE0AD
:10A2E0000E94AAAE64E171E183EF9DE00E94CC99E7
:10A2F000409118085091190860911A0870911B0834
:10A300002AE083EF9DE00E94EA9783EF9DE00E94A0
:10A310003698C75ADF4F0FB6F894DEBF0FBECDBFD9
:10A32000DF91CF911F910F91FF90EF90DF90CF9031
:10A33000BF90AF909F908F907F906F905F904F9065
:10A340003F902F90089564E271E183EF9DE00E94B9
:10A35000CC990E943F29AB01BC012AE083EF9DE02C
:10A360000E94EA976CE171E1B0CF4F925F926F92D9
:10A370007F92AF92BF92CF92DF92EF92FF920F93B4
:10A380001F93CF93DF93CDB7DEB76D970FB6F894D9
:10A39000DEBF0FBECDBF67EF71E183EF9DE00E948E
:10A3A000CC9983EF9DE00E9436980E9433BC2B012C
:10A3B0003C018091C109882341F10E9433BC9B017B
:10A3C000AC01A12CB12C650110E1E12E17E2F12EB8
:10A3D00000E010E0C301B2010E942122811115C0EA
:10A3E0008091C3099091C409059741F08091C509F6
:10A3F0009091C609892B11F00E94644E0E94304F43
:10A4000082E090E00E94B82AD4CF8091C109FF2455
:10A41000F394882359F064ED71E189EE9DE00E9488
:10A42000CC9989EE9DE00E943698F12C6EEB71E19B
:10A4300083EF9DE00E94CC9983EF9DE00E943698C7
:10A44000809128088F5F80932808E091C509F091DA
:10A45000C609309781F1068117810115110559F15F
:10A46000D80118968C918F708530B9F7C8010E9479
:10A47000B2AE882391F3F80160817181CE0101961B
:10A480000E941471CE0101960E94CF68882359F072
:10A490008A859B85009739F0DC01ED91FC9102845F
:10A4A000F385E02D1995CE0101960E94A071F80167
:10A4B00002811381D2CF109227081092260866EBF2
:10A4C00071E183EF9DE00E94CC9983EF9DE00E94B3
:10A4D000369864E670E080E090E00E9401BC109243
:10A4E00047091092C2096EE971E183EF9DE00E9475
:10A4F000CC990E943F29AB01BC012AE083EF9DE08B
:10A500000E94EA978091A6079091A707009711F003
:10A510000E949CB61092A7071092A60710922508D9
:10A52000109224081092C6091092C5091092490988
:10A53000109248091092BF091092BE091092BA09F0
:10A540001092B90969E971E183EF9DE00E94CC990D
:10A550000E943F29AB01BC012AE083EF9DE00E94ED
:10A56000EA9783EF9DE00E9436981092C00980918F
:10A5700028088150809328088F2D6D960FB6F89487
:10A58000DEBF0FBECDBFDF91CF911F910F91FF9026
:10A59000EF90DF90CF90BF90AF907F906F905F90E3
:10A5A0004F9008958F929F92BF92CF92DF92EF9239
:10A5B000FF920F931F93CF93DF93CDB7DEB7A3978F
:10A5C0000FB6F894DEBF0FBECDBF8091A607909165
:10A5D000A707892B09F452C28091C10981114EC28B
:10A5E0008091C1098F5F8093C1096BE77CE08FED9B
:10A5F0009DE00E94CC998FED9DE00E9436980091DD
:10A60000A6071091A70760E376E0C8010E9423AE79
:10A610009093C6098093C50966E376E0C8010E945D
:10A6200023AE90934909809348096BEF76E0C80107
:10A630000E9423AE90932508809324086DE376E072
:10A64000C8010E9423AE9093BF098093BE090E9467
:10A65000BB2D1092270810922608E091C509F091B1
:10A66000C609309709F4FAC0E680F7800091C50961
:10A670001091C6090115110509F4E9C0E114F104AE
:10A6800009F4E5C0D70118968C918F70853091F749
:10A69000C7010E94B2AE823068F3B701CE010196C5
:10A6A0000E94AE71CE0101960E94CF68882309F402
:10A6B00068C08A859B85009769F570E060E0CE01EF
:10A6C00001960E94CA698C01912C812C97FF06C0CB
:10A6D00011950195110988248394912CCE0101963E
:10A6E0000E94C570C82ED12C8985853009F452C0CE
:10A6F000863009F046C0B02E61E0802F0E94A9BAD2
:10A7000061E0892809F481C0CA94CD2809F081C08C
:10A7100060E07FC0DC01ED91FC910484F585E02DC3
:10A720001995892B49F08A859B85DC01ED91FC9177
:10A730000284F385E02D19958A859B85DC01ED91D6
:10A74000FC910680F781E02D1995892BD1F0CE017F
:10A7500001960E94C570882341F040E051E060E01E
:10A7600070E0CE0101960E94906B8D819E81892BB5
:10A7700041F040E052E060E070E0CE0101960E94BE
:10A78000906BD7011296ED90FC90CE0101960E943D
:10A79000A0716CCFCD2829F462E0CE0101960E9411
:10A7A000947040E051E060E070E0CE0101960E94BC
:10A7B000906B8D819E81892B41F040E052E060E0FA
:10A7C00070E0CE0101960E94906B61E0802F0E94A4
:10A7D000A9BA60E0802F0E947BBA63E77CE083EF38
:10A7E0009DE00E94CC99B80183EF9DE00E94AAAE43
:10A7F0006EE67CE083EF9DE00E94CC996CE67CE005
:10A8000083EF9DE00E94CC99BCCFCA94CD2809F07B
:10A810007FCFC62ED12C8B2D0E947BBA67E67CE0C1
:10A8200083EF9DE00E94CC99B80183EF9DE00E94E8
:10A83000AAAE65E67CE083EF9DE00E94CC99B6016C
:10A8400083EF9DE00E94AAAE63E67CE0D9CFF801D9
:10A8500086819781909327088093260883EF9DE057
:10A860000E943698E0912408F0912508309709F469
:10A870008AC08091C1098F5F8093C10906811781C9
:10A880000115110509F47AC0D80118968C918F70C2
:10A89000863009F069C01F8F0E8F70E060E0CE0136
:10A8A0004E960E948A8D8AA19BA1892B09F45CC0D7
:10A8B0008091A6079091A707892B09F455C0EE8CCB
:10A8C000FF8CF70180858F70863099F561E275E025
:10A8D000C7010E9423AE0097F1F0DC0118962C917D
:10A8E00018972F702530B9F41696CD90DC90C114CE
:10A8F000D104F9F0DA82C982B701CE0101960E9433
:10A900008A8DED81FE811082118212821382F601FE
:10A91000C280D380ECCFFA82E98270E060E0CE01A1
:10A9200001960E948A8D62E070E0CE0101960E943D
:10A930009686EAA1FBA1108211821282138288A15D
:10A94000843068F462E0823008F060E089A10E94FF
:10A95000A9BAEAA1FBA18181807F818305C08034EF
:10A9600041F060E0823431F0D80112960D911C91D3
:10A9700087CF62E089A10E94A9BAF6CF8091C10970
:10A9800081508093C10966E57CE08FED9DE00E94D7
:10A99000CC996EE47CE08FED9DE00E94CC9981E043
:10A9A0002091C5093091C609232B09F480E00E944B
:10A9B000931665E47CE08FED9DE00E94CC9981E0E8
:10A9C0002091240830912508232B09F480E00E946F
:10A9D00093166EE37CE08FED9DE00E94CC9981E0C0
:10A9E0002091BE093091BF09232B09F480E00E9419
:10A9F000931665E37CE08FED9DE00E94CC998091F9
:10AA000047090E9493168FED9DE00E94369860E3FF
:10AA10007CE08FED9DE00E94CC990E943F29AB0124
:10AA2000BC012AE08FED9DE00E94EA978FED9DE04A
:10AA30000E94369881E08093C2098CEA9DE00E94D2
:10AA4000B715882351F08CEA9DE00E94B72B84E073
:10AA500090E09093C4098093C3098091C3099091B9
:10AA6000C409079731F484E090E09093C40980937F
:10AA7000C3098091C10981508093C109A3960FB683
:10AA8000F894DEBF0FBECDBFDF91CF911F910F9124
:10AA9000FF90EF90DF90CF90BF909F908F900895A0
:10AAA0004F925F926F927F928F929F92AF92BF92DE
:10AAB000CF92DF92EF92FF920F931F93CF93DF938A
:10AAC000CDB7DEB7C859D1090FB6F894DEBF0FBEB7
:10AAD000CDBF8E010F5B1F4FD8011D921C92FE014E
:10AAE000ED5BFF4F8EE1DF011D928A95E9F78091C2
:10AAF000BB0D9091BC0D892B09F4CFC10E9403AF0F
:10AB0000882309F4CAC182E70E94EEAE8091BB0D92
:10AB10009091BC0DDC01ED91FC910088F189E02D54
:10AB200060E270E019954FE150E0B8018091BB0DF3
:10AB30009091BC0D0E9448AF7C018091BB0D90911B
:10AB4000BC0DDC01ED91FC910488F589E02D19958F
:10AB5000E114F10409F4A1C1F801EE0DFF1D10820A
:10AB60008091C80D1F928F938091C70D1F928F9374
:10AB70008091C60D1F928F938091C50D1F928F9368
:10AB80008091C40D1F928F938091C30D1F928F935C
:10AB900082E496E09F938F931F9280E48F93FE014F
:10ABA00031966F01FF93EF930E94C3F561EE7EE053
:10ABB0008FED9DE00E94CC99B8018FED9DE00E9441
:10ABC0006699B6018FED9DE00E9466998FED9DE03C
:10ABD0000E9436987E01F1E6EF0EF11CD701139624
:10ABE0001C921E92129788EE93E0A0E0B0E0F7016D
:10ABF00084839583A683B78388E0848788EE93E077
:10AC00009687858781E294E091838083108A1786F6
:10AC1000128B018B148A138A80E590E0968B858BCA
:10AC2000118E65E07EE083EF9DE00E94CC996DEB94
:10AC30007DE0CE0185589F4F0E94FE96BE0165586B
:10AC40007F4F83EF9DE00E94BE9983EF9DE00E94BD
:10AC50003698CE0185589F4F0E94CB9661E776E0EB
:10AC6000CE0183579F4F0E94079761E776E0CE01A0
:10AC700085589F4F0E940797BE0165587F4FCE01B0
:10AC80008B579F4F0E94FE966DEB7DE0CE018B5758
:10AC90009F4F0E946796BE0163577F4F0E94679641
:10ACA000BC01CE018D569F4F0E94FE96CE018B5760
:10ACB0009F4F0E94CB96CE0185589F4F0E94CB9606
:10ACC000CE0183579F4F0E94CB9683E796E0CB57E8
:10ACD000DF4F99838883C558D040C757DF4F19820B
:10ACE0001882C958D040C557DF4F19821882CB58F7
:10ACF000D040CD56DF4F88819981C359D040C95784
:10AD0000DF4F99838883C758D0406BED7EE083EF97
:10AD10009DE00E94CC990E943F29AB01BC012AE032
:10AD200083EF9DE00E94EA9783EF9DE00E943698B2
:10AD300064E670E080E090E00E9401BC89E99AE45A
:10AD4000D70150969C938E931F9761E478E981EA2E
:10AD500090EA0E945AEA8C010FB6F894DEBF0FBE4B
:10AD6000CDBF892B09F4F4C083E090E00E9417E77F
:10AD7000D8011D969C938E931C97FC01F182E08272
:10AD80001282C7010E94B715882319F0C7010E94DB
:10AD9000B72BD70153966D917C9154975596AD90F2
:10ADA000BC906115710509F48FC0CE0185589F4F85
:10ADB0000E94029AA501BE0165587F4FC7010E94FB
:10ADC000F22B181619060CF0C0C0D7015196BC9092
:10ADD00051975296AC90DF92CF9280E69EE09F937F
:10ADE0008F931F930F930E94E1EADF92CF928BE53E
:10ADF0009EE09F938F931F930F930E94E1EAD801E7
:10AE00001C96ED91FC9181E08283DF92CF9288E5E0
:10AE10009EE09F938F931F930F930E94E1EAD801C6
:10AE20001C96ED91FC911282AF92BF9282E29EE05D
:10AE30009F938F931F930F930E94E1EA0FB6F894AC
:10AE4000DEBF0FBECDBFB12C89E1C82E8EE0D82E5B
:10AE50008B2D94E08902F0011124A5E8B0E0AC0F3D
:10AE6000BD1FEA0FFB1F808191810097A9F122810C
:10AE7000338121153105C9F33F932F939F938F930E
:10AE8000DF92CF921F930F930E94E1EAB3940FB623
:10AE9000F894DEBF0FBECDBFDBCF40E250E063E1F0
:10AEA0007FE0C8010E9487E965EF7EE08FED9DE0BD
:10AEB0000E94CC99B8018FED9DE00E9466998FEDBC
:10AEC0009DE00E9436984CCEF70161897289A501F8
:10AED000C7010E94D91575CF8DE59EE09F938F9392
:10AEE0001F930F930E94E1EAD70158961C921E927D
:10AEF0005797D8011C96ED91FC91C080D1800F909E
:10AF00000F900F900F9033E3A32EB12CD601ED914B
:10AF1000FC910084F185E02DC601199541975CF400
:10AF2000B1E0AB1AB10839F064E170E080E090E084
:10AF30000E9401BCEBCFD601ED91FC910084F1851C
:10AF4000E02DC6011995419734F4C8010E947AA0FA
:10AF500010E000E05AC067E077E0CE0183579F4FD2
:10AF60000E940797912CA12CD601ED91FC910688A7
:10AF7000F789E02DC60119958823E1F1BDE0AB12F8
:10AF800001C0A92CD601ED91FC910688F789E02D2E
:10AF9000C60119958111D9C0D601ED91FC910084AB
:10AFA000F185E02DC6011995892B09F4E0C0D60181
:10AFB000ED91FC910284F385E02DC6011995B82E20
:10AFC000BAE08B1709F4D5C0EDE08E1709F4D1C0B3
:10AFD000FFEF8F1709F4CBC0682FCE0183579F4F27
:10AFE0000E94BD959A2CAB2CBFCFBAE0BB12FACF12
:10AFF000AB12F8CFCC24C394D12CCE0183579F4FF2
:10B000000E94CB96CD2809F4A3CFD7015796ED9097
:10B01000FC906DEC7EE083EF9DE00E94CC99B7013F
:10B0200083EF9DE00E94AAAE83EF9DE00E943698D8
:10B0300064E670E080E090E00E9401BC011511051B
:10B0400009F456C1B8ECEB16F10409F02FC161EC1C
:10B050007EE08FED9DE00E94CC9964EF71E080E08E
:10B0600090E00E9401BCEF961FAE1EAEEF97C15854
:10B07000DF4F19821882CF57D0408FEF9FEFCF5705
:10B08000DF4F99838883C158D0408EE792E0ED96D8
:10B090009FAF8EAFED97CD57DF4F19830883C3580D
:10B0A000D040F8948091A6079091A707892B11F0C2
:10B0B0000E94B551CE0185589F4F0E94CEB6909305
:10B0C000A7078093A6077894C8010E947AA0809170
:10B0D000A6079091A707892B09F0D6C067E077E013
:10B0E000CE0183579F4F0E940797CE0183579F4FF2
:10B0F0000E94D5C1CE0183579F4F0E94CB966AEA2A
:10B100007EE089EE9DE00E94CC99F12CE12CCE01ED
:10B110008D569F4F0E94CB96C701C856DF4F0FB682
:10B12000F894DEBF0FBECDBFDF91CF911F910F917D
:10B13000FF90EF90DF90CF90BF90AF909F908F9057
:10B140007F906F905F904F900895D601ED91FC91A4
:10B150000084F185E02DC6011995892B09F01CCFDB
:10B1600064E670E080E090E00E9401BC0BCFBB245D
:10B17000BA9461E876E08EE49CE00E946699BE0194
:10B1800063577F4F8EE49CE00E94BE998EE49CE062
:10B190000E94369860E17EE0CE0185589F4F0E9464
:10B1A000D096BE0165587F4FCE0183579F4F0E94B6
:10B1B0003195982ECE0185589F4F0E94CB969920AD
:10B1C00099F1CF56DF4F28813981C159D04049E0EC
:10B1D00050E0BE0163577F4FCE0185589F4F0E94BC
:10B1E0001C97ED968EAD9FADED97412C512C320101
:10B1F000009719F00E9402E92B014201CE01855807
:10B200009F4F0E94CB964114510429F0D7015896C4
:10B210005C924E925797B4018EE49CE00E94AAAED5
:10B220008EE49CE00E943698F70187849088811410
:10B230009104D1F0CF56DF4F88819981C159D04018
:10B24000892B91F0BE0163577F4FCE0185589F4FE8
:10B250000E94FE96CE0185589F4FF4011995CE01AC
:10B2600085589F4F0E94CB9667E077E0CE018357C9
:10B270009F4F0E949B96FFEFBF12B7CEC8010E945E
:10B280007AA0D12CC12CB9CE0E94D2528091C20991
:10B29000882329F00E9462B167FF0E94771C63EA4D
:10B2A0007EE08FED9DE00E94CC9931CFE0E3EE1679
:10B2B000E1E0FE0651F46FE87EE08FED9DE00E9434
:10B2C000CC99C8010E947AA022CF67E77EE089EE80
:10B2D0009DE00E94CC99C8010E947AA0B70189EE36
:10B2E0009DE00E94AAAE89EE9DE00E9436980FCFA5
:10B2F00064E67EE083EF9DE00E94CC99EE24EA9420
:10B30000FE2C05CF0F931F93CF93DF93EB01029792
:10B310000CF485C00A811B8167EF7DE0C8010E94A3
:10B3200032E9892B51F481E00E9402B288EC90E06E
:10B33000DF91CF911F910F91089563EF7DE0C801D8
:10B340000E9432E9892B11F480E0EECF63ED7DE0BD
:10B350008FED9DE00E94CC990E9462B163FB66274D
:10B3600060F981E0682770E08FED9DE00E94AAAE51
:10B370008FED9DE00E9436988091BB0D9091BC0DA1
:10B38000892BE9F10A811B810E9403AF8823B9F15F
:10B39000F80101900020E9F73197E01BF10BB0971D
:10B3A00070F582E70E94EEAE8091BB0D9091BC0DCE
:10B3B000DC01ED91FC910088F189E02D60E270E004
:10B3C0001995B8018091BB0D9091BC0D0E946699B2
:10B3D0008091BB0D9091BC0DDC01ED91FC91019031
:10B3E000F081E02D60E019958091BB0D9091BC0D2E
:10B3F000DC01ED91FC910488F589E02D19956A81B5
:10B400007B818FED9DE00E9466996CEC7DE08FED75
:10B410009DE00E94CC998FED9DE00E94369880912E
:10B42000C3099091C40902977CF10E945055883C51
:10B43000910539F424E030E03093C4092093C30926
:10B4400077CF8F3F9807C9F461EB7DE083EF9DE0F4
:10B450000E94CC9983EF9DE00E9436981092C0091B
:10B4600083E090E09093C4098093C3098CEA9DE047
:10B470000E94B72B89EC90E05BCF2091C20921118B
:10B48000D9CF2FE030E0D8CF64EA7DE089EE9DE0AF
:10B490000E94CC9989EE9DE00E94369884EF91E05D
:10B4A00047CFCF93DF93CDB7DEB72E970FB6F89483
:10B4B000DEBF0FBECDBF8091C109811178C060EEA3
:10B4C0007CE08FED9DE00E94CC998FED9DE00E9485
:10B4D00036981092DB0D1092DA0D80E090E1909397
:10B4E000D60D8093D50D84E890E09093DD0D809388
:10B4F000DC0D81E08093D70D80E090E29093D90D30
:10B500008093D80D82E78093DE0D89EC9DE00E9448
:10B51000905F8B37910509F0B9C068EC7CE083EF50
:10B520009DE00E94CC9983EF9DE00E9436981C829A
:10B530001B8284E992E09A83898389EC9DE09E8353
:10B540008D838FEF9FEF98878F838091A6079091CF
:10B55000A707892B11F00E94B551CE0101960E94D8
:10B56000CEB69093A7078093A60789EC9DE00E9432
:10B57000155C8091A6079091A707892BD9F46CEBF5
:10B580007CE089EE9DE00E94CC9989EE9DE00E94CE
:10B59000369867E077E0CE0109960E940797CE01C2
:10B5A00009960E94D5C1CE0109960E94CB9690E0E3
:10B5B00080E014C069EA7CE08FED9DE00E94CC99A8
:10B5C0008FED9DE00E9436980E94D2528091BB0D73
:10B5D0009091BC0D892B59F481E090E02E960FB626
:10B5E000F894DEBF0FBECDBFDF91CF9108950E94CA
:10B5F00003AF882389F382E70E94EEAE8091BB0DF2
:10B600009091BC0DDC01ED91FC910088F189E02D59
:10B6100060E670E019956091BB0D7091BC0D40E043
:10B62000CE0109960E949097BE01675F7F4F8DEB18
:10B630009DE00E94D195CE0109960E94CB96809103
:10B64000BB0D9091BC0DDC01ED91FC910488F58956
:10B65000E02D19956BE87CE083EF9DE00E94CC998A
:10B660006DEB7DE0CE0109960E94FE96BE01675FFC
:10B670007F4F83EF9DE00E94BE9983EF9DE00E9483
:10B680003698CE0109960E94CB96A6CF89EC9DE014
:10B690000E949A5B892BA1F089EC9DE00E94C45B1B
:10B6A00067E077E0CE0101960E940797CE010196F0
:10B6B0000E94D5C1CE0101960E94CB960E9444C241
:10B6C00089EC9DE00E94155C68E97CE08FED9DE0CF
:10B6D0000E94CC998FED9DE00E94369868CF0E9421
:10B6E000515A892B49F486EF9FEF9093C4098093B8
:10B6F000C30984EF91E0089588EC90E008958AE012
:10B7000090E0089581E090E0089588E090E0089549
:10B71000CF93DF93EC01E881F9810484F585E02D76
:10B72000199529893A892F5F3F4F3A8B298BDF91F1
:10B73000CF910895CF93DF93EC018E8581110DC0D9
:10B7400081E090E049895A892C853D85421753074D
:10B7500008F080E0DF91CF910895E881F9810484B9
:10B76000F585E02DCE0119958F3F910549F780E0D1
:10B7700090E0F0CFFC01848595856817790708F47F
:10B78000CB01928B818B0895DC011E962C911E9724
:10B79000222339F0ED91FC910190F081E02D6FEFC3
:10B7A00019940895FC0187859089089581E0089592
:10B7B00090E080E00895FC0122813381232B49F041
:10B7C000868197818130910539F01CF003970397AA
:10B7D00030F090E080E0089581E090E0089582E00C
:10B7E00090E008950F931F93CF93DF9300D000D084
:10B7F0001F921F92CDB7DEB781E028960FB6F8945E
:10B80000DEBF0FBECDBFDF91CF911F910F91089585
:10B8100090E080E0089564E379E1811102C06FE275
:10B8200079E183EF9DE00C94CC99DC0155962C9145
:10B830005597273781F4ED91FC91008CF18DE02D27
:10B8400019956BE076E183EF9DE00E94CC9983EF40
:10B850009DE00C9436980895DC011296ED91FC91D0
:10B86000309771F090859F70923039F0953041F4A7
:10B87000CF010E94B2AE90E0089581E090E008957B
:10B8800090E080E0089565E0FC01808191810E9454
:10B890009BAE009761F0FC01808585958595859527
:10B8A0008595181624F4082E000C990B089590E045
:10B8B00080E00895CF93DF93009709F490C0FC01D6
:10B8C0002081222309F48BC0EC0162E17AE10E941D
:10B8D00050E9892B09F45FC065EC79E1CE010E9443
:10B8E00050E9892B09F45AC069EE79E1CE010E9432
:10B8F00050E9892B09F455C06AE776E1CE010E9430
:10B9000050E9892B09F450C066E776E1CE010E9428
:10B9100050E9892B09F44BC062E776E1CE010E9421
:10B9200050E9892B09F446C06EE676E1CE010E940B
:10B9300050E9892B09F441C06AE676E1CE010E9404
:10B9400050E9892BE9F166E676E1CE010E9450E9E3
:10B95000892BC9F161E676E1CE010E9450E9892B7D
:10B96000A9F16DE576E1CE010E9450E9892B89F1BC
:10B9700066E17AE1CE010E9450E9892B69F169E51F
:10B9800076E1CE010E9450E9892B49F58DE090E0E7
:10B99000DF91CF91089582E090E0FACF89E090E0C6
:10B9A000F7CF81E090E0F4CF88E090E0F1CF85E040
:10B9B00090E0EECF86E090E0EBCF87E090E0E8CF3C
:10B9C0008AE090E0E5CF8BE090E0E2CF8CE090E081
:10B9D000DFCF83E090E0DCCF84E090E0D9CF90E04F
:10B9E00080E0D6CFCF92DF92EF92FF920F931F931A
:10B9F000CF93DF93CDB7DEB7C054D1090FB6F8941B
:10BA0000DEBF0FBECDBF8091C3099091C4090597D9
:10BA100009F449C06115710509F445C069017A014D
:10BA20008B0140E450E0CE0101960E94A9F56FE23F
:10BA300070E0CE0101960E9470F5892B41F49801C7
:10BA400043E050E060E4CE0101960E9418284FE3E5
:10BA500050E0B601CE0101960E948BF50E9441AEE6
:10BA6000882309F18091C3099091C4090697D9F4FC
:10BA70008091A807811117C0B701CE0101960E94DD
:10BA800001BD81E090E0C05CDF4F0FB6F894DEBFEF
:10BA90000FBECDBFDF91CF911F910F91FF90EF901F
:10BAA000DF90CF90089590E080E0EDCF6F927F928D
:10BAB0008F929F92AF92BF92CF92DF92EF92FF92BE
:10BAC0000F931F93CF93DF93CDB7DEB7A0970FB639
:10BAD000F894DEBF0FBECDBF8C01862E7A01DC014B
:10BAE0008D919C911197892B09F466C01496ED9164
:10BAF000FC91309709F460C080818071BFEF6B13B7
:10BB00005DC0B1F481E0A0960FB6F894DEBF0FBE21
:10BB1000CDBFDF91CF911F910F91FF90EF90DF90FC
:10BB2000CF90BF90AF909F908F907F906F9008952F
:10BB30004330510539F3818082942FE082226FE4F3
:10BB400076E183EF9DE00E94CC994AE050E0D80175
:10BB500013966C9183EF9DE00E943A986DE476E134
:10BB600083EF9DE00E94CC99D8011496ED91FC9151
:10BB700061816F704AE050E083EF9DE00E943A9847
:10BB80006AE476E183EF9DE00E94CC994AE050E0C0
:10BB9000682D83EF9DE00E943A9883EF9DE00E941C
:10BBA0003698D8011496ED91FC9181818F7088129E
:10BBB00007C080818F7E808380E0A5CF8111FCCF7C
:10BBC000198E1A8E1B8E1C8E1D8E1E8E1F8E18A215
:10BBD0008A8D8F708A8FD8011496ED91FC918181A6
:10BBE0008F708815A9F1B3E0EB16F10489F168E4D0
:10BBF00076E183EF9DE00E94CC994AE050E0F801A5
:10BC0000638183EF9DE00E943A9866E476E183EFDA
:10BC10009DE00E94CC99D8011496ED91FC91618130
:10BC20006F704AE050E083EF9DE00E943A9863E431
:10BC300076E183EF9DE00E94CC994AE050E0682DC8
:10BC400083EF9DE00E943A9883EF9DE00E94369832
:10BC5000F80120813181FCE0F81508F416C1E82DC7
:10BC6000F0E08827E95CF14A8F4F0C941AF1445EAA
:10BC7000815E025F195F255F025FDB5E025F285F06
:10BC8000335FEF5E365F425FD8011496CD90DC9053
:10BC9000F60181818F70853009F4F7C050F482304D
:10BCA000C1F062E976E0C9010E9423AE3C01912C0B
:10BCB0004BC08730D1F08A30A1F76BE876E0C9013C
:10BCC0000E9423AE3C01D6019C9092FA992490F8F0
:10BCD0003BC065E876E0C9010E9423AE3C01D60175
:10BCE0009C9090FA992490F82FC064E876E0C901FE
:10BCF0000E9423AE3C01F601908091FA992490F8BD
:10BD000023C067E976E0C9010E9423AE3C01D80157
:10BD10001496ED91FC91808180FB992490F8982FE6
:10BD20009E7F80FF916090836114710469F461E0EB
:10BD3000CE0149960E945B33298B3A8B4B8B5C8BEF
:10BD40006D8B7E8B8F8B988FF801A080B18062EA1B
:10BD500075E0C5010E9423AE6C0167EA75E0C5017C
:10BD60000E9423AE5C01892B81F4C114D10469F4D3
:10BD700060E0CE0149960E945B3329833A834B836E
:10BD80005C836D837E838F839887D8011496ED91B1
:10BD9000FC916114710409F07CC0898D811179C016
:10BDA000B82DBF708B2E8181807F882A818280810F
:10BDB0008F7E8083A7CE6CE976E0C9010E9423AE16
:10BDC0003C01D8011496ED91FC91808181FB99246E
:10BDD00090F8982F9D7F81FF92609083B5CF62EAA3
:10BDE00076E0C9010E9423AE3C01D8011496ED9182
:10BDF000FC91808182FB992490F8982F9B7F82FF91
:10BE00009460EBCF62E976E0C9010E9423AE3C0169
:10BE1000892B09F04CCF62E0CE0149960E945B333A
:10BE200029873A874B875C876D877E878F87988BBA
:10BE30003ECF68EA76E0C9010E9423AE3C01D801FA
:10BE40001496ED91FC9190804CCF6DEA76E0F3CFA3
:10BE500063EB76E0C9010E9423AE3C01D801149641
:10BE6000ED91FC9149CF69EB76E0F4CF60EC76E0A0
:10BE7000C9010E9423AE3C01D8011496ED91FC91BA
:10BE8000908023CF66EC76E0F3CF912C712C612C5F
:10BE90005BCF83E0E816F104B9F0982D9F70892EEE
:10BEA0008181807F882A818280818F7E8083E98C56
:10BEB000FA8C0B8D1C8D2D8D3E8D4F8D58A1692DCB
:10BEC000C3010E943B3D1ECE81818F70881509F40D
:10BED00019CE829490EF8922882A818280818061A4
:10BEE00068CF1F93CF93DF93FC01162FC389D489AA
:10BEF000818992899C012F5F3F4F328B218BC80F24
:10BF0000D91FCE010E9469F0181721F0612FCE01D0
:10BF10000E9471F081E090E0DF91CF911F91089530
:10BF2000FC0181899289248535858217930740F425
:10BF300023893489820F931F0E9469F090E008954D
:10BF40008FEF9FEF0895CF93DF93CDB7DEB7609764
:10BF50000FB6F894DEBF0FBECDBF19821A821B82C6
:10BF60001C821D821E821F8218868A818F708A839E
:10BF70006FEF70E0CE0101960E947D3360960FB6A0
:10BF8000F894DEBF0FBECDBFDF91CF9108952F9201
:10BF90003F924F925F926F927F928F929F92AF9259
:10BFA000BF92CF92DF92EF92FF920F931F93CF93A6
:10BFB000DF93CDB7DEB762970FB6F894DEBF0FBE42
:10BFC000CDBF5C014B0129013A01CA01B9010E94B0
:10BFD00017F21B013F926F9382E695E09F938F9338
:10BFE000CE0101967C019F938F930E9400F60F90E3
:10BFF0000F900F900F900F900F9020E030E0A9016C
:10C00000C301B2010E944DF2181624F077FA709421
:10C0100077F87094F70101900020E9F731976F01EC
:10C02000CE18DF088EE28083A2E0B0E0AC0FBD1F27
:10C03000AC0DBD1DBA8BA98BB10137FE03C0719544
:10C0400061957109072E000C880B990B0E944CEF2B
:10C050009B01AC01C301B2010E9438F120E030E045
:10C0600040E251E40E94ABEF0E9417F2605DE98963
:10C07000FA896083FE01EC0DFD1D1382D501ED915F
:10C08000FC910288F389E02D9801A701B401C50154
:10C09000199562960FB6F894DEBF0FBECDBFDF9143
:10C0A000CF911F910F91FF90EF90DF90CF90BF90B5
:10C0B000AF909F908F907F906F905F904F903F9048
:10C0C0002F900895CF92DF92EF92FF920F931F93DC
:10C0D000CF93DF93CDB7DEB760970FB6F894DEBF8E
:10C0E0000FBECDBF7C016B01CA01B9012AE0AE01D0
:10C0F0004F5F5F4F0E94F4E9D701ED91FC910288F8
:10C10000F389E02D9801AE014F5F5F4FB601C70183
:10C11000199560960FB6F894DEBF0FBECDBFDF91C4
:10C12000CF911F910F91FF90EF90DF90CF900895E6
:10C13000CF93DF93EC01DB01898182958F7086308C
:10C14000E1F128F481508230C8F080E014C08730DB
:10C1500009F18A508230C8F72FEF30E00E9431F1A8
:10C1600024E630E040E050E00E94B1F02C833D83B3
:10C170004E835F8381E0DF91CF9108952FEF30E010
:10C180000E9431F124E630E040E050E00E94B1F03E
:10C190002C83F0CF2FEF30E00E9431F124E630E025
:10C1A00040E050E00E94B1F0CA01B9010E944CEF9A
:10C1B0006C837D838E839F83DDCF2CE933E60E94E1
:10C1C00031F124E630E040E050E00E94B1F02C83F1
:10C1D0003D834E835F83B9CFDC011196EC911197BB
:10C1E000E295EF70E150EB3008F039C0F0E08827BD
:10C1F000E350FF498F4F0C941AF1206120612F61A9
:10C20000086108611161286128612861086108617D
:10C2100014966D917D918D919C9117970E944CEF92
:10C22000089514966D917D918D919C91179724E6B8
:10C2300030E040E050E00E94B1F0CA01B901EECF19
:10C2400014966C9170E090E080E00E944AEF0895AF
:10C2500014966D917D918D919C911797089560E052
:10C2600070E0CB010895DC011196EC911197E295F5
:10C27000EF70E150EB3008F037C0F0E08827EC5B5E
:10C28000FE498F4F0C941AF15661566174614F61EB
:10C290004F6165615C615C615C614F614F611496E7
:10C2A0006D917D918D919C911797089514966C9145
:10C2B00070E090E080E0089514966D917D918D91ED
:10C2C0009C9117970E9417F2089514966D917D9195
:10C2D0008D919C91179724E630E040E050E00E9459
:10C2E000B1F0CA01B901089560E070E0CB01089592
:10C2F000CF92DF92EF92FF920F931F93CF93DF9332
:10C3000000D000D01F921F92CDB7DEB709831A83E9
:10C310002B833C834D835E836F837887FC01208170
:10C3200031812115310589F490E080E028960FB61F
:10C33000F894DEBF0FBECDBFDF91CF911F910F915B
:10C34000FF90EF90DF90CF9008958C01C9010E947B
:10C35000B2AEE82EF12CF6E0EF16F10494F40E9450
:10C360006EA0009721F0FC012085207F2087BC0172
:10C37000F801808191810E9422B2FFEFEF1AFF0A3B
:10C38000EACF65E0F801808191810E949BAE8C012B
:10C39000892B51F28981803138F6CE0101960E94B5
:10C3A0003361161617061806190624F4F80180855D
:10C3B0008D7089F0F80180858F7080876FEC76E151
:10C3C00083EF9DE00E94CC9983EF9DE00E94369818
:10C3D00081E090E0ABCF0E9433BC6B017C01CE01C9
:10C3E00001960E943361C60ED71EE81EF91EF801A1
:10C3F000C186D286E386F48689818295807F8260B9
:10C40000808764EC76E183EF9DE00E94CC99CE01B9
:10C4100001960E943361AB01BC012AE030E083EF5A
:10C420009DE00E94DC986EEB76E183EF9DE00E9438
:10C43000CC99F80141855285638574852AE030E006
:10C4400083EF9DE00E94DC98BFCFEF92FF920F93A5
:10C450001F93CF93DF93CDB7DEB7C056D1090FB688
:10C46000F894DEBF0FBECDBF7C016A960FAF6A970E
:10C470006B961FAF6B976C962FAF6C976D963FAF17
:10C480006D976E964FAF6E976F965FAF6F97A09652
:10C490006FAFA097A1967FAFA19798E0FE01E75AF2
:10C4A000FF4FDE01AF5ABF4F01900D929A95E1F711
:10C4B0006A96EFAD6A97E150ED3008F07DC0F0E08C
:10C4C0008827EA59FD498F4F0C941AF1CC62CE624D
:10C4D000DA62DC62D8627362CA62DC62DC62D062F9
:10C4E000D262D662D46267E0CE018F5A9F4F0E941B
:10C4F0005B336AEA76E183EF9DE00E94CC994AE0E3
:10C5000050E062966FAD629783EF9DE00E943A988B
:10C510006FE976E183EF9DE00E94CC99CE018F5ABE
:10C520009F4F0E943361AB01BC012AE030E083EFF2
:10C530009DE00E94DC9883EF9DE00E943698629611
:10C540000FAD629763961FAD639764962FAD6497A6
:10C5500065963FAD659766964FAD669767965FADFA
:10C56000679768966FAD689769967FAD6997C701C1
:10C570000E94786181E090E0C05ADF4F0FB6F894D6
:10C58000DEBF0FBECDBFDF91CF911F910F91FF9006
:10C59000EF90089566E0A8CF62E0A6CF61E0A4CF57
:10C5A0006BE0A2CF6AE0A0CF6CE09ECF6DE09CCFA5
:10C5B00063E09ACF65E098CF90E080E0DDCFFC01AA
:10C5C000A7812A2F2E7FD1F0818182958F70815093
:10C5D0008330A0F4A695A150BB0B2BE531E00E945F
:10C5E00031F124E630E040E050E00E94B1F0DA01A1
:10C5F000C90187569F4FAF4FBF4F08958FEF9FEFF1
:10C600000895CF93DF93EC016115710539F48F81A3
:10C6100081708F8381E0DF91CF9108958981982F78
:10C6200092959F7029F180E09430A8F79B01770FD5
:10C63000440B550B2959310941095109A4E6B0E0D1
:10C640000E94D0F02BE531E040E050E00E94B1F0D4
:10C6500037FF02C030E020E02536310514F024E633
:10C6600030E02F5F220F8F818170282B2F83D2CF54
:10C670008F7080628983DACF2F923F924F925F92C0
:10C680006F927F928F929F92AF92BF92CF92DF92E2
:10C69000EF92FF920F931F93CF93DF93CDB7DEB747
:10C6A00068970FB6F894DEBF0FBECDBF1C01098797
:10C6B0001A872B873C874D875E876F87788B22E1AF
:10C6C000E216F10408F035C0F701E055FC4F308167
:10C6D000398BCE0109960E94DF6297FD04C0BC0130
:10C6E000C1010E9401639A85892F8F70D101119633
:10C6F000EC911197E07FE82B1196EC9311978985C7
:10C700008C93E295EF70EC3008F063C0F0E088277E
:10C71000E357FC498F4F0C941AF19A65B663B663E0
:10C7200038659B63C6650165426542654265016582
:10C730000165198ACECFB12C92959F709D3008F07B
:10C74000C9C4E92FF0E08827E755FC498F4F0C94C6
:10C750001AF1E963006620660066C965C96500666E
:10C7600000666A686A6800660066CD6492959F708C
:10C770009D3008F022C1E92FF0E08827ED53FC49F5
:10C780008F4F0C941AF1E963A16495645764D363E5
:10C79000D0637864A564DD64DD6462646264CD6442
:10C7A0008889F10187838F85D10116968C9316971E
:10C7B0008E8515968C9315978D8514968C9314976A
:10C7C0009295907F11968C9111978F70982B11965E
:10C7D0009C93B989BB2309F467C0F10181818295DB
:10C7E0008F702B2F30E08217130609F45DC066E4CA
:10C7F0007AE183EF9DE00E94CC99D10111966C9172
:10C8000062956F704AE050E083EF9DE00E943A9895
:10C8100063E47AE183EF9DE00E94CC994AE050E026
:10C82000698983EF9DE00E943A9861E47AE183EFA1
:10C830009DE00E94CC99F101008119821A821B822D
:10C840001C821D821E821F82188689898295807FA4
:10C850009A819F70892B8A830983EE24EA94FE2CA7
:10C860001181228133814481558166817781CE0196
:10C8700001960E943C63D1012C9311963C93119731
:10C8800012964C93129713965C93139714966C938D
:10C89000149715967C93159716968C931697179662
:10C8A0009C93C1010E94A43188E0F10182C18F856F
:10C8B0009889F1018683878190FB80F987838E8533
:10C8C000858387CF8D859E85AF85B8898F3F9105FC
:10C8D000A105B10529F024F08FEF90E0A0E0B0E0D1
:10C8E000B7FF03C080E090E0DC01F101848371CFE9
:10C8F0006D857E858F85988924E630E040E050E0A4
:10C900000E94B1F02F3F31054105510529F024F077
:10C910002FEF30E040E050E057FF03C020E030E070
:10C92000A901D10114962C9354CF8F859889F101D8
:10C930008683878190FB80F987838E8585838D85AB
:10C94000D5CF8D8514968C9344CFCD84DE84EF842F
:10C95000F88820E030E0A901C701B6010E9445EF48
:10C9600087FD17C020E030E04FE753E4C701B60170
:10C970000E944DF2181634F4C12CD12CAFE7EA2EE8
:10C98000A3E4FA2EC701B6010E941EF2F1016483EE
:10C9900020CFC12CD12C7601F5CFD10111968C91ED
:10C9A00011978F70806C11968C9311978D859E8551
:10C9B00015969C938E9314970CCF66EC7AE183EFD7
:10C9C0009DE00E94CC996A8562956F704AE050E0C4
:10C9D00083EF9DE00E943A9863EC7AE183EF9DE05B
:10C9E0000E94CC99F101618162956F704AE050E03C
:10C9F00083EF9DE00E943A9883EF9DE00E94369875
:10CA0000E8CE92959F70933091F09C3031F24D8535
:10CA10005E856F857889F1014483558366837783CA
:10CA20009295907F81818F70982B9183D2CE60E018
:10CA3000C1010E94B233D10114968C9314978F8553
:10CA4000988916968C93169717968C91179790FB4A
:10CA500080F917968C9317978E8515968C9315975A
:10CA600011968C9111978F70806211968C93B1CE34
:10CA700060E0CE0109960E94B233D10114968C93E6
:10CA80001497EECF92959F709D3008F066C0E92F05
:10CA9000F0E08827E15BFA498F4F0C941AF1E963C3
:10CAA0006A6599651765996599655C6589658965A4
:10CAB000896578658465CD648D859E85AF85B889E7
:10CAC000F10184839583A683B78381818F7080660B
:10CAD00081837FCE6D8570E090E080E00E944AEF18
:10CAE000D10114966D937D938D939C93179771CE7E
:10CAF0006D857E858F8598890E944CEFF101648356
:10CB000075838683978365CE6D857E858F859889AD
:10CB1000E5CF9295907FF10181818F70982B918361
:10CB20008D859E85AF85B88984839583A683B783D9
:10CB300050CE9295907FD10111968C9111978F7064
:10CB4000982B11969C938D859E85AF85B889F101B0
:10CB500084839583A683B7833CCE61EB7AE183EF30
:10CB60009DE00E94CC996A8562956F704AE050E022
:10CB700083EF9DE00E943A986EEA7AE183EF9DE0B0
:10CB80000E94CC99D10111966C912ECFBB24B39405
:10CB9000D3CD4D855E856F857889F10144835583BA
:10CBA000668377839295907F81818F70982B918394
:10CBB00088E0DE01119601900D928A95E1F72981B6
:10CBC0003A814B815C816D817E818F8198856896E9
:10CBD0000FB6F894DEBF0FBECDBFDF91CF911F918E
:10CBE0000F91FF90EF90DF90CF90BF90AF909F900C
:10CBF0008F907F906F905F904F903F902F9008950F
:10CC0000963009F43AC148F46D85913071F06FEFB8
:10CC100070E0933051F060E008C0973009F439C1FA
:10CC20009A506D857E859230B0F784E68F8788892B
:10CC30008E7F888B1E868A858F7080628A876D873B
:10CC40002E8530E0AFEFB0E00E94E3F024E630E064
:10CC500040E050E00E94B1F069017A01FFEFCF1689
:10CC6000D104E104F10429F024F0C12CD12C760187
:10CC7000CA9486012D852A8B622E712CBB2009F463
:10CC800071C088898695A82FA150BB0B2D01BFEFDD
:10CC90004B165B0609F01EC1003811050CF000C1EF
:10CCA0008FE790E08C199D09869DD001879DB00D7E
:10CCB000969DB00D11242FEF30E00E9431F121E854
:10CCC0003EE740E050E00E94B1F0F1012783ABE97C
:10CCD000B0E0A70196010E94D0F0EFE78E2E912CD4
:10CCE000A12CB12CA50194010E94B1F089019A01F7
:10CCF0000C591F4F2F4F3F4FAEEFB1E0A7019601E8
:10CD00000E94D0F0A50194010E94B1F0D3010E94CD
:10CD1000D0F02FEF30E040E050E00E94B1F0390158
:10CD20002FEF6216710421F01CF066246A94712CB6
:10CD300061EA7AE183EF9DE00E94CC99B80183EF2C
:10CD40009DE00E94AAAE63E97AE183EF9DE00E9434
:10CD5000CC99B30183EF9DE00E94AAAE83EF9DE0E2
:10CD60000E943698E8E7FEE1E491F0E0EE0FFF1F45
:10CD7000E25AF14E85919491EEECFEE1E4912F851B
:10CD800038893170AFEFBFEF0E94E3F02DE631E05C
:10CD900040E050E00E94B1F044275527AAEFB5E0EB
:10CDA0000E94D0F0DC01CB019058AF4FBF4FCD01B6
:10CDB000BB2797FDB095AB2F8E3FE1E09E0708F0B3
:10CDC00062C1382F8F3F910508F47FC14EEF481B99
:10CDD00050E03FEFF301319678012FEFE21AF20AAB
:10CDE000009510E03E9DC0013F9D900D1124292F1C
:10CDF0003327200F311FDF010E9431F14B015C010D
:10CE00008824AA24BB245E9D90015F9D300D1124CF
:10CE1000232F3327200F311F0E9431F1BB27A92F69
:10CE2000982F872F882A992AAA2A4E9D90014F9DD4
:10CE3000300D1124232F3327200F311FDF010E94D3
:10CE400031F1B82FA72F962F882788279927BB273E
:10CE500088299929AA29F101A6839583848367E605
:10CE60007AE183EF9DE00E94CC99C1010E94A43138
:10CE700060E080E00E94A9BAACCC6D857E858F858C
:10CE8000988924E630E040E050E00E94B1F0B9011A
:10CE9000CCCE6D857E858F8598890E9417F2C5CE90
:10CEA000A70196012058310941095109ABE9B0E0C9
:10CEB0000E94D0F02FE730E040E050E00E94B1F057
:10CEC00089019A010C591F4F2F4F3F4FD1011796DF
:10CED0001C922ECF9201AAEBBFEF0E9429F144E6EB
:10CEE000842E912CA12CB12CA50194010E94B1F0AB
:10CEF000DA01C9018C599F4FAF4FBF4F8B8B9C8B71
:10CF0000AD8BBE8B26E430E0D2010E9431F1A50149
:10CF100094010E94B1F049015A019EE1890E911CD1
:10CF2000A11CB11C003811050CF093C08FE790E0F4
:10CF30008C199D09869DD001879DB00D969DB00DE1
:10CF40001124A50194010E94DBF09B01AC01AFEF1D
:10CF5000B0E00E94D0F024E63AE640E050E00E94C3
:10CF6000B1F0D10117962C932B893C894D895E89AC
:10CF70002C0D3D1D4E1D5F1DAEEFB1E00E94D0F0A7
:10CF800023EE30E040E050E00E94B1F029013A0188
:10CF9000388F2F8BAFEFB0E0A70196010E94D0F041
:10CFA0002FE730E040E050E00E94B1F08901EA89CB
:10CFB000AE2FB0E0A30192010E94D0F02FEF30E03D
:10CFC00040E050E00E94B1F039012F3F310521F0DF
:10CFD0001CF066246A94712C6DE87AE183EF9DE081
:10CFE0000E94CC992AE030E04B895C896D897E896A
:10CFF00083EF9DE00E94DC9867E87AE183EF9DE093
:10D000000E94CC992AE030E0B501A40183EF9DE0B5
:10D010000E94DC986FE77AE183EF9DE00E94CC9953
:10D02000B80183EF9DE00E94AAAE67E77AE183EF43
:10D030009DE00E94CC99B30183EF9DE00E94AAAECF
:10D040006EE67AE183EF9DE00E94CC996F89788D3E
:10D0500081CEA70196012058310941095109ABE958
:10D06000B0E00E94D0F02FE730E040E050E00E94B6
:10D07000B1F089019A010C591F4F2F4F3F4FD10139
:10D0800017961C92A9CF8C3FF3E09F0768F48D3F61
:10D0900022E0920728F452E0580F3FEF40E09ACE8A
:10D0A0003CEF381B5FEFFACF8A3F35E0930781F002
:10D0B0008B3FE4E09E0728F444E0480F5FEF30E048
:10D0C00089CE5AEF581B30E001C050E04FEF82CEBE
:10D0D00050E0F9CF65E57AE183EF9DE00E94CC99BD
:10D0E0006A8562956F704AE050E083EF9DE00E9490
:10D0F0003A9862E57AE142CDFC019181892F8295CF
:10D100008F7021F0823029F080E008959F70906246
:10D1100091839B0177FF02C030E020E02E3681E052
:10D12000380714F02DE631E02683878130FB80F943
:10D13000878381E008950F931F93CF93DF938C0132
:10D14000FC01C081D1816FE270E0CE010E94B8F590
:10D150000097D9F0FC011192CF010E945A5CEC01BA
:10D1600063E976E183EF9DE00E94CC99BE0183EFF5
:10D170009DE00E94AAAE83EF9DE00E943698CE010A
:10D18000DF91CF911F910F910895CE010E945A5CBB
:10D19000EC01892BA1F3F80111821082F0CFDC01A0
:10D1A000ED91FC91309729F090859F7081E095304A
:10D1B00009F080E00895EF92FF920F931F93CF93B1
:10D1C000DF93EC017B018E819F81892BD9F48881CB
:10D1D00099810E94B2AE082F10E00530110594F439
:10D1E0000E946EA0009721F0FC012085207F2087FF
:10D1F0009F838E83BC01888199810E9422B20F5F38
:10D200001F4FEBCFEE81FF813097D9F08085982FAB
:10D210009F70A9F4807F82608087EE81FF811186F4
:10D22000128613861486EE81FF81F782E682C7019B
:10D23000DF91CF911F910F91FF90EF900895923061
:10D2400061F3F12CE12CF3CFCF92DF92EF92FF92BA
:10D250000F931F93CF93DF93EC016A017B018E81C3
:10D260009F81892BD9F4888199810E94B2AE082FC1
:10D2700010E00530110594F40E946EA0009721F093
:10D28000FC012085207F20879F838E83BC018881BD
:10D2900099810E9422B20F5F1F4FEBCFEE81FF8179
:10D2A000309749F18085982F9F7019F5807F8260B3
:10D2B0008087EE81FF81C186D286E386F48667E8A7
:10D2C00076E183EF9DE00E94CC992AE030E0B7013F
:10D2D000A60183EF9DE00E94DC9883EF9DE0DF9143
:10D2E000CF911F910F91FF90EF90DF90CF900C9412
:10D2F00036989230F1F2DF91CF911F910F91FF900C
:10D30000EF90DF90CF900895FC0186819781009780
:10D3100099F0FC0120852F70223029F461857285F7
:10D32000838594850895253039F460E00E949BAE92
:10D33000009711F0FC01F2CF60E070E0CB0108959E
:10D34000FC01A481B581109721F118969C91189742
:10D350009F708EEF890F823010F091111AC01996CC
:10D360004D935D936D937C931C97A481B581189622
:10D370009C911897907F926018969C930480F581F9
:10D38000E02D8085982F907F903619F48F70806AF9
:10D39000808708950F931F93CF93DF93FC01C28181
:10D3A000D3812097F9F088858F70823049F4672BFC
:10D3B000C9F489859A85DF91CF911F910F910895C6
:10D3C000853081F48B01CE010E94B2AE8017110628
:10D3D00049F044F0602FCE010E949BAEFC01818594
:10D3E0009285E9CF90E080E0E6CFCF92DF92EF9296
:10D3F000FF920F931F93CF93DF93EC018881998164
:10D400000E94B2AE082F10E0043011059CF40E9477
:10D410006EA0009739F0DC0118962C911897207FA8
:10D4200018962C93BC01888199810E9422B20F5FCB
:10D430001F4FEACFC880D98060E0C6010E949BAE32
:10D44000FC011185188761E0C6010E949BAE7C013A
:10D450009B838A8362E0C6010E949BAE9D838C837E
:10D4600064E0C6010E949BAE6C019F838E831031E5
:10D4700009F497C070F4133071F11A3009F45BC0ED
:10D48000DF91CF911F910F91FF90EF90DF90CF90A0
:10D490000895123109F4FDC0133191F786E090E050
:10D4A0000E9417E7FC01D383C2838BEB92E0918348
:10D4B0008083C114D10409F407C1D60118968C9158
:10D4C00018978F70823009F0FFC016968D919C914D
:10D4D00095838483F6C08AE090E00E9417E78C0170
:10D4E000DC011396DC93CE9312978FED92E08D932F
:10D4F0009C9370E060E0CE010E94CA6997FD12C063
:10D50000F80195838483CE010E942C5CF8019783F7
:10D51000868385E093E091838083118610861A8745
:10D520000987AECF919581959109D80115969C9365
:10D530008E931497E8CF87E090E00E9417E78C0164
:10D54000DC011396DC93CE93129783E793E0119658
:10D550009C938E9387E79AE016969C938E931597EB
:10D56000CE010E942C5C892BD1F270E060E0CE01EC
:10D570000E94CA69F8018483813071F028F08230FA
:10D5800071F684E19BE002C08EE49CE0D80116961F
:10D590009C938E931597C3CF81EB9BE096838583F5
:10D5A000BECF8BE090E00E9417E78C01FC01D38393
:10D5B000C2838FE493E091838083168270E060E001
:10D5C000CE010E94CA6997FD46C0D80115969C936A
:10D5D0008E931497D80114968D919C91009719F011
:10D5E000863591052CF080E290E0F80195838483E4
:10D5F000E114F10409F43FC0D70118968C918F70A3
:10D600008530C9F5C7010E94B2AE8230A0F161E059
:10D61000C7010E949BAEFC01892B69F180858F7048
:10D62000823011F561857285838594850E944CEF67
:10D6300020E030E04AE754E40E94ABEF0E941EF283
:10D640006115710581059105D1F0F8016783708737
:10D650008187928764CF919581959109F80195838F
:10D66000848381E08683B6CF833029F46185728517
:10D6700083859485DDCF60E070E0CB01D9CF88E869
:10D6800093E1A0E0B0E0F80187839087A187B2879B
:10D6900046CF86E090E00E9417E7FC01D383C28367
:10D6A0008BE293E09183808315821482E114F1046C
:10D6B00041F0D70118968C918F70863011F4F58265
:10D6C000E482FA87E987DCCE90E080E001CFCF9258
:10D6D000DF92EF92FF926A017B0163E0FC0180819F
:10D6E00091810E949BAEFC01892BA9F080858D70F1
:10D6F00091F4C094D094E094F094CC24CA948185A1
:10D700009285A385B4858C219D21AE21BF2181877F
:10D710009287A387B487FF90EF90DF90CF90089512
:10D72000CF92DF92EF92FF926A017B0163E0FC01EE
:10D73000808191810E949BAEFC01892BA9F090858C
:10D74000892F8D7089F4907F92609087CC24FF247C
:10D7500041855285638574854C295D296E297F2911
:10D760004187528763877487FF90EF90DF90CF9057
:10D770000895CF92DF92EF92FF926A017B0163E0FE
:10D78000FC01808191810E949BAE009791F0FC0189
:10D7900020852F70223069F4618572858385948598
:10D7A0006C217D218E219F21FF90EF90DF90CF9003
:10D7B000089560E070E0CB01F7CFAF92BF92CF92B7
:10D7C000DF92EF92FF920F931F93CF93DF93CDB72A
:10D7D000DEB7CD56D1090FB6F894DEBF0FBECDBF70
:10D7E0005C01A7960FAFA797A8961FAFA897A99619
:10D7F0002FAFA997AA963FAFAA97AB964FAFAB971B
:10D80000AC965FAFAC97AD966FAFAD97AE967FAF6E
:10D81000AE9723961FAE1EAE2397FE01ED5BFF4F22
:10D8200082E1DF011D928A95E9F7729611921192B9
:10D8300087E0DF011D928A95E9F7CE018A599F4F53
:10D840000E94A431F0FE2CC0A796EFADA797E83157
:10D8500008F050C1F0E08827EF5CF3498F4F0C943B
:10D860001AF1806D496C776D7A6D7A6D776D496CC0
:10D870007A6D7A6D7A6D7A6D7A6D7A6D7A6D496CA2
:10D88000496C7A6D7A6D7A6D496C496C496C7A6D28
:10D89000806D6EE37AE1CE018B5A9F4F0E9459E969
:10D8A0000E9441AE882309F407C18091A807811125
:10D8B00003C1C114D10409F05EC030E020E043E0B0
:10D8C00050E060E4CE0101960E941828D501ED9148
:10D8D000FC91608171814FE350E0CE0101960E947E
:10D8E0008BF5F1FE10C1A7968FADA797823009F492
:10D8F0000AC1853009F407C1A8968FADA897829513
:10D900008F709FE0980F9F70923018F0883009F068
:10D91000FAC001E020E032E044E150E0BE016F5B7C
:10D920007F4FCE018A599F4F0E94832FBE016F5BAC
:10D930007F4FCE0101960E9401BD66E27AE183EF3E
:10D940009DE00E94CC99BE016F5F7F4F83EF9DE009
:10D950000E94669963E27AE183EF9DE00E94CC9990
:10D96000BE016F5B7F4F83EF9DE00E94669983EF5E
:10D970009DE00E943698A8968FADA897807F87017A
:10D9800000271072882311F0F1FC04C00115110565
:10D9900009F4F5C030E020E043E050E060E4CE015F
:10D9A00001960E941828D501ED91FC91608171814A
:10D9B0004FE350E0CE0101960E948BF5C114D104D3
:10D9C00069F06FE175E0CE0101960E9465F54FE3C5
:10D9D00050E0B601CE0101960E948BF56FE175E033
:10D9E000CE0101960E9465F54FE350E066E17AE1D1
:10D9F0000115110511F462E17AE1CE0101960E9450
:10DA000069E9A8968FADA89782958F70845082306F
:10DA100008F09FC067E1CE018A599F4F0E945B3397
:10DA20006F962FAF6F97A0963FAFA097A1964FAF7D
:10DA3000A197A2965FAFA297A3966FAFA397A49664
:10DA40007FAFA497A5968FAFA597A6969FAFA697F1
:10DA500000E020E033E044E150E0BE016F5B7F4F27
:10DA6000CE018A599F4F0E94832F6CE07AE183EFA9
:10DA70009DE00E94CC99BE016F5F7F4F83EF9DE0D8
:10DA80000E94669969E07AE183EF9DE00E94CC995B
:10DA9000BE016F5B7F4F83EF9DE00E94669983EF2D
:10DAA0009DE00E9436980E9441AE882329F0809123
:10DAB000A807882309F455C0A701FF0C660B770B54
:10DAC000C5010E94906B90E080E0C359DF4F0FB614
:10DAD000F894DEBF0FBECDBFDF91CF911F910F91A4
:10DAE000FF90EF90DF90CF90BF90AF9008956AE3E2
:10DAF0007AE1D1CE6CE27AE183EF9DE00E94CC998D
:10DB0000E894F0F8CDCEF0FE36CF66968FAD6697EE
:10DB1000882309F430CFBE016B5A7F4FCE010196A6
:10DB20000E9401BD6DE17AE183EF9DE00E94CC99F6
:10DB3000BE016F5F7F4F83EF9DE00E9466996AE1AF
:10DB40007AE183EF9DE00E94CC99BE016B5A7F4F32
:10DB50000ACF20E032E0012B11F020E033E000E0BA
:10DB60007ACFBE016F5B7F4FCE0101960E9401BD4F
:10DB700040E052E060E070E0C5010E94676BF0FE9B
:10DB800090C0A796EFADA797E150E53118F5F0E00A
:10DB90008827E253F2498F4F0C941AF1D96EEA6D3F
:10DBA000EA6DEA6DEA6DD96EEA6DEA6DEA6DEA6DCD
:10DBB000EA6DEA6DEA6DDE6ED66EEA6DEA6DEA6DCB
:10DBC000E36DD06ED36E6FEF79E1CE018B5A9F4F2C
:10DBD0000E9459E930E020E043E050E060E4CE01EB
:10DBE00001960E941828D501ED91FC916081718108
:10DBF0004FE350E0CE0101960E948BF5C114D10491
:10DC000069F06FE175E0CE0101960E9465F54FE382
:10DC100050E0B601CE0101960E948BF56FE175E0F0
:10DC2000CE0101960E9465F54FE350E069EE79E17F
:10DC3000CE0101960E9469E963EE79E183EF9DE0F0
:10DC40000E94CC99BE016F5F7F4F83EF9DE00E94E1
:10DC5000669960EE79E183EF9DE00E94CC99BE0168
:10DC60006B5A7F4F83EF9DE00E94669983EF9DE0A2
:10DC70000E9436980E9441AE882309F41DCF8091FE
:10DC8000A807811119CFBE016B5A7F4FCE010196B3
:10DC90000E9401BD40E051E060E070E0C5010E94DB
:10DCA000676BF2FE7AC040E050E061E070E0C501D1
:10DCB0000E94B96B672B682B692B09F482C068ED51
:10DCC00079E1CE018B5A9F4F0E9459E930E020E064
:10DCD00043E050E060E4CE0101960E941828D5018F
:10DCE000ED91FC91608171814FE350E0CE0101968E
:10DCF0000E948BF5C114D10469F06FE175E0CE018B
:10DD000001960E9465F54FE350E0B601CE01019601
:10DD10000E948BF56FE175E0CE0101960E9465F5DA
:10DD20004FE350E065EC79E1CE0101960E9469E98C
:10DD30006FEB79E183EF9DE00E94CC99BE016F5FAC
:10DD40007F4F83EF9DE00E9466996CEB79E183EF52
:10DD50009DE00E94CC99BE016B5A7F4F83EF9DE0FE
:10DD60000E94669983EF9DE00E9436980E9441AE22
:10DD7000882309F4A1CE8091A80781119DCEBE0110
:10DD80006B5A7F4FCE0101960E9401BD40E054E0E6
:10DD900060E070E0C5010E94676B81E090E095CE85
:10DDA0006AEF79E112CF66EF79E10FCF6DEE79E19D
:10DDB0000CCFF5018085853009F00CCF64E07AE165
:10DDC00004CF40E050E062E070E0C5010E94B96B12
:10DDD000672B682B692B19F061ED79E172CF6AEC42
:10DDE00079E16FCFAF92BF92CF92DF92EF92FF9225
:10DDF0000F931F93CF93DF9300D000D01F921F92F9
:10DE0000CDB7DEB75C017B0160FF03C0E894E0F8AA
:10DE1000F4F8F4FC0DC00E943F29663971058105B4
:10DE2000910530F08091C3099091C409059719F5C7
:10DE3000A70144275770052E000C660B770BC50110
:10DE40000E94906B6BEA79E183EF9DE00E94CC9990
:10DE50008FEF9FEF28960FB6F894DEBF0FBECDBFB1
:10DE6000DF91CF911F910F91FF90EF90DF90CF90B6
:10DE7000BF90AF90089519821A821B821C821D8266
:10DE80001E821F8218868A818F708A8340E053E049
:10DE9000B501CE0101960E94A43240E057E060E057
:10DEA00070E0C5010E94B96BE62AF72AD12CC12C7B
:10DEB00009811A812B813C814D815E816F8178853A
:10DEC000C5010E94DD6BC6CF4F925F926F927F9229
:10DED000AF92BF92CF92EF92FF920F931F93CF9387
:10DEE000DF9300D000D01F921F92CDB7DEB75C0148
:10DEF00009831A832B833C834D835E836F837887EA
:10DF000062E076E183EF9DE00E94CC99CE0101961C
:10DF10000E94A4318981811134C00A810F700130BF
:10DF2000A9F160F1023021F010E0053009F041C0A4
:10DF3000D501ED91FC9100A0F1A1E02D09811A819C
:10DF40002B813C814D815E816F817885C50119955A
:10DF500081E090E028960FB6F894DEBF0FBECDBFEB
:10DF6000DF91CF911F910F91FF90EF90CF90BF90D5
:10DF7000AF907F906F905F904F900895CC24C394A2
:10DF8000D7CF813061F1823009F4BCC065EF75E113
:10DF900083EF9DE00E94CC994AE050E0698183EFD5
:10DFA0009DE00E943A9883EF9DE00E94369801E040
:10DFB00010E065EE75E183EF9DE00E94CC99B80119
:10DFC00083EF9DE00E94AAAE83EF9DE00E94369809
:10DFD000CE0101960E94A43190E080E0BBCF8A81FF
:10DFE00082958F70863009F474C0D8F481508230E5
:10DFF000E0F16EE170E0CE0101960E949860F501BB
:10E000006281738140E052E0CE0101960E94F231BC
:10E0100060E072E1D50112968D919C910E94F26EA2
:10E020001BC0873079F18A50823018F78D819E812C
:10E03000AF81B88585369105A105B10524F084E648
:10E0400090E0A0E0B0E0B7FF03C080E090E0DC012A
:10E050009C01243131056CF2D501ED91FC9100A0B9
:10E06000F1A1E02DCC24C39469CF2D8130E0A4E64A
:10E07000B0E00E94E3F02FEF30E040E050E00E947B
:10E08000B1F0E7CF4D805E806F80788420E030E093
:10E09000A901C301B2010E9445EF87FD11C020E034
:10E0A00030E048EC52E4C301B2010E944DF2181670
:10E0B00054F4412C512C88EC682E82E4782E03C055
:10E0C000412C512C3201C301B2010E9417F29B0175
:10E0D000C0CF6D817E818F81988524E630E040E05D
:10E0E00050E00E94B1F0253631054105510524F07C
:10E0F00024E630E040E050E057FFABCF20E030E0D6
:10E10000A901A7CF1D821E821F821886D501ED911D
:10E11000FC9100A0F1A1E02DCC24C39402E01A816F
:10E120002B813C8140E00FCFCF93C62F63E0FC01F1
:10E13000808191810E949BAEFC01892B21F1908509
:10E14000892F8D7001F5907F9260908781859285EF
:10E15000A385B4858827BB278C2B81879287A387CB
:10E16000B4876FE776E183EF9DE00E94CC994AE0A7
:10E1700050E06C2F83EF9DE00E943A9883EF9DE082
:10E18000CF910C943698CF91089563E0FC01808183
:10E1900091810E949BAE009719F0FC018185089542
:10E1A0008FEF089581E090E008950F931F93CF9330
:10E1B000DF9300D000D01F921F92CDB7DEB7198237
:10E1C0001A821B821C821D821E821F8218862A814F
:10E1D0002F702A83FC0102811381C8010E94C5703F
:10E1E000813041F020F0823011F0853081F490E0F0
:10E1F00080E002C081E090E028960FB6F894DEBF80
:10E200000FBECDBFDF91CF911F910F91089540E0D8
:10E2100052E0B801CE0101960E94A43260E0CE0126
:10E2200001960E94B233E8CF8F929F92AF92BF9235
:10E23000CF92DF92EF92FF920F931F93CF93DF93D2
:10E24000CDB7DEB767970FB6F894DEBF0FBECDBF70
:10E250008C017B014C018BE0880E911C9F8A8E8A79
:10E26000F801128611861386148E138E672B09F41B
:10E2700063C0A090C509B090C609A114B10409F407
:10E280005BC06FE270E0C7010E9470F56C01892BE2
:10E2900009F44AC0F701DE01119690E080E0BD016B
:10E2A0002191222341F02F3231F08431910519F070
:10E2B0002D930196F5CF860F971FFC011082C501A3
:10E2C0000E9423AEF80191838083B6016F5F7F4F78
:10E2D0004FE050E0C4010E94A9F5CE0146960E948D
:10E2E0009B68F801948F838F8E899F89892B09F40D
:10E2F0001386C8010E94CF68882319F0C8010E94C4
:10E30000F56967960FB6F894DEBF0FBECDBFDF91FB
:10E31000CF911F910F91FF90EF90DF90CF90BF9022
:10E32000AF909F908F900895B701C5010E9423AED2
:10E33000F80191838083DDCFF80111821082D9CF5B
:10E34000DC0119968D919C91009739F0DC01ED91DB
:10E35000FC910280F381E02D19940895CF93DF930F
:10E36000EC01798368831A8619861B861C8E1B8EA6
:10E370000E94CF68882329F0CE01DF91CF910C94C1
:10E38000F569DF91CF9108954F925F926F927F92DE
:10E390008F929F92AF92BF92CF92EF92FF920F9384
:10E3A0001F93CF93DF93CDB7DEB76D970FB6F89479
:10E3B000DEBF0FBECDBF009709F4A4C0FC012085CD
:10E3C0002F70253009F09EC02A015B01868097805E
:10E3D0008091C1098F5F8093C1098114910409F470
:10E3E0008CC0F40180858F70843009F082C0618513
:10E3F00072858091C5099091C6090E9423AE3C01A7
:10E40000009709F476C0FC0180858F70853009F093
:10E4100070C0B301CE0101960E94AE71A114B10487
:10E42000A9F0CE0101960E94CF68882379F0C12C13
:10E430007201F5010081118122813381448155816E
:10E4400066817781CE0101960E94857360E0C301E9
:10E450000E949BAE0097D1F1FC0120852F702230E5
:10E46000A9F581859285A385B4850797A105B10596
:10E4700069F561E0C3010E949BAEA201B5010E9453
:10E48000C471A114B10489F5882379F18091C1097F
:10E4900081508093C109CE0101960E94A07181E054
:10E4A0006D960FB6F894DEBF0FBECDBFDF91CF9152
:10E4B0001F910F91FF90EF90CF90BF90AF909F90E2
:10E4C0008F907F906F905F904F900895A114B1044A
:10E4D00061F4CE0101960E94CF68882331F0CE010D
:10E4E00001960E948472892B89F6CE0101960E94C2
:10E4F000A071F4018280938070CF8091C109815016
:10E500008093C10980E0CCCFDF92EF92FF920F930E
:10E510001F93CF93DF9300D000D01F921F92CDB7EF
:10E52000DEB77C0119821A821B821C821D821E8228
:10E530001F8218868A818F708A83D701ED91FC91A2
:10E540006081718183EF9DE00E9466996CE579E1BD
:10E5500083EF9DE00E94CC99C7010E94CF68811192
:10E560001BC063E579E183EF9DE00E94CC9983EFC6
:10E570009DE00E9436980FEF1FEFC80128960FB656
:10E58000F894DEBF0FBECDBFDF91CF911F910F91E9
:10E59000FF90EF90DF900895C7010E94C570D82EBC
:10E5A000F70181859285009791F0DC01ED91FC9156
:10E5B0000688F789E02D19958C0197FD08C081E048
:10E5C0000115110509F480E00E940B5CD6CFF7011C
:10E5D0008085873009F42EC0EFEFED0DE43150F562
:10E5E000F0E08827E950FD488F4F0C941AF10B7327
:10E5F00014731A731A7314730B731A731A731A73CE
:10E600001A731A731A731A730B731A731A731A73B1
:10E610001A730B730B7364E379E183EF9DE00E943F
:10E62000CC9901E010E0A9CF80E00E940B5C10E0E3
:10E6300000E0A3CF40E052E0B701CE0101960E9476
:10E64000A432D70118968C911897873079F160F42D
:10E65000833009F454C0843061F064E479E183EFDD
:10E660009DE00E94CC99E3CF883009F448C08930FE
:10E67000A1F760E0CE0101960E94B2338C0169E3FC
:10E6800079E183EF9DE00E94CC99B80183EF9DE092
:10E690000E94AAAE83EF9DE00E94369891E080E050
:10E6A000012B09F490E0092F182F67CF1296ED91F6
:10E6B000FC9180858F7010E000E0853001F761E506
:10E6C00079E183EF9DE00E94CC9950E040E070E05A
:10E6D00060E0F701828193810E94C471F82E082FB7
:10E6E00010E06EE479E183EF9DE00E94CC998F2DDC
:10E6F0000E940B5C83EF9DE00E9436983ECFCE01D6
:10E7000001960E9433618B01BACF2F923F924F92B4
:10E710005F926F927F928F929F92AF92BF92CF92B1
:10E72000DF92EF92FF920F931F93CF93DF93CDB7BA
:10E73000DEB7C25CD1090FB6F894DEBF0FBECDBF05
:10E740001C01C755DF4F0883C95AD040C655DF4F5B
:10E750001883CA5AD040C555DF4F2883CB5AD040C2
:10E76000C455DF4F3883CC5AD040C355DF4F488360
:10E77000CD5AD040C255DF4F5883CE5AD040C155F4
:10E78000DF4F6883CF5AD040C055DF4F7883C05BDE
:10E79000D040CF54DF4FF982E882C15BD040CD54E6
:10E7A000DF4FC882C35BD0400E943F296B01C95430
:10E7B000DF4F79836883C75BD040683C7105A4F460
:10E7C0006BE179E189EE9DE00E94CC99B60189EE7A
:10E7D0009DE00E94AAAE89EE9DE00E943698CC246E
:10E7E000CA94DC2C0C94BA7D0E9433BCC154DF4F18
:10E7F000688379838A839B83CF5BD040C655DF4F84
:10E800008881CA5AD0408F70482E512C2091C3095C
:10E810003091C409C354DF4F39832883CD5BD04086
:10E82000CF54DF4FE881F981C15BD040309721F0B0
:10E83000808181110C940684D1011B968C918823D0
:10E8400041F0C1010B96CF54DF4F99838883C15BA0
:10E85000D0404114510411F00C944F84CF54DF4F39
:10E86000E881F981C15BD040309711F00C940A84A3
:10E87000F101438C548C4114510411F40C944F84D5
:10E88000C655DF4F8881CA5AD0408F7011F00C9462
:10E890004F84642DCE0187559F4F0E943433C75655
:10E8A000DF4F2883C959D040C656DF4F3883CA5935
:10E8B000D040C556DF4F4883CB59D040C456DF4FB8
:10E8C0005883CC59D040C356DF4F6883CD59D040D0
:10E8D000C256DF4F7883CE59D040C156DF4F888370
:10E8E000CF59D040C056DF4F9883C05AD0400C94C7
:10E8F0004F84D1018D919C91892B09F470CFB4E0A4
:10E900004B16510471F5C755DF4F0881C95AD040E5
:10E91000C655DF4F1881CA5AD040C555DF4F2881F0
:10E92000CB5AD040C455DF4F3881CC5AD040C35564
:10E93000DF4F4881CD5AD040C255DF4F5881CE5A63
:10E94000D040C155DF4F6881CF5AD040C055DF4F0E
:10E950007881C05BD040C1010E9478616C010C9449
:10E96000BA7DC755DF4F1881C95AD040143009F419
:10E97000AAC228F4112391F1B12CA12C61C288EF15
:10E98000810F8230C8F788E0FE01E755FF4FDE01B6
:10E99000119601900D928A95E1F7C655DF4FE881F7
:10E9A000CA5AD0408E2F807F09F401C3E295EF70E0
:10E9B000E150EB3008F0FBC2F0E08827ED51FB4856
:10E9C0008F4F0C941AF1C577C577D777B677B6779E
:10E9D0006178507850785078B677B67719821A8275
:10E9E0001B821C821D821E821F8218868A818F7064
:10E9F0008A83C655DF4F8881CA5AD040807F09F488
:10EA0000BBCF0AE04016510409F41CC20CF0F6C05A
:10EA10004114510409F416C122E04216510409F0D0
:10EA2000ABCFB12CA12C612C77247A94B101CE010B
:10EA300001960E947FB28A81982F92959F70945F71
:10EA40009F70923060F4C655DF4F9881CA5AD0400B
:10EA500092959F70923019F48F7080628A83D101F1
:10EA600018969C91973071F4C655DF4F8881CA5A29
:10EA7000D040807E803211F0803421F48A818F7002
:10EA800080628A83F101A185B285892F90E0109779
:10EA900041F0ED91FC911197048CF58DE02DCD01A5
:10EAA00019957C01C755DF4F0881C95AD040C6551A
:10EAB000DF4F1881CA5AD040C555DF4F2881CB5A45
:10EAC000D040C455DF4F3881CC5AD040C355DF4FBA
:10EAD0004881CD5AD040C255DF4F5881CE5AD040E0
:10EAE000C155DF4F6881CF5AD040C055DF4F788184
:10EAF000C05BD040CE0101960E943C63CF57DF4FF0
:10EB00002883C158D040CE57DF4F3883C258D040F9
:10EB1000CD57DF4F4883C358D040CC57DF4F588381
:10EB2000C458D040CB57DF4F6883C558D040CA5730
:10EB3000DF4F7883C658D040C957DF4F8883C75806
:10EB4000D040C857DF4F9883C858D040CE010196B7
:10EB50000E94A431662069F1C655DF4F8881CA5AE8
:10EB6000D04082958F709FE0980F9F70923020F078
:10EB70008A5F8F708230E8F48A8182958F7081502D
:10EB80008230B8F42D8130E0AFEFB0E00E94E3F0C6
:10EB900024E630E040E050E00E94B1F02F3F310524
:10EBA0004105510529F024F02FEF30E040E050E01E
:10EBB0002D8388E0FE013196DE01A755BF4F0190FD
:10EBC0000D928A95E1F7F2E1BF2A812CD1011896C6
:10EBD0008C911897873009F005C7C954DF4FE88139
:10EBE000F981C75BD040EE35F1400CF06CC46CEAA3
:10EBF00078E189EE9DE00E94CC99EDCD3BE0431693
:10EC0000510409F4CDC08CE04816510409F0B4CE8B
:10EC1000B101CE0101960E947FB2CE0187559F4F70
:10EC20000E94DF62BC01CE0101960E94016388E070
:10EC3000FE013196DE01A755BF4F01900D928A95D6
:10EC4000E1F7FBC0EF2B59F068ED78E183EF9DE031
:10EC50000E94CC9983EF9DE00E9436988DCEC10131
:10EC60000E9484728C0161E070E01816190614F09D
:10EC700070E060E083EF9DE00E94AAAE62E475E080
:10EC800083EF9DE00E946699CE0187559F4F0E94B9
:10EC90003361AB01BC012AE030E083EF9DE00E94CC
:10ECA000DC9883EF9DE00E943698CE0187559F4FF8
:10ECB0001016110614F00C94FA830E943361B12CE3
:10ECC000A12C672B682B692B89F562E0CE01875553
:10ECD0009F4F0E945B33CF56DF4F2883C159D040EE
:10ECE000CE56DF4F3883C259D040CD56DF4F4883D0
:10ECF000C359D040CC56DF4F5883C459D040CB566F
:10ED0000DF4F6883C559D040CA56DF4F7883C65954
:10ED1000D040C956DF4F8883C759D040C856DF4F0F
:10ED20009883C859D040AA24A394BA2C662463942B
:10ED3000772473947BCE61E0CE0187559F4F0E946C
:10ED40005B33C757DF4F2883C958D040C657DF4FC2
:10ED50003883CA58D040C557DF4F4883CB58D0407E
:10ED6000C457DF4F5883CC58D040C357DF4F688318
:10ED7000CD58D040C257DF4F7883CE58D040C157CE
:10ED8000DF4F8883CF58D040C057DF4F9883C0599A
:10ED9000D040AA24A394BA2C66246394712C46CE46
:10EDA000B101CE0101960E947FB2C255DF4F88812A
:10EDB000CE5AD0409A8192959F7041F0923051F096
:10EDC000B12CA12C88248394612C0AC29A819F7053
:10EDD00090629A8390E08536910514F084E690E085
:10EDE0008E8388E0FE013196DE01A755BF4F01906A
:10EDF0000D928A95E1F762E0CE0187559F4F0E9400
:10EE00003433EA962FAFEA97EB963FAFEB97EC9649
:10EE10004FAFEC97ED965FAFED97EE966FAFEE9735
:10EE2000EF967FAFEF97C158DF4F8883CF57D04021
:10EE3000C058DF4F9883C058D040A12C22E1B22E99
:10EE4000812CC2CFB101CE0101960E947FB2C15583
:10EE5000DF4F6881CF5AD040C055DF4F7881C05B0B
:10EE6000D0407170CE0101960E947C68682E882384
:10EE700009F4BEC288E0FE013196DE01A755BF4FFE
:10EE800001900D928A95E1F762E0CE0187559F4F80
:10EE90000E943433E2962FAFE297E3963FAFE397B9
:10EEA000E4964FAFE497E5965FAFE597E6966FAFD0
:10EEB000E697E7967FAFE797E8968FAFE897E996F2
:10EEC0009FAFE997BACFC1010E9484721816190644
:10EED0003CF562E0CE0187559F4F0E945B33AA96B6
:10EEE0002FAFAA97AB963FAFAB97AC964FAFAC970F
:10EEF000AD965FAFAD97AE966FAFAE97AF967FAF63
:10EF0000AF97E0968FAFE097E1969FAFE197AA2485
:10EF1000A394BA2C812C662463947724739456CEE0
:10EF200061E0CE0187559F4F0E945B33A2962FAFC1
:10EF3000A297A3963FAFA397A4964FAFA497A59689
:10EF40005FAFA597A6966FAFA697A7967FAFA79737
:10EF5000A8968FAFA897A9969FAFA997AA24A39424
:10EF6000BA2C812C66246394712C30CEC355DF4FAC
:10EF7000288139814A815B81CD5AD040A4E6B0E036
:10EF80000E94D0F06B017C010DC0C355DF4FC880DB
:10EF9000CD5AD04004E6C09E600111240D2C000C17
:10EFA000EE08FF08C114D104E104F10429F405E0DE
:10EFB000C02ED12CE12CF12C193041F4F094E094C6
:10EFC000D094C094C11CD11CE11CF11CB101CE0134
:10EFD00087559F4F0E947FB260E0CE0187559F4FBB
:10EFE0000E945B336A962FAF6A976B963FAF6B9721
:10EFF0006C964FAF6C976D965FAF6D976E966FAFD7
:10F000006E976F967FAF6F97A0968FAFA097A196E0
:10F010009FAFA19712E04116510409F4ACC00CF067
:10F0200059C0662463944114510409F0A5CCD10160
:10F0300019968D919C911A97009709F09EC0189689
:10F040008C9190E0A0E58A2E912CA12CB12C8530DA
:10F05000910549F0812C912C5401449721F0812C89
:10F06000912C54018A94C655DF4FE881CA5AD0408A
:10F07000E295EF70E150EB3008F0B0C1F0E0882786
:10F08000EB5BF7488F4F0C941AF1C578C578EE7991
:10F09000EE79EE79BB79797979797979F378F378C2
:10F0A00020E030E048EC52E4C355DF4F68817981BD
:10F0B0008A819B81CD5AD0400E94ABEF0E9417F20B
:10F0C00061CFC355DF4FC880D980EA80FB80CD5A1D
:10F0D000D04068CF3AE04316510409F48EC18BE06A
:10F0E0004816510409F048CCC655DF4F8881CA5AEA
:10F0F000D04082958F70823009F0DAC1C701B60125
:10F1000024E630E040E050E00E94B1F0C255DF4F0D
:10F110008881CE5AD04090E0280F391F37FF02C0B7
:10F1200030E020E02536310514F024E630E0C25509
:10F13000DF4F2883CE5AD04062E0CE0187559F4FE3
:10F140000E9434332A962FAF2A972B963FAF2B97E6
:10F150002C964FAF2C972D965FAF2D972E966FAFB5
:10F160002E972F967FAF2F9760968FAF60976196FF
:10F170009FAF619762CE612C5ACFDC01ED91FC917B
:10F18000048CF58DE02D19955DCFC355DF4F1881A7
:10F19000CD5AD040C701B60124E630E040E050E04F
:10F1A0000E94B1F0DA01C901810F911DA11DB11DAD
:10F1B000B7FF03C080E090E0DC018F3F9105A1051F
:10F1C000B10529F024F08FEF90E0A0E0B0E0C35546
:10F1D000DF4F8883CD5AD040A12CF2E1BF2E812C85
:10F1E00077247A94F3CCC355DF4F088119812A81A3
:10F1F0003B81CD5AD040C754DF4F088319832A83FF
:10F200003B83C95BD04014E6C116D104E104F1048C
:10F210000CF041C0A4E6B0E0C754DF4F288139812B
:10F220004A815B81C95BD0400E94D0F0C60ED71ED8
:10F23000E81EF91E81149104A104B104B9F0A501DE
:10F2400094010E94D0F0362F272FB701A60177FF37
:10F2500003C040E050E0BA01C32ED22E7C014C1511
:10F260005D056E057F0514F46A017B01C355DF4F10
:10F27000C882D982EA82FB82CD5AD040C655DF4F80
:10F280008881CA5AD0408F708066C655DF4F888308
:10F29000CA5AD040A1CFC701B60124E630E040E011
:10F2A00050E00E94B1F0C754DF4F88819981AA8154
:10F2B000BB81C95BD040280F391F4A1F5B1F8114D7
:10F2C0009104A104B10461F057FF03C020E030E0D5
:10F2D000A90182169306A406B50614F4A5019401AB
:10F2E000C355DF4F288339834A835B83CD5AD0408F
:10F2F00073CFC355DF4F688179818A819B81CD5A55
:10F30000D0400E9417F2C754DF4F688379838A8305
:10F310009B83C95BD040C701B60124E630E040E0E2
:10F3200050E00E94B1F0C754DF4F688179818A8133
:10F330009B81C95BD040620F731F841F951F81148E
:10F340009104A104B10461F097FF03C060E070E094
:10F35000CB0186169706A806B90614F4C501B401B8
:10F360000E944CEFC355DF4F688379838A839B8368
:10F37000CD5AD04031CFC355DF4F88819981AA81C2
:10F38000BB81CD5AD040C80ED91EEA1EFB1E811487
:10F390009104A104B104C9F0A4E6B0E0A501940170
:10F3A0000E94D0F0362F272FB701A60177FF03C0A8
:10F3B00040E050E0BA01C32ED22E7C014C155D0511
:10F3C0006E057F0514F46A017B01C355DF4FC882C7
:10F3D000D982EA82FB82CD5AD040FECE88E0FE017F
:10F3E0003196DE01A755BF4F01900D928A95E1F746
:10F3F000B12CA12C88248394F3CEC655DF4F88818D
:10F40000CA5AD04082958F70823009F051C0C7012E
:10F41000B60124E630E040E050E00E94B1F0C15572
:10F42000DF4F8881CF5AD040C055DF4F6881C05B25
:10F43000D040962F9170280F391F2E3691E0390752
:10F440002CF437FF05C02DE631E002C030E020E0AB
:10F45000C155DF4F2883CF5AD040C055DF4F888138
:10F46000C05BD04030FB80F9C055DF4F8883C05B64
:10F47000D04062E0CE0187559F4F0E9434336296A0
:10F480002FAF629763963FAF639764964FAF6497D1
:10F4900065965FAF659766966FAF669767967FAF25
:10F4A000679768968FAF689769969FAF6997C5CC45
:10F4B00088E0FE013196DE01A755BF4F01900D9205
:10F4C0008A95E1F77DCCCD54DF4F1881C35BD040E6
:10F4D000112339F11296ED91FC9180858F70853062
:10F4E00001F5C354DF4FE881F981CD5BD0403597FA
:10F4F000C1F0C1010E948472772473941816190612
:10F500000CF0712CCF54DF4F48815981C15BD04042
:10F51000BE0167557F4FD10112968D919C910E943B
:10F52000C471C755DF4F8881C95AD040853009F46E
:10F53000EBC128F4833009F46CC0C501E7C0863004
:10F5400009F4F7C08730C9F7C1010E94C570182FB0
:10F55000863009F0DDC0E1E04E165104C9F5C6550C
:10F56000DF4F8881CA5AD040807F91F1711005C069
:10F57000C1010E94435C892B59F1C755DF4F0881B7
:10F58000C95AD040C655DF4F1881CA5AD040C55518
:10F59000DF4F2881CB5AD040C455DF4F3881CC5A39
:10F5A000D040C355DF4F4881CD5AD040C255DF4FC0
:10F5B0005881CE5AD040C155DF4F6881CF5AD040D4
:10F5C000C055DF4F7881C05BD040C1010E942562E9
:10F5D00060E878E183EF9DE00E94CC9966E070E0FE
:10F5E00083EF9DE00E94AAAE83EF9DE00E943698D3
:10F5F00062E0CE0187559F4F0E945B3329AF3AAF3F
:10F600004BAF5CAF6DAF7EAF8FAF21969FAF2197B1
:10F610007AC0C1010E94C570853021F093E0C92EE7
:10F62000D12CA8C2B1E04B165104C9F5C655DF4F25
:10F630008881CA5AD040807F91F1772029F0C1019A
:10F640000E94435C892B59F1C755DF4F0881C95A85
:10F65000D040C655DF4F1881CA5AD040C555DF4F3C
:10F660002881CB5AD040C455DF4F3881CC5AD04086
:10F67000C355DF4F4881CD5AD040C255DF4F588126
:10F68000CE5AD040C155DF4F6881CF5AD040C055C7
:10F69000DF4F7881C05BD040C1010E94256267E9DD
:10F6A00078E183EF9DE00E94CC9965E070E083EF04
:10F6B0009DE00E94AAAE83EF9DE00E943698B101C2
:10F6C000CE0187559F4F0E947FB261E0CE018755E2
:10F6D0009F4F0E945B3322962FAF229723963FAF16
:10F6E000239724964FAF249725965FAF25972696AC
:10F6F0006FAF269727967FAF279728968FAF2897CB
:10F7000029969FAF2997C50181609160912C82C095
:10F7100062E678E183EF9DE00E94CC99612F70E072
:10F7200083EF9DE00E94AAAE83EF9DE00E94369891
:10F7300075CF40E050E061E070E0C1010E94B96B1C
:10F74000672B682B692B09F0DCC0FFEF7F1209C023
:10F75000C1010E94847277247394181619060CF064
:10F76000712C01E040165104D1F5C655DF4F888158
:10F77000CA5AD040807F99F1772031F0C1010E94B0
:10F78000435C892B09F4B6C0C755DF4F0881C95ABD
:10F79000D040C655DF4F1881CA5AD040C555DF4FFB
:10F7A0002881CB5AD040C455DF4F3881CC5AD04045
:10F7B000C355DF4F4881CD5AD040C255DF4F5881E5
:10F7C000CE5AD040C155DF4F6881CF5AD040C05586
:10F7D000DF4F7881C05BD040C1010E94256271106B
:10F7E00089C0B101CE0187559F4F0E947FB261E071
:10F7F000CE0187559F4F0E945B3329AB3AAB4BAB91
:10F800005CAB6DAB7EAB8FAB98AFC5018160916097
:10F81000E6E09E2E5C016894A0F8C655DF4F288173
:10F82000CA5AD040322F3F70323058F4C755DF4F9C
:10F830003881C95AD040332321F05C016894A0F884
:10F84000B0F8207F09F4C3C06894B1F8CD54DF4FFD
:10F850006882C35BD040CC24C394D12C81100C941B
:10F860009D84F10181859285009709F033C640E0BF
:10F8700050E062E070E0C1010E94B96B672B682B19
:10F88000692B09F459C664E077E189EE9DE00E9496
:10F89000CC9989EE9DE00E943698B2FC96C769EE3D
:10F8A00076E183EF9DE00E94CC99B60183EF9DE065
:10F8B0000E94AAAE62EE76E183EF9DE00E94CC99B1
:10F8C0000E9433BCAB01BC01C154DF4F08811981D8
:10F8D0002A813B81CF5BD040401B510B620B730BE5
:10F8E0002AE083EF9DE00E94EA9783EF9DE00E946B
:10F8F000369840C168E478E183EF9DE00E94CC999E
:10F900008DCE63E378E1F8CF1FEF711209C0C1011A
:10F910000E94847277247394181619060CF0712CC7
:10F9200021E042165104D1F5C655DF4F8881CA5AED
:10F93000D040807F99F1711006C0C1010E94435CE4
:10F94000892B09F441C0C755DF4F0881C95AD040FF
:10F95000C655DF4F1881CA5AD040C555DF4F2881A0
:10F96000CB5AD040C455DF4F3881CC5AD040C35514
:10F97000DF4F4881CD5AD040C255DF4F5881CE5A13
:10F98000D040C155DF4F6881CF5AD040C055DF4FBE
:10F990007881C05BD040C1010E9425627720A1F030
:10F9A00062E0CE0187559F4F0E945B3329A73AA79B
:10F9B0004BA75CA76DA77EA78FA798ABC5018160F9
:10F9C000916075E0972E26CF66E178E195CF40E013
:10F9D00052E0B101CE0187559F4F0E94A4328111A0
:10F9E00033CF34CF3FEF731294C0C1010E948472B1
:10F9F00077247394181619060CF48EC0712C68E0E5
:10FA000078E183EF9DE00E94CC99072D072C000C34
:10FA1000110BC954DF4F19830883C75BD040B8016D
:10FA200083EF9DE00E94AAAE61E078E183EF9DE064
:10FA30000E94CC99662D70E083EF9DE00E94AAAEF3
:10FA400083EF9DE00E943698CF54DF4FE880F98025
:10FA5000C15BD040E114F10409F4B1C06EE37AE176
:10FA6000C7010E9450E9CC24C394D12C892B09F4FE
:10FA700059C06AE37AE1C7010E9450E942E0C42E0E
:10FA8000D12C892B09F44EC06DED76E1C7010E949F
:10FA900050E935E0C32ED12C892B09F443C069ED20
:10FAA00076E1C7010E9450E926E0C22ED12C892BB5
:10FAB000C9F16FEF79E1C7010E9450E9892B79F113
:10FAC0006AEF79E1C7010E9450E9892B09F46DC002
:10FAD00064E07AE1C7010E9450E90EE0C02ED12C0B
:10FAE000892B01F16DEE79E1C7010E9450E91FE019
:10FAF000C12ED12C892BB1F066EF79E1C7010E94AC
:10FB000050E9D12CC12C892B69F4B5E1CB2ED12C35
:10FB100009C0772009F473CF6624639470CF93E112
:10FB2000C92ED12CC1010E94C570082F10E001150B
:10FB3000110531F4C954DF4F08811981C75BD040EA
:10FB4000C114D10409F460C00C151D0591F165EED6
:10FB500077E183EF9DE00E94CC99B80183EF9DE0AF
:10FB60000E94AAAE83EF9DE00E943698ADEFCA2EA8
:10FB7000DD24DA94C601CE53DF4F0FB6F894DEBF12
:10FB80000FBECDBFDF91CF911F910F91FF90EF90EE
:10FB9000DF90CF90BF90AF909F908F907F906F90AD
:10FBA0005F904F903F902F90089584E1C82ED12C04
:10FBB000B9CFCF54DF4F19821882C15BD040C755EF
:10FBC000DF4FE881C95AD040E63108F037C4F0E091
:10FBD0008827E251F2488F4F0C941AF13F829A80A5
:10FBE0003C803D7E3F82D47F507FCE7E3F823F82ED
:10FBF000238149819681F481038103811E821E82C3
:10FC00001E82038103810381D10119968D919C91FC
:10FC1000009709F4AFCFDC01ED91FC910488F589E0
:10FC2000E02DC62CC755DF4F0881C95AD040C655B4
:10FC3000DF4F1881CA5AD040C555DF4F2881CB5AB3
:10FC4000D040C455DF4F3881CC5AD040C355DF4F28
:10FC50004881CD5AD040C255DF4F5881CE5AD0404E
:10FC6000C155DF4F6881CF5AD040C055DF4F7881F2
:10FC7000C05BD04019950C94AE74C1010E94C57050
:10FC8000853009F0CBCCB1E04B16510409F040C0EF
:10FC9000CD54DF4FE881C35BD040EE23C9F1C65598
:10FCA000DF4F8881CA5AD040807F91F1711005C022
:10FCB000C1010E94435C892B59F1C755DF4F088170
:10FCC000C95AD040C655DF4F1881CA5AD040C555D1
:10FCD000DF4F2881CB5AD040C455DF4F3881CC5AF2
:10FCE000D040C355DF4F4881CD5AD040C255DF4F79
:10FCF0005881CE5AD040C155DF4F6881CF5AD0408D
:10FD0000C055DF4F7881C05BD040C1010E942562A1
:10FD100060ED77E183EF9DE00E94CC9965E070E0B3
:10FD200083EF9DE00E94AAAE83EF9DE00E9436988B
:10FD3000B101CE0187559F4F0E947FB2D101189625
:10FD40008C918530E1F46EE0CE0187559F4F0E9483
:10FD50005B3329A33AA34BA35CA36DA37EA38FA31C
:10FD600098A76894A0F8B0F8912CCC24CA94DC2C05
:10FD7000B1E0CD54DF4FB883C35BD0406FCD61E0BD
:10FD8000CE0187559F4F0E945B33298F3A8F4B8F4F
:10FD90005C8F6D8F7E8F8F8F98A3E3CFC1010E9400
:10FDA000C570182F863009F078C0E1E04E16510476
:10FDB00009F040C0CD54DF4FF881C35BD040FF2332
:10FDC000C9F1C655DF4F8881CA5AD040807F91F172
:10FDD000711005C0C1010E94435C892B59F1C755C0
:10FDE000DF4F0881C95AD040C655DF4F1881CA5A23
:10FDF000D040C555DF4F2881CB5AD040C455DF4F86
:10FE00003881CC5AD040C355DF4F4881CD5AD040BD
:10FE1000C255DF4F5881CE5AD040C155DF4F68815F
:10FE2000CF5AD040C055DF4F7881C05BD040C10170
:10FE30000E94256269EB77E183EF9DE00E94CC99F7
:10FE400066E070E083EF9DE00E94AAAE83EF9DE044
:10FE50000E94369862E0CE0187559F4F0E945B3327
:10FE6000298B3A8B4B8B5C8B6D8B7E8B8F8B988F1A
:10FE700040E050E068E070E0C1010E94676B689468
:10FE8000A0F8B0F8912CCC24CA94DC2C01E0CD541D
:10FE9000DF4F0883C35BD040E1CC6BE977E13ACC1C
:10FEA00040E050E061E070E0C1010E94B96B672B57
:10FEB000682B692B09F075C011E04116510409F057
:10FEC00041C0CD54DF4F2881C35BD0402223D1F104
:10FED000C655DF4F8881CA5AD040807F99F177207C
:10FEE00031F0C1010E94435C892B09F457C0C7550A
:10FEF000DF4F0881C95AD040C655DF4F1881CA5A12
:10FF0000D040C555DF4F2881CB5AD040C455DF4F74
:10FF10003881CC5AD040C355DF4F4881CD5AD040AC
:10FF2000C255DF4F5881CE5AD040C155DF4F68814E
:10FF3000CF5AD040C055DF4F7881C05BD040C1015F
:10FF40000E94256271102AC0B101CE0187559F4FD2
:10FF50000E947FB261E0CE0187559F4F0E945B33C4
:10FF600029873A874B875C876D877E878F87988B39
:10FF700040E050E068E070E0C1010E94906B68943E
:10FF8000A0F8B0F8F6E09F2ECC24CA94DC2C31E027
:10FF9000CD54DF4F3883C35BD04060CC61E877E15C
:10FFA000ABCC6CE677E1A8CC81E04816510409F0AF
:10FFB00041C0CD54DF4F9881C35BD0409923D1F12C
:10FFC000C655DF4F8881CA5AD040807F99F17110A1
:10FFD00006C0C1010E94435C892B09F44AC0C75581
:10FFE000DF4F0881C95AD040C655DF4F1881CA5A21
:10FFF000D040C555DF4F2881CB5AD040C455DF4F84
:020000021000EC
:100000003881CC5AD040C355DF4F4881CD5AD040BB
:10001000C255DF4F5881CE5AD040C155DF4F68815D
:10002000CF5AD040C055DF4F7881C05BD040C1016E
:100030000E9425627720E9F062E0CE0187559F4F4C
:100040000E945B3329833A834B835C836D837E8379
:100050008F8398876894A0F8B0F8E5E09E2ECC24B2
:10006000CA94DC2CA1E0CD54DF4FA883C35BD04001
:10007000F5CB6FE477E140CCC655DF4F1881CA5A03
:10008000D040812F8F70912C823008F014C2C101B2
:100090000E94C570853009F4C1CAB1E04B16510405
:1000A000D9F5CD54DF4FE881C35BD040EE23A1F1F9
:1000B000107F91F1711005C0C1010E94435C892B32
:1000C00059F1C755DF4F0881C95AD040C655DF4F97
:1000D0001881CA5AD040C555DF4F2881CB5AD0402D
:1000E000C455DF4F3881CC5AD040C355DF4F4881CB
:1000F000CD5AD040C255DF4F5881CE5AD040C1555D
:10010000DF4F6881CF5AD040C055DF4F7881C05B48
:10011000D040C1010E9425626894A0F8B0F8912CEB
:10012000CC24CA94DC2CF1E0CD54DF4FF883C35BC0
:10013000D04094CB01E04016510409F040C0CD54AA
:10014000DF4F1881C35BD0401123C9F1C655DF4F83
:100150008881CA5AD040807F91F1772029F0C1016F
:100160000E94435C892B59F1C755DF4F0881C95A5A
:10017000D040C655DF4F1881CA5AD040C555DF4F11
:100180002881CB5AD040C455DF4F3881CC5AD0405B
:10019000C355DF4F4881CD5AD040C255DF4F5881FB
:1001A000CE5AD040C155DF4F6881CF5AD040C0559C
:1001B000DF4F7881C05BD040C1010E942562C655E7
:1001C000DF4F8881CA5AD0408F70912C823008F05E
:1001D00046CFC755DF4F9880C95AD040992009F4BF
:1001E000C4CD772081F066E377E183EF9DE00E9444
:1001F000CC9961E0C1010E94947060E071E1C1019D
:100200000E94F26E0BCAC655DF4F8881CA5AD04091
:10021000982F9F70923008F038C1C755DF4F9880F3
:10022000C95AD040992009F47BCF807F31F4B101C5
:10023000CE0187559F4F0E947FB26894A0F823E0BB
:10024000B22A912CA1CE6894B2F8CD54DF4F8881A8
:10025000C35BD040882309F415CEC655DF4F888193
:10026000CA5AD040807F81F040E050E061E070E009
:10027000C1010E94B96B672B682B692B59F5C1012D
:100280000E94435C892B31F5912CCC24CA94DC2C40
:10029000E5CA6894B2F891E04916510409F000C12A
:1002A000CD54DF4FA881C35BD040AA2309F4CFC04F
:1002B000C655DF4F8881CA5AD040807F29F340E07D
:1002C00050E061E070E0C1010E94B96B672B682BC0
:1002D000692BA9F6C755DF4F0881C95AD040C655CA
:1002E000DF4F1881CA5AD040C555DF4F2881CB5AFD
:1002F000D040C455DF4F3881CC5AD040C355DF4F72
:100300004881CD5AD040C255DF4F5881CE5AD04097
:10031000C155DF4F6881CF5AD040C055DF4F78813B
:10032000C05BD040C1010E942562AECF912CA12CB0
:1003300084E0B82EB1E04B16510409F025CECD541F
:10034000DF4FE881C35BD040912CA12C14E0B12E8B
:10035000EE2309F48AC0C655DF4F8881CA5AD040BF
:10036000807F09F4B2C040E050E062E070E0C1017B
:100370000E94B96B672B682B692B31F4C1010E9475
:10038000435C892B09F4A1C0C755DF4F0881C95AC6
:10039000D040C655DF4F1881CA5AD040C555DF4FEF
:1003A0002881CB5AD040C455DF4F3881CC5AD04039
:1003B000C355DF4F4881CD5AD040C255DF4F5881D9
:1003C000CE5AD040C155DF4F6881CF5AD040C0557A
:1003D000DF4F7881C05BD040C1010E942562912C23
:1003E000A12C74E0B72E9CCE912CA12CA4E0BA2EA7
:1003F00001E04016510409F05EC0CD54DF4F188172
:10040000C35BD040912CA12CE4E0BE2E112309F453
:1004100026CEC655DF4F8881CA5AD040807F09F466
:1004200054C040E050E062E070E0C1010E94B96B4E
:10043000672B682B692B09F4A7CFA0CFC655DF4FD8
:100440008881CA5AD040807F69F46894B0F8912CB2
:10045000CC24CA94DC2C21E0CD54DF4F2883C35B2D
:10046000D040FCC933E0B32A912CCC24CA94DC2CB4
:1004700081E0CD54DF4F8883C35BD040EFC9CD54BA
:10048000DF4F6882C35BD040FFCE912CCC24CA944E
:10049000DC2CE1E0CD54DF4FE883C35BD040DEC904
:1004A000912CCC24CA94DC2C11E0CD54DF4F18835E
:1004B000C35BD040D3C9CC24CA94DC2C91E0CD548A
:1004C000DF4F9883C35BD040C9C9912CA12C64E055
:1004D000B62EDBCEDC01ED91FC91008CF18DE02D90
:1004E000C755DF4F0881C95AD040C655DF4F188124
:1004F000CA5AD040C555DF4F2881CB5AD040C45589
:10050000DF4F3881CC5AD040C355DF4F4881CD5A98
:10051000D040C255DF4F5881CE5AD040C155DF4F31
:100520006881CF5AD040C055DF4F7881C05BD04042
:10053000199581119CC9A7C9A114B10439F0A5016D
:10054000B101CE0187559F4F0E94F231F1018185A3
:100550009285009709F45FC0CF54DF4FE880F9809F
:10056000C15BD040DC01ED91FC910488F589E02D60
:10057000CD54DF4FC880C35BD040C755DF4F0881E3
:10058000C95AD040C655DF4F1881CA5AD040C55508
:10059000DF4F2881CB5AD040C455DF4F3881CC5A29
:1005A000D040C355DF4F4881CD5AD040C255DF4FB0
:1005B0005881CE5AD040C155DF4F6881CF5AD040C4
:1005C000C055DF4F7881C05BD04019956C01F101B7
:1005D00081859285DC01ED91FC91048CF58DE02DF7
:1005E0001995059711F46894A0F8B2FCE6C099201B
:1005F00021F0692DC1010E949470C354DF4FE8813E
:10060000F981CD5BD040B501359709F448C9C101E6
:100610000E94F26E44C98085853009F46AC0863034
:1006200031F7C755DF4F8880C95AD040882009F478
:1006300060C070E060E0C1010E94CA698C0100974F
:10064000B1F2F12CE12C97FF06C01195019511092B
:10065000EE24E394F12CC80101978635910538F614
:10066000D02E61E0802F0E94A9BAEFEFE80DE531AE
:1006700010F5F0E08827E05CFC478F4F0C941AF1EE
:10068000558357835B835B835783558357835B8392
:100690005B835B835B835B835B83558355835B8376
:1006A0005B835B835B8355835583F1E0EF266E2D7F
:1006B0008D2D0E947BBA6FEF76E183EF9DE00E9463
:1006C000CC99B80183EF9DE00E94AAAE6DEF76E170
:1006D00083EF9DE00E94CC99B70183EF9DE00E94DB
:1006E000AAAE83EF9DE00E9436986894A0F8B0F817
:1006F00064C002E04016510409F463C013E04116DF
:10070000510429F04A94452809F071CFEECFC10178
:100710000E948469892B49F4D101ED91FC9160819B
:1007200071818DEC96E00E941CBDCE0187559F4FD4
:100730000E94EC6020E030E048EC52E40E94ABEF15
:100740000E9417F2CD54DF4F688379838A839B839D
:10075000C35BD040CD54DF4FC880D980C35BD0404D
:1007600088E00E9483222B013C0169EF76E183EF50
:100770009DE00E94CC99CD54DF4F68817981C35BA5
:10078000D04083EF9DE00E94AAAE64EF76E183EF54
:100790009DE00E94CC99B301A201662777272AE049
:1007A00083EF9DE00E94EA9783EF9DE00E943698D8
:1007B000B201A601C1010E942469CC24C394D12CAA
:1007C00016CF6894A0F8B1F8F8CFC354DF4F088172
:1007D0001981CD5BD0400530110509F460C840E0B7
:1007E00054E0B101CE0187559F4F0E94F23160E085
:1007F00074E00DCF0E943361672B682B692B11F0D9
:100800000C949B76B12CA12C0C94CC764114510401
:1008100009F045C08081882311F40C943874CE010E
:100820008F549F4F0E949B682C01C655DF4F8881D3
:10083000CA5AD0408F7071F5642DCE0187559F4FF5
:100840000E943433CF55DF4F2883C15AD040CE5554
:10085000DF4F3883C25AD040CD55DF4F4883C35A4B
:10086000D040CC55DF4F5883C45AD040CB55DF4FD2
:100870006883C55AD040CA55DF4F7883C65AD040E6
:10088000C955DF4F8883C75AD040C855DF4F98837A
:10089000C85AD0404114510411F40C94387460E1EA
:1008A00079E183EF9DE00E94CC99B60183EF9DE052
:1008B0000E94AAAE69E079E183EF9DE00E94CC99A5
:1008C000D101ED91FC916081718183EF9DE00E94E7
:1008D000669963E079E183EF9DE00E94CC99CF5463
:1008E000DF4F68817981C15BD04083EF9DE00E943A
:1008F000669961E079E183EF9DE00E94CC99CE0199
:1009000087559F4F0E94A431CF54DF4FE881F98172
:10091000C15BD040309711F40C947974808184329B
:1009200011F00C9479746DEE78E183EF9DE00E94F4
:10093000CC9983EF9DE00E9436988CEFC82EDD2481
:10094000DA9418C92F923F924F925F926F927F92E2
:100950008F929F92AF92BF92CF92DF92EF92FF92CF
:100960000F931F93CF93DF93CDB7DEB7A8970FB642
:10097000F894DEBF0FBECDBF5C014B015090B709AC
:10098000552009F4BEC08091C1098F5F8093C109D1
:10099000E091C509F091C609309709F4AAC06680B4
:1009A00077802090C5093090C6092114310409F4DC
:1009B0009CC06114710409F498C0D30118968C91FD
:1009C0008F70853091F7C3010E94B2AE823068F318
:1009D000B301CE0101960E94AE71CE0101960E9434
:1009E000CF68882309F464C040E058E060E070E01C
:1009F000CE0101960E94B96B672B682B692B09F415
:100A000057C01E8E1F8E18A219A21AA21BA21CA2CA
:100A10001DA28F8D8F708F8F40E053E0BE016F5FFE
:100A20007F4FCE014E960E94A4326EE679E183EFAD
:100A30009DE00E94CC9940E058E060E070E0CE017B
:100A400001960E94676B8A859B85009789F1DC017E
:100A5000ED91FC910488F589E02DCC24C394F12C10
:100A6000E12C0E8D1F8D28A139A14AA15BA16CA19B
:100A70007DA119958F3F9807D9F0E981FA816081AE
:100A80007181892BE9F483EF9DE00E9466996CE601
:100A900079E183EF9DE00E94CC9964E679E183EFF0
:100AA0009DE00E94CC9983EF9DE00E943698512CE6
:100AB000F30162807380CE0101960E94A07171CF14
:100AC00083EF9DE00E94669962E679E183EF9DE005
:100AD0000E94CC996EE579E183EF9DE00E94CC996C
:100AE00083EF9DE00E943698E3CF83EF9DE00E9464
:100AF00036988091C10981508093C109511010929C
:100B0000B70965E0D5018D919C910E949BAE1C01B7
:100B1000009709F4BCC0FC01808585958595859575
:100B200085958EA341845284638474840E9433BC6F
:100B3000FEA1FF2309F4ABC0461A570A680A790AD6
:100B40001E8E1F8E18A219A2FE8F1F8D1F70106A95
:100B50001F8F4AA25BA26CA27DA224E082169104A0
:100B600049F5D12CC12CE12C90E2F92E0F2F28A1B0
:100B700039A14AA15BA16CA17DA1C5010E94DD6BD9
:100B8000C301B20128EE33E040E050E00E94B1F032
:100B9000BA01A9012AE030E083EF9DE00E94DC98D1
:100BA0006CE979E183EF9DE00E94CC9983EF9DE0B1
:100BB0000E94369877FE6BC082E0481651046104AB
:100BC00080E878060CF463C00E943F292B0178A7C7
:100BD0006FA3D12CC12CE12C80E2F82E0E8D1F8D3D
:100BE00028A139A14AA15BA16CA17DA1C5010E94E8
:100BF000DD6BAFA1B8A5A83CB10554F563E879E178
:100C000089EE9DE00E94CC99B20189EE9DE00E94A0
:100C1000AAAE89EE9DE00E9436988FEF9FEFA896CE
:100C20000FB6F894DEBF0FBECDBFDF91CF911F91FD
:100C30000F91FF90EF90DF90CF90BF90AF909F907B
:100C40008F907F906F905F904F903F902F9008957E
:100C500019821A821B821C821D821E821F821886A4
:100C60001A811F701A83BEA1B983CC24C394F12CBE
:100C7000E12C0B2F2B813C8140E05E816F817885D8
:100C8000C5010E948573F10180858F708087F1E036
:100C90008F169104E9F440E053E060E070E0C50194
:100CA0000E94B96B611571058105910589F020914C
:100CB000C3093091C4092630310551F4C5010E94A1
:100CC000F26E40E053E060E070E0C5010E94676BA7
:100CD000D50119968D919C91009719F490E080E0D0
:100CE0009ECFDC01ED91FC910484F585E02D1995F2
:100CF000892BA1F3F50181859285DC01ED91FC91B1
:100D00000480F581E02DB401199589CFCF93DF934D
:100D1000EC01FB0124813581408151816281738125
:100D20000E94DC98CE01DF91CF9108953F924F92BF
:100D30005F926F927F928F929F92AF92BF92CF926B
:100D4000DF92EF92FF920F931F93CF93DF93CDB774
:100D5000DEB7CE56D1090FB6F894DEBF0FBECDBFB9
:100D6000DC0114962D913C91232B09F421C69B01A3
:100D7000225031092230310508F091C23B014C016B
:100D8000FC018281803409F4F7C208F04AC0843043
:100D900008F085C28091B6098F5F8093B609A301E0
:100DA0006FEFC4010E94565DD40112960C91129708
:100DB0000695017013961C9113978AEC810F803170
:100DC00008F043C06CED76E08D919C910E9423AEBB
:100DD0007C010097D1F1FC0180858F708530A9F5E9
:100DE0008091160D181324C08091170D803401F5E1
:100DF0008091180D9091190D5C01990FCC08DD08B8
:100E000060E0C7010E949BAEFC0181859285A385AD
:100E1000B485A816B906CA06DB060CF065C0512CCD
:100E20003EC0823409F4A8C208F439C28058AFCF5A
:100E30001093160D80E48093170D812F0E94BCBB88
:100E40009093190D8093180DD7CF212F30E0F90121
:100E5000EC5DF04E8491F901E253F14E1491F901E9
:100E6000E858F14EF490FF2009F43BC081110E9434
:100E700014BAEF2DF0E0EE0FFF1FE75DF94EA591DC
:100E8000B491EC911E2331E020E009F430E0832F8F
:100E9000922F552453940817190609F0C0CFF3E098
:100EA0006F16710409F488C0D4011496ED91FC9179
:100EB000E181EF70E150EC3008F07EC0F0E088276F
:100EC000EB59F8478F4F0C941AF186870289BC873B
:100ED000F28702890B8802893F886C888588C788D9
:100EE000E98890E080E0D5CF61E0C7010E949BAE29
:100EF00055245394FC0181859285A385B4858A1578
:100F00009B05AC05BD050CF0CACF89CF0E9433BC50
:100F10009B01AC0144275527D4011496ED91FC9117
:100F20006281738190E080E0AA24AA94BA2CC12C3B
:100F3000D12C18EEE12E13E0F12E00E010E00E941B
:100F400021228823C9F1F4010081118168EA76E049
:100F5000C8010E9423AE892B41F46DEA76E0C801F6
:100F60000E9423AE892B09F40EC142E050E063E0F9
:100F7000C4010E94565D20C00E9433BC9B01AC019D
:100F800044275527D4011496ED91FC916281738119
:100F900090E080E0AA24AA94BA2CC12CD12C1CE2A7
:100FA000E12EFF24F39400E010E00E94212242E0B1
:100FB00050E064E0811184C0D4011496ED91FC915D
:100FC000808183FB992790F9951509F4D2C1982F58
:100FD000907E09F439C1982F907E90528F71892BA1
:100FE000808358C10E9433BC9B01AC014427552724
:100FF000D4011496ED91FC916281738190E080E0C0
:10100000AA24AA94BA2CC12CD12C16E9E12EF12CD9
:1010100000E010E0CACF0E9433BC9B01AC01442722
:101020005527D4011496ED91FC916281738190E073
:1010300080E0AA24AA94BA2CC12CD12C18EEE12E5F
:1010400013E0F12E00E010E00E942122882309F431
:10105000B3CFF4010081118163EB76E0C8010E94F7
:1010600023AE892B41F469EB76E0C8010E9423AEE0
:10107000892B09F488C042E050E068E079CF0E94F3
:1010800033BC9B01AC0144275527D4011496ED9144
:10109000FC916281738190E080E0AA24AA94BA2C2A
:1010A000C12CD12C1CE2E12EFF24F39400E010E0CF
:1010B0000E94212242E050E069E0882309F47CCFBD
:1010C000C4010E94565D0E9433BCD4011496ED9178
:1010D000FC917383628370CF0E9433BC9B01AC018F
:1010E00044275527D4011496ED91FC9162817381B8
:1010F00090E080E0AA24AA94BA2CC12CD12C16E945
:10110000E12EF12C00E010E0D3CF0E9433BC9B0114
:10111000AC0144275527D4011496ED91FC916281CE
:10112000738190E080E0AA24AA94BA2CC12CD12C1F
:1011300018EEE12E13E0F12E00E010E00E942122D3
:10114000882309F439CFF4010081118160EC76E045
:10115000C8010E9423AE892B39F466EC76E0C80101
:101160000E9423AE892B21F042E050E06BE000CFDB
:1011700062EA76E0C8010E9423AE42E050E066E0F9
:10118000892B09F4F5CE42E050E06DE0F1CE0E94EB
:1011900033BC9B01AC0144275527D4011496ED9133
:1011A000FC916281738190E080E0AA24AA94BA2C19
:1011B000C12CD12C1CE2E12EFF24F39400E010E0BE
:1011C0000E942122882309F4F7CE42E050E06CE02F
:1011D00077CF0E9433BC9B01AC0144275527D40133
:1011E0001496ED91FC916281738190E080E0AA24D5
:1011F000AA94BA2CC12CD12C16E9E12EF12C00E0D6
:1012000010E0DECF0E9433BC9B01AC014427552780
:10121000D4011496ED91FC916281738190E080E09D
:10122000AA24AA94BA2CC12CD12C18E5E12E12E0E4
:10123000F12E00E010E00E942122882309F4BCCEA8
:1012400042E050E060E094CE0E9433BCD40114969A
:10125000ED91FC91159773836283E181EF705520C6
:1012600009F445C0E230F1F050F4EE23E9F1D40185
:101270001496ED91FC91808150FA83F9B1CEE5305E
:1012800089F0A3016AE0E73091F7C4010E94565D3E
:101290008111EDCF8091B60981508093B60990E01D
:1012A00080E088C3F401008111816CE976E0C80117
:1012B0000E9423AE892BA9F463EB76E0C8010E945B
:1012C00023AE892B71F469EB76E0C8010E9423AE4E
:1012D000892B39F464E876E0C8010E9423AE892B9B
:1012E00019F0A30166E0D1CFA30161E0CECFE150B8
:1012F000ED3008F0BCCFF0E08827EE57F6478F4F6F
:101300000C941AF18F893789928992893789958946
:101310003789B689B689B689B689B6899289A30113
:1013200062E0B3CFA30165E0B0CF0D911C916CE9F1
:1013300076E0C8010E9423AE892BA9F463EB76E026
:10134000C8010E9423AE892B71F469EB76E0C801D5
:101350000E9423AE892B39F464E876E0C8010E942C
:1013600023AE892B19F0A30167E08FCFA30160E0C2
:101370008CCF8F71806434CEB3E06B16710409F4A6
:101380008ECF6CED76E0F401808191810E9423AED6
:101390008C01D40113968C919091160D8913EBC09A
:1013A0009091170D903409F0E6C08091180D90913E
:1013B000190D3C010115110509F40DC1F801208535
:1013C0002F70253009F007C1C8010E94B2AE382E37
:1013D000F3E0F81708F0DBC063E0C8010E949BAEA1
:1013E000DC0119968D919C913AE0E32EE89E600114
:1013F000E99ED00C1124A396DFAECEAEA39762E097
:10140000C8010E949BAEDC0119968D919C91E89ECB
:101410002001E99E500C11246201052C000CEE08FD
:10142000FF08AF96CCAEDDAEEEAEFFAEAF9761E09B
:10143000C8010E949BAE5C0160E0C8010E949BAEA7
:10144000DC011996CD90DD90ED90FC901C97A7964D
:10145000CCAEDDAEEEAEFFAEA7979301072C000C2D
:10146000440B550B2C193D094E095F09A396CEACD0
:10147000DFACA397B601DD0C880B990BAF96CCAC13
:10148000DDACEEACFFACAF976C197D098E099F09FE
:101490000E947FF0D50119962D913D914D915C915F
:1014A0001C97A796CCACDDACEEACFFACA7972C1983
:1014B0003D094E095F09A7962CAF3DAF4EAF5FAF18
:1014C000A7970E94B1F0AF96ACACBDACCEACDFAC90
:1014D000AF97A20EB31EC41ED51E45E0E42E3E14E7
:1014E00009F468C081E090E0A396EEACFFACA3974E
:1014F000A701FF0C660B770B4A155B056C057D0594
:101500000CF461C0B601A5016201052C000CEE08C7
:10151000FF084C155D056E057F050CF459C06A0186
:101520007B0122E032126BC06301770CEE08FF08EA
:1015300060E0C8010E949BAEFC0181859285A38575
:10154000B485C816D906EA06FB060CF44CC261E065
:10155000C8010E949BAEFC0181859285A385B4855C
:101560008C159D05AE05BF050CF099CE81E090E08D
:10157000A0E0B0E03BC28093160D90E49093170D6D
:101580000E94BCBB9093190D8093180D12CF8AE076
:10159000869D5001879DB00C11240B2C000CCC08AB
:1015A000DD08512C412C20E038E2A3963FAF2EAF4E
:1015B000A39798CF64E0C8010E949BAEDC01199606
:1015C0008D919C9191CF66246A9423E0722E9CCFDA
:1015D000712C612CA6CF2AE0289F6001299FD00C96
:1015E00011240D2C000CEE08FF08512C412C20E09A
:1015F00038E2A3963FAF2EAFA39781E090E0D401ED
:101600001496ED91FC9162817381A301461B570BE7
:1016100057FF03C0519541955109841795070CF464
:10162000BFC08081982F929596959770963008F05C
:10163000BAC09F5F9295990F907E8F71892BB2C02F
:10164000F70161857285DB018C9181115EC2A11465
:10165000B10409F472C0D50118968C9118978F7057
:10166000843009F06AC019966D917C91CE01019683
:101670000E941471CE0101960E94CF68882309F45C
:1016800058C06114710409F45FC0E114F10431F031
:10169000F70180858F70843009F441C025961CAE17
:1016A0001DAE1EAE1FAE259729961CAE1DAE1EAEFA
:1016B0001FAE299723961FAD23971F7023961FAF48
:1016C000239781E022968FAF2297CC24C394F12CEC
:1016D000E12C01E024962FAD249725963FAD259768
:1016E00040E027965FAD279728966FAD28972996FB
:1016F0007FAD2997CE0101960E9485731AC001150E
:10170000110529F0F80180858F70843019F069ED9A
:1017100075E0FBC161857285FB01808196CF618593
:101720007285FB018081882321F0CE0101960E9401
:1017300014B3CE0101960E94A071D4011496ED91CC
:10174000FC9173826282ABCD0115110531F0D80195
:1017500018968C918F708430E9F025961CAE1DAEE2
:101760001EAE1FAE259729961CAE1DAE1EAE1FAE37
:10177000299723961FAD23971F7023961FAF23979A
:1017800082E022968FAF2297CC24C394F12CE12CD7
:1017900002E0A0CFF80161857285DB018C91C3CF97
:1017A00080818F7180838081803AB8F0C201550CAE
:1017B000AA0BBB0BC816D906EA06FB0671F0A39666
:1017C000EEADFFADA397CF01FF0FAA0BBB0BC81661
:1017D000D906EA06FB0609F062CD6616770609F41B
:1017E0005ECD6D961CAE1DAE1EAE1FAE6D976B9698
:1017F0008FAD6B978F7080666B968FAF6B976D9682
:101800008CAD9DADAEADBFAD6D9765968CAF9DAF08
:10181000AEAFBFAF6597AAE0B0E0A70196010E9406
:10182000D0F069966CAF7DAF8EAF9FAF699768E1DE
:1018300076E183EF9DE00E94CC994AE050E0D4012C
:1018400013966C9183EF9DE00E943A9866E176E1F1
:1018500083EF9DE00E94CC99CE018F5A9F4F0E944A
:10186000A43161E275E0F401808191810E9423AE90
:10187000B12CA12CD12CC12C6296EFAC629763964F
:10188000FFAC639764960FAD649765961FAD65973F
:1018900066962FAD669767963FAD679768964FAD92
:1018A000689769965FAD69976FEF0E943B3DD401E1
:1018B0000D911C9162EA75E0C8010E9423AE7C0183
:1018C00067EA75E0C8010E9423AE8C010097E1F140
:1018D000FC0180858F708430B9F56185728540E4A4
:1018E00050E0CE0101960E94A9F56FE270E0CE01B2
:1018F00001960E9470F5892B59F4D80119962D9103
:101900003C9143E050E060E4CE0101960E9418282B
:1019100000E020E032E040E150E0BE016F5B7F4F2D
:10192000CE018F5A9F4F0E94832F0E9441AE882381
:1019300059F08091A807811107C0BE016F5B7F4FEE
:10194000CE0101960E9401BDE114F10409F4F5CE27
:10195000F70180858F70843009F0EFCE6185728544
:10196000CE0101960E941471CE0101960E94CF68AB
:10197000882309F4DECECC24C394F12CE12C6296AA
:101980000FAD629763961FAD639764962FAD649712
:1019900065963FAD659766964FAD669767965FAD66
:1019A000679768966FAD689769967FAD6997A2CE85
:1019B0008FEF9FEFC259DF4F0FB6F894DEBF0FBE17
:1019C000CDBFDF91CF911F910F91FF90EF90DF90EE
:1019D000CF90BF90AF909F908F907F906F905F90CF
:1019E0004F903F90089580E090E0DC01F401248165
:1019F0003581F90142815381052E000C660B770B6E
:101A000084179507A607B70709F449CC3C01D40110
:101A10000D911C9162EA75E0C8010E9423AE5C0141
:101A200067EA75E0C8010E9423AE6C01A114B104FD
:101A300019F4892B09F481CE67E976E0C8010E9488
:101A400023AE7C0162E976E0C8010E9423AE8C01DE
:101A50006EE176E183EF9DE00E94CC994AE050E090
:101A6000F401638183EF9DE00E943A986CE176E196
:101A700083EF9DE00E94CC99B30183EF9DE00E942B
:101A8000AAAE83EF9DE00E943698C114D10409F4F8
:101A9000DECDD60118968C9118978F70843009F09E
:101AA000D6CD19966D917C9140E450E0CE0101961F
:101AB0000E94A9F50E9441AE882309F4C8CD809107
:101AC000A8078111C4CD6FE270E0CE0101960E949B
:101AD00070F5892B51F4F6012185328543E050E001
:101AE00060E4CE0101960E9418286114710409F483
:101AF00006CEE114F10439F0D70118968C918F705D
:101B0000843009F49DCD6EEC75E0CE0101960E9403
:101B100001BD9DCDEF92FF920F931F93CF93DF9363
:101B2000EC018B011D821C821A821B82E880F980E5
:101B3000E114F10409F45DC08091A6079091A70714
:101B4000892B09F456C0672B09F48701F8018085B9
:101B50008F708630A9F460EE76E0C8010E9423AE53
:101B6000009719F0FC0181858A836BE777E0C80153
:101B70000E9423AE009709F443C0FC0181858B834A
:101B800062EE76E0C7010E9423AE009779F561E12D
:101B900076E183EF9DE00E94CC994AE050E06B81B2
:101BA00083EF9DE00E943A986FE076E183EF9DE03D
:101BB0000E94CC994AE050E06A8183EF9DE00E9448
:101BC0003A9883EF9DE00E94369820E030E0A9012A
:101BD00062EE76E0888199810E9440B262EE76E002
:101BE000888199810E9423AE009719F009969D8300
:101BF0008C83DF91CF911F910F91FF90EF9008950B
:101C0000F801808191810E94E4E8B9CFFC0161155F
